:1000000000600020A548030805E5020819E502087C
:100010002DE5020841E5020855E502080000000050
:1000200000000000000000000000000069E5020878
:100030007DE5020800000000B55A00087BE80008D2
:10004000A14B0308A54B0308A94B03081FEB0208AB
:10005000B14B030887EC0208D1E7020861E9020806
:10006000EDE90208C54B0308C94B0308CD4B030853
:10007000D14B0308D54B0308D94B0308DD4B0308CC
:10008000E14B0308E54B0308E94B0308ED4B03087C
:10009000F14B0308F54B0308F94B0308FD4B03082C
:1000A000014C0308054C0308094C03080D4C0308D8
:1000B000114C0308154C0308194C03081D4C030888
:1000C000214C0308254C0308294C030895E5020838
:1000D000314C0308354C0308394C03083D4C0308E8
:1000E0008BEA0208EBEB0208494C03084D4C03086D
:1000F000514C0308554C0308594C03085D4C030848
:10010000614C0308654C0308694C03086D4C0308F7
:10011000714C0308754C0308794C03087D4C0308A7
:10012000814C0308854C0308894C03088D4C030857
:10013000914C0308954C0308994C03089D4C030807
:10014000A14C0308A54C0308A94C0308AD4C0308B7
:10015000B14C0308B54C0308B94C0308BD4C030867
:10016000C14C0308C54C0308C94C0308CD4C030817
:10017000D14C0308D54C0308D94C0308DD4C0308C7
:10018000E14C0308E54C030838B50020ADF8000049
:10019000044601F094FF05464FF48051204602F0DA
:1001A000F2F90A21284602F077F900E0641C062CD7
:1001B00012D2DFF8FC0C215C8DF800102018007AB8
:1001C0008DF80100022300AA7221072002F06FF8C7
:1001D0000028EBD1002032BD012032BD2DE9FC41C9
:1001E0000746884602F030FB04460020ADF80400C4
:1001F000DFF8C05C288C0646B8F1000F02D0384307
:10020000288401E0B8432884012000900DF1060302
:10021000AB227221062002F0A4F8002801D10020B0
:10022000C4E1288C0E2800F2A681DFE810F00F0050
:10023000A4011C00A4013F00A4013F00A401B700D9
:10024000A401B700A401B700A401B70080208DF875
:10025000040000208DF805009DF8060000F0FD0068
:100260008DF8060087E116F00C0F01D001206875AB
:1002700081208DF8040001AEEE207070022301AAE7
:100280007221092002F013F8002801D100208DE12D
:100290007078E87080208DF80400032070709DF85D
:1002A000060000F0FD008DF8060064E1304600070E
:1002B00001D4022E01D1012068759D208DF8040023
:1002C00001AE0C207070022301AA7221092001F0F6
:1002D000EEFF002801D1002068E19E208DF8040087
:1002E0000C207070022301AA7221092001F0DFFFA7
:1002F000002801D1002059E181208DF80400FD2063
:100300007070022301AA7221092001F0D0FF002899
:1003100001D100204AE17078E8708E208DF8040049
:10032000287A002812D00C218F2002F05EFB0421D5
:100330008F2002F031FB3021902002F056FB30215B
:10034000902002F029FB4520707011E00C218F20D5
:1003500002F04BFB08218F2002F01EFB3021902081
:1003600002F043FB1021902002F016FB82207070F7
:10037000022301AA7221092001F099FF002801D16E
:10038000002013E180208DF80400272070709DF874
:10039000060000F0FD008DF80600ECE016F00807FE
:1003A00001AE4FD102F02AFC01206875A4208DF81F
:1003B000040000207070DFF87C0D00210170022322
:1003C00001AA7221092001F072FF002801D100204A
:1003D000ECE0A5208DF8040000207070DFF8580DC7
:1003E00000210170022301AA7221092001F05FFFA0
:1003F000002801D10020D9E0A7208DF804000020BA
:100400007070DFF8A80D00210170022301AA72218B
:10041000092001F04CFF002801D10020C6E0A920EE
:100420008DF8040000207070DFF8840D0021017049
:10043000022301AA7221092001F039FF002801D10D
:100440000020B3E081208DF80400FE2070700223AC
:1004500001AA7221092001F02AFF002801D1002001
:10046000A4E07078E8708E208DF80400287A0028C7
:1004700012D00C218F2002F0B8FA04218F2002F054
:100480008BFA3021902002F0B0FA3021902002F057
:1004900083FA4F20707011E00C218F2002F0A5FA32
:1004A00008218F2002F078FA3021902002F09DFA86
:1004B0002121902002F070FA84207070022301AA9A
:1004C0007221092001F0F3FE002801D100206DE027
:1004D000002F20D1B4F88A00B4F88C10401AE883B9
:1004E000B4F88A108900A98389B2FF2901D3FE21BB
:1004F000A98380B28100652902DB6420E88301E0E2
:100500008000E883A98BE88B0A1AEA8392B20FF283
:10051000A00001F056FEA6208DF80400287A0028DD
:100520000AD06021A32002F060FA4121A32002F04A
:1005300033FA5720707009E06021A32002F055FAC9
:100540004121A32002F028FA8B207070022301AA17
:100550007221092001F0ABFE002801D1002025E026
:1005600080208DF80400672070709DF8060040F030
:1005700002008DF80600022301AA7221092001F071
:1005800096FE002801D1002010E0AB208DF8040079
:100590009DF806008DF80500022301AA72210920AA
:1005A00001F085FE401E8041C043C00FBDE8F681CA
:1005B000233E6755703D25642C674C6F3D256400D4
:1005C00010B534220021DFF8900C02F0A1FEDFF814
:1005D000E4480120A07102F0A5FE02F02FFA0120EC
:1005E0002073DFF8EC0D0021017010BD10B582B052
:1005F0000FF25C0001F0E5FD0020ADF80000802066
:100600008DF8000000AC03206070022300AA722164
:10061000062001F04CFE002818D0DFF89808817AF7
:1006200000290DD08C218DF800100021617081709F
:10063000022300AA7221062001F039FE002805D00D
:10064000FFF7BEFF01210020FFF7C8FD13BD00002A
:10065000233E484C5300000010B582B00FF240001A
:1006600001F0AFFD0020ADF80000044600E0641C7E
:10067000052C12D2DFF85C0D215C8DF800102018DB
:10068000007A8DF80100022300AA7221072001F0F0
:100690000EFE0028EBD1002016BD012016BD000083
:1006A000233E50525000000030B583B00FF284005A
:1006B00001F087FD0020ADF804008DF80600DFF89A
:1006C000F447607180208DF8040001AD032068704C
:1006D000022301AA7221072001F0E9FD002801D1BF
:1006E00000203EBD8C208DF8040000206870A070B2
:1006F000022301AA7221072001F0D9FD002801D1AF
:1007000000203EBD0120607201460420FFF766FD17
:10071000002801D100203EBD012000900DF106030C
:10072000E5227221072001F01CFE401E8041C043DB
:10073000C00F3EBD233E50524F00000000B583B0B5
:100740000FF2600001F03DFD0020ADF806008DF8CD
:10075000040080208DF8060003208DF80700022396
:100760000DF106027221072001F0A1FD002801D140
:1007700000200EBDDFF83C07002141720420FFF786
:100780002DFD002801D100200EBD0120009001ABFD
:10079000E5227221072001F0E4FD401E8041C043A4
:1007A000C00F0EBD233E5052430000000120704791
:1007B00030B583B004460020ADF80400DFF8F456ED
:1007C000A87B00282CD1A87A002802D0287C207091
:1007D00031E0012000900DF10503932272210720E2
:1007E00001F0BFFD00280DD09DF80500800722D53F
:1007F0000120009001AB9C227221072001F0B1FD85
:10080000002801D100203EBD9DF80400697951FA0D
:1008100080F080B2400820709DF8040068710AE002
:10082000012808D1DFF8300A41696A79891849102E
:1008300021704069687101203EBD2DE9F04391B0FF
:10084000044602F001F8054601F039FC0646002096
:10085000ADF80800ADF80C008DF80A0001200090FA
:100860000DF10A0393227221072001F07AFD00287E
:1008700001D1002024E20220009003AB94227221D7
:10088000072001F06EFD002801D1002018E2DFF8FA
:1008900024769DF80D009DF80C1041EA0020DFF849
:1008A0000C1D4843F978C1F580713A79DFF8003DB5
:1008B000D25C12FB01F140F24232514390FBF1F065
:1008C000797B002902D0B97A002901D1B86208E009
:1008D000B86AF97D4A1CFA75062902D3002179739A
:1008E000F975397A00290CD141F6593188422DDB4E
:1008F00001213972F86200203876FFF777FE012077
:10090000DEE1F96A411A44F62162914215DA40F6B5
:10091000B831884218DA9DF80A20920614D53A7E3A
:10092000531C3B76C92A04D2BA7A002A0ED18842D7
:100930000CDA884201DA00213972F8620020387638
:10094000FFF754FE0120BBE1002038769DF80A0035
:10095000800640F1B4810020B873012000900DF1B1
:100960000A0393227221072001F0FBFC002801D129
:100970000020A5E19DF80A0080071BD5012000900A
:1009800003AB9C227221072001F0EBFC002801D16F
:10099000002095E19DF80C00797951FA80F080B241
:1009A000400860709DF80C00F8739DF80C00787199
:1009B00060783874387B002802D00020387371E1E9
:1009C000DFF8108D607888F80000B87900280AD028
:1009D00002F03EF8002806D1B87A002803D06078EB
:1009E00002F048F87AE0787A002839D0B87AB978F5
:1009F000084335D1002030758C208DF808000DF1AA
:100A00000809202089F80100B870022302AA722187
:100A1000072001F04CFC002801D1002050E1892082
:100A20008DF80800002089F80100022302AA722133
:100A3000072001F03CFC002801D1002040E18B2080
:100A40008DF80800B5F88A0089F80100022302AA8F
:100A50007221072001F02BFC002801D100202FE19A
:100A6000B87A00280ED105F18A004288B5F88A10BC
:100A70000FF2542001F0A5FB61780FF25C2001F029
:100A8000A0FB2BE0414684B06846182203F048F8EA
:100A90000FBC02F058FC04A802F0BBFCDFF8B49CC9
:100AA000484604A9342203F03BF899F81C000028BA
:100AB00007D034224946DFF8A00703F05CF8012094
:100AC000787009F11C00417D88F81410817D88F848
:100AD0001510007D002801D0FFF772FD787A0028FC
:100AE00000F0E080B87A002840F0DC806078B5F84B
:100AF0008A10884231D3307D00282ED10120F87130
:100B000020702078307589208DF808000DF10809D3
:100B100005F18A00408889F80100022302AA7221A7
:100B2000072001F0C4FB002801D10020C8E08B2081
:100B30008DF80800FF2089F80100022302AA722123
:100B4000072001F0B4FB002801D10020B8E0617853
:100B50000FF2901001F035FBA4E005F28A00418805
:100B60006278914231D3317D01292ED10120F87173
:100B7000002020702078307589208DF808000DF154
:100B80000809002089F80100022302AA7221072027
:100B900001F08DFB002801D1002091E08B208DF821
:100BA0000800B5F88A0089F80100022302AA722120
:100BB000072001F07CFB002801D1002080E0617853
:100BC0000FF2281001F0FDFA6CE0B5F88A10627897
:100BD000914235D3317D002932D1797C01292FD141
:100BE0000120F87100202070207830750020787482
:100BF00089208DF808000DF10809002089F801000E
:100C0000022302AA7221072001F051FB002801D122
:100C1000002055E08B208DF80800B5F88A0089F88F
:100C20000100022302AA7221072001F040FB0028E4
:100C300001D1002044E00FF2BC0001F0C2FA31E023
:100C40006178428891422DD3317D01292AD1797C66
:100C5000012927D10021797489218DF808100DF11F
:100C60000809408889F80100022302AA722107209E
:100C700001F01DFB002801D1002021E08B208DF820
:100C80000800FF2089F80100022302AA7221072030
:100C900001F00DFB002801D1002011E00FF25C00F3
:100CA00001F08FFA0120009003ABE52272210720AA
:100CB00001F057FB401E8041C043C00F00E0002000
:100CC00011B0BDE8F0830000233E55703D25642C33
:100CD0004C6F3D2564000000233E505241572025B3
:100CE00064000000233E503120256400233E503232
:100CF00020256400233E526554483100233E52654E
:100D0000544832002DE9F84304460D46694EB07C44
:100D1000002805D000F011FF0020F0743075C5E008
:100D200001F092FD804600273846ADF8000020789B
:100D3000072823D16078FF2820D12946601CFFF7BF
:100D400037FD6078B8F88A10884208D301202070F7
:100D5000627821780FF2601001F033FA0CE0B8F8F5
:100D60008C006178884207D33846207062782178F9
:100D70000FF2441001F025FA012097E00020F074F2
:100D8000307529462046FFF758FD00280DD0707AAF
:100D900000280AD0F079002807D00FF2301001F0B7
:100DA00010FA0020F07101203075B07A002877D059
:100DB000DFF84C8DD8F8189009F10C00417DC0681F
:100DC000D9F80C20801800F049FA002868D0DFF824
:100DD00000060078411E8941C90FF174707800281F
:100DE00001D000207070707A002857D0D9F80C001C
:100DF00040780DF1000989F80100B18B814218D2C9
:100E000001F05DF9007D002813D1707E401C7076E2
:100E1000C0B202282DD100207076012701F04FF9D1
:100E20003946017599F801100FF2A80001F0C9F9CF
:100E30001FE099F80100F18B884218D201F03FF9C8
:100E4000007D012813D1707E401C7076C0B202284C
:100E50000FD100207076012701F031F900210175D2
:100E600099F801100FF2780001F0ABF901E00020D1
:100E70007076002F12D0D8F81C8001F020F9007D88
:100E80008DF8000008F10C00427D00A9C068D8F878
:100E90000C30C01802F06FFE012030750020307059
:100EA00003F0F2FE00283FF469AF307DBDE8F28325
:100EB000B09A0020C8990020233E536C65657020CD
:100EC000414443202564202564000000233E505502
:100ED00050000000233E677570312025640000003B
:100EE000233E67757032202564000000F8B5074680
:100EF0000020ADF8000001F0A7FC0546DFF8104D1A
:100F0000012060743878A5F88A0005F28A0678789E
:100F10007080B5F88A00002802D07088002808D1B7
:100F20000FF2940001F04DF97820A5F88A00002016
:100F3000708089208DF8000000AF708878700223DF
:100F400000AA7221072001F0B2F900280DD08B20F1
:100F50008DF80000B5F88A007870022300AA72218B
:100F6000072001F0A4F9002801D10020F2BD728809
:100F7000B5F88A100FF2480001F023F9B5F88A009D
:100F80007188401AE083B5F88A108900A18389B27C
:100F9000FF2901D3FE21A18380B28100652902DBF4
:100FA0006420E08301E08000E083A08BE18B401AA5
:100FB000E0830120F2BD0000233E5054483D300044
:100FC000233E5448534554202564202564000000E6
:100FD00080B50FF21801072004F0C0FA0FF23001BB
:100FE0000A20BDE8044004F0B9BA00005906000820
:100FF000A90600083D070008AD0700080000000032
:10100000050D0008ED0E00080000000000000000C3
:1010100059060008A90600083D070008AD070008AA
:1010200000000000B1070008ED0E000800000000FD
:101030000000000010B582B00FF2540001F0C1F8BA
:101040000020ADF80000FFF79FF8002803D10FF251
:10105000480001F0B6F8002400E0641C0B2C12D20A
:10106000DFF87C0D2118097B8DF80010205C8DF8CD
:101070000100022300AA7221062001F018F90028BD
:10108000EBD1002016BD03F033F8012016BD00009F
:10109000233E474550000000233E47504641494CFF
:1010A0000000000038B50FF2940001F08AF800202B
:1010B000ADF8000080208DF8000000AC03206070C7
:1010C000022300AA7221062001F0F1F8002801D1C4
:1010D000002032BD8C208DF8000000206070DFF809
:1010E000305BA870022300AA7221062001F0DFF80D
:1010F000002801D1002032BDA3208DF80000DFF8C8
:10110000E00CC0786070022300AA7221062001F072
:10111000CEF8002801D1002032BD0120A872FFF7CF
:101120004FFA01210820FFF759F8401E8041C043C3
:10113000C00F32BDEF620120F0620120233E47451F
:101140004F00000010B582B00FF2680001F039F8CE
:101150000020ADF8000080208DF8000000AC0320D6
:101160006070022300AA7221062001F0A0F8002876
:1011700001D1002016BDDFF86C0C0021817208201F
:10118000FFF72CF8002801D1002016BD9F208DF814
:10119000000000206070022300AA7221062001F0E6
:1011A00086F8401E8041C043C00F16BDF162012089
:1011B000F2620120233E47454300000001207047B2
:1011C00030B58DB0DFF8485AA879002814D001F066
:1011D0003FFC002810D0DFF8FC44201D0FC801F0B0
:1011E00035FD01F03EFC002832D00020A87101201E
:1011F00060752075A0752BE0A879002828D1DFF84C
:10120000D444214684B06846182202F089FC0FBC01
:1012100002F0CCF800A802F0FCF8DFF838552846B8
:1012200000A9342202F07CFC05F11C00417D2175EF
:10123000817D6175007D002801D0FFF7C1F9287F0D
:10124000002805D034222946DFF8FC0C02F093FC7C
:1012500001200DB030BD00003C5F012010B584B00E
:10126000044602A8002101600846ADF804000120F0
:10127000009001AB93227221062001F072F8002841
:1012800000F088809DF8040010F0040004D1DFF81D
:101290008019497800297DD0002806D0DFF8700930
:1012A0004178002901D101218173012000900DF1C5
:1012B0000503AE227221062001F053F8002869D000
:1012C0009DF80500002817D00420009002ABFC22F6
:1012D0007221062001F045F800285BD0DFF8F40306
:1012E0009DF80810416002A94A7882608A78C2603D
:1012F000C9780161FFF764FFDFF84C1C0A78DFF85A
:1013000010094378002B227007D000226270A2706F
:10131000E27022716271A2710BE04A6962708A699F
:10132000A2704A68E2708A682271CA6862710A69AA
:10133000A2710A6AE2714A6A22728A6A6272CA6A8F
:10134000A2724A7FE272DFF8042C12782273DFF86F
:10135000002C12786273DFF8FC2B1278A273DFF88E
:10136000F82B1278E273DFF8F42B12782274DFF88E
:10137000F02B12786274DFF8EC2B1278A274C27B27
:10138000E274002202700878042801D11046087027
:10139000012000E0002004B010BDDFF8480AC07C46
:1013A000704780B5052802D1084600F002F80120F8
:1013B00002BD80B5017841F04103DFF8AC1BCB7072
:1013C000027801780FF6C03000F0FBFE012002BD6C
:1013D0008E660120C09A002070B584B004460020BB
:1013E000019002A8002101600E460FF6B03000F017
:1013F000E8FE01210820FEF7F1FEA0208DF8040090
:1014000001AD30466870022301AA7221062000F067
:101410004EFF002801D13046C5E0A1208DF8040020
:10142000FF206870022301AA7221062000F03FFF0E
:10143000002801D13046B6E0AB208DF80400012031
:101440006870022301AA7221062000F030FF0028F4
:1014500001D13046A7E0012000900DF10603802263
:101460007221062000F07DFF002801D130469AE06D
:1014700080208DF804009DF8060040F0450068705B
:10148000022301AA7221062000F011FF002801D1D9
:10149000304688E0A3208DF80400DFF84409C078C6
:1014A0006870022301AA7221062000F000FF0028C4
:1014B00001D1304677E0012000900DF10703AF2203
:1014C0007221062000F04DFF002801D100206AE0C3
:1014D0009DF80700C0070BD50420009002ABFC224A
:1014E0007221062000F03DFF00280CD100205AE0B8
:1014F0003046461CB0F57A7FDDDB0FF6A82000F001
:1015000060FE00204FE09DF80800207002A841789E
:1015100061708178A170C078E070012000900DF1B9
:10152000060380227221062000F01BFF002801D153
:10153000002038E080208DF80400DFF8A808417A08
:10154000002905D09DF8060000F0BF0068700CE08F
:101550009DF8061001F0BB016970C07A002804D123
:101560009DF8060000F0BA006870022301AA7221FB
:10157000062000F09CFE002801D1002013E0AB20E3
:101580008DF8040000206870022301AA7221062051
:1015900000F08DFE002801D1002004E00021082089
:1015A000FEF71CFE012004B070BD0000D8D0010081
:1015B000402000080FF68C21062003F0CFBF1CB599
:1015C0000FF6EC1000F0FDFD00208DF80400ADF8E2
:1015D0000600044600E0641C052C13DADFF88C09D1
:1015E000215C8DF806102018007A8DF80700022380
:1015F0000DF106027221092000F059FE0028EAD1FF
:10160000002016BD0120009001ABD62272210620D9
:1016100000F0A7FE002801D1002016BD9DF804109F
:101620000FF6941000F0CDFDDFF8B8079DF8041018
:10163000C9098176012016BD30B583B0DFF8A44713
:10164000A07E002804D00FF6801000F0BAFD03E061
:101650000FF67C1000F0B5FD0020ADF804008020EE
:101660008DF8040001AD03206870022301AA7221E5
:10167000092000F01CFE002801D100203EBD8F2073
:101680008DF804000B206870022301AA7221092042
:1016900000F00DFE002801D100203EBD0320207186
:1016A0000120A075E07201460220FEF797FD002898
:1016B00001D100203EBD012000900DF10603E6227D
:1016C0007221092000F04DFE401E8041C043C00F32
:1016D0003EBD00005C62012000B583B00FF6F8004B
:1016E00000F06FFD0020ADF8060080208DF80600A8
:1016F00003208DF8070002230DF106027221092054
:1017000000F0D5FD002801D100200EBD0120009081
:1017100001AB8F227221092000F023FE002801D1A5
:1017200000200EBDDFF8BC060021C1720220FEF7CA
:1017300055FD002801D100200EBD0120009001AB15
:10174000E6227221092000F00CFE401E8041C043B9
:10175000C00F0EBD705F0120012070472DE9F041E0
:1017600084B004460020ADF804000290DFF8900336
:10177000456A002085F85E00DFF86866B07D0128C4
:1017800003D0707D002840F090800220009001ABD3
:1017900094227221092000F0E4FD00282DD09DF84C
:1017A0000400A07101AF7878E0710220009001ABD5
:1017B00096227221092000F0D4FD00281DD09DF84A
:1017C00004002070787860700220009001AB9822AD
:1017D0007221092000F0C5FD00280ED09DF80400FC
:1017E000A0707878E0700220009001AB9A227221FC
:1017F000092000F0B6FD002801D1002097E09DF8F7
:101800000400207178786071F0782072307960720D
:101810006078217841EA0020E178A27842EA01214B
:101820006279237943EA0222E379A77947EA03231D
:1018300002AF009700F0CCF800281BD1B07D012842
:1018400034D10020B075DFF828075B21017000213A
:101850004170852181700021C170AE21017100218C
:101860004171702181710121C171EE21017200214C
:1018700041721BE00020B075DFF8F406217801709A
:1018800061784170A1788170E178C170217901712E
:1018900061794171A1798171E179C171217A017216
:1018A000617A41720298706238E037D0DFF8C00682
:1018B00001782170417861708178A170C178E17000
:1018C00001792171417961718179A171C179E171E8
:1018D000017A2172407A60720020707560782178F8
:1018E00041EA0020E178A27842EA01216279237975
:1018F00043EA0222E379A77947EA0323F77894F8C9
:1019000008C086F803C096F80480647A347102AC8B
:10191000009400F05DF8F77086F80480029840F6B5
:101920008451884202D1012085F85E00012004B074
:10193000BDE8F0811CB504460020ADF806008DF826
:1019400004000120009001AB8F227221092000F0D9
:1019500008FD002801D1002016BD9DF8040000F00C
:10196000FC008DF80400012C0AD0042C04D0102CAB
:101970001FD0402C22D026E040F001008DF804005A
:101980008F208DF806009DF804008DF80700DFF821
:1019900054449DF8040000F00300207102230DF16F
:1019A00006027221092000F082FC00280DD10020DF
:1019B00016BD40F002008DF80400E1E740F003009E
:1019C0008DF80400DCE7002016BD0120607316BD11
:1019D0002DE9F04105460E46174670193818C01A11
:1019E000401C441024B2002C00D50024DFF8F4136E
:1019F00008790FF24C62805CC978C1F5807110FBE8
:101A000001F240F6DC2C0CFB02F88902B1F5803FB4
:101A100001D34FF6FF71C9000A22B1FBF2F1102881
:101A20002DD18B422BD30120FFF784FF00283ED11C
:101A3000311B0698AC4206DA02682B1B4FF4B475D2
:101A400005FB03220260B44205DA02684FF47A73A0
:101A500003FB01210160BC4201DA016801600168F9
:101A6000002901D50021016040F2A641B8FBF1F147
:101A70000268B2FBF1F101600120BDE8F08110289D
:101A800007D1642B05D24020FFF754FF00280ED168
:101A9000CEE7402802D164398B4203D20128C7D156
:101AA000642BC5D21020FFF745FF0028C0D00020CE
:101AB000E3E70FF2B451092003F050BDC94988741F
:101AC0000120704710B5DFF8AC44202020700020C2
:101AD00060700A20A0700020E0700A2020710020B1
:101AE00060713220A0710020E07207222146DFF8E9
:101AF000880402F040F800206072012010BD000050
:101B00000060002000B583B000A800210A4606C08E
:101B10000722DFF860140DF1010002F02CF8A0207C
:101B20008DF80000082300AA7221072000F0BFFBF7
:101B3000401E8041C043C00F0EBD00B583B00020E1
:101B40008DF80400DFF82C04417B012903D100F05B
:101B5000AAF901200EBD418AFF290CD000290DD021
:101B6000C27A521CC272491E4182417AD2B291425B
:101B700001D20021C17200F014F805E0818A41828F
:101B80000021C17200F00DF80120009001ABE322AA
:101B90007221072000F0E5FB401E8041C043C00FCA
:101BA0000EBD38B50020ADF80000DFF8C843608AEC
:101BB000002801D1A07A60720722E07AC0EBC00051
:101BC000DFF8B4134118204601F0D5FFFFF79AFF64
:101BD00080208DF8000000AD81206870022300AAEB
:101BE0007221072000F063FB002801D1002032BDE4
:101BF000A7208DF80000208A6870022300AA7221B5
:101C0000072000F054FB401E8041C043C00F32BD8E
:101C1000C899002030B585B0044600208DF80C002E
:101C2000ADF80E006079029020790190E078009084
:101C3000A378627821780FF2A83000F0C2FA012070
:101C4000009003AB80227221072000F08AFB00285D
:101C500001D1002061E0C74D9DF80C0028720120E1
:101C6000009003AB8F227221072000F07AFB00283E
:101C700001D1002051E09DF80C00A87301200090D4
:101C800003AB90227221072000F06BFB002801D1EA
:101C9000002042E09DF80C00E87300F0A5F88F20CA
:101CA0008DF80E000DF10E050B20687002230DF16A
:101CB0000E027221072000F0FAFA002801D100205C
:101CC0002BE090208DF80E000120687002230DF1AA
:101CD0000E027221072000F0EAFA002801D100204C
:101CE0001BE0A64D8122FF21284601F011FB802236
:101CF0002146681C01F03FFF0020287081232A46FE
:101D00007221072000F0D3FA002805D10FF2E82055
:101D100000F057FA002000E0012005B030BD80B58A
:101D200001780F2904DA934A527A521C8A4205DA62
:101D30000FF2D02000F045FA002002BD4278202AA0
:101D400001D3202242700022C2704271C1EBC10156
:101D5000894A20238B54891800224A704278002A2D
:101D600001D1002201E05200521E8A7182788A70ED
:101D7000C278CA7002790A7140794871012002BDA7
:101D80007C48417A491C417281720120704738B504
:101D90000446784D6C82FFF795FE002C00D0AC8293
:101DA00021460FF2702000F00CFA012032BD71497B
:101DB00048730120704772490870012070477048CD
:101DC0000078704780B56B4908730A7B52000A821D
:101DD00001460FF2502000F0F4F9012002BD00008E
:101DE000489A0020C899002000B583B00020ADF8C3
:101DF00006008DF8040080208DF8060001208DF883
:101E0000070002230DF106027221072000F04FFAAD
:101E1000002801D100200EBD10200090594BA022B7
:101E20007221072000F09DFA002801D100200EBD8C
:101E30000120009001AB80227221072000F091FA6E
:101E4000401E8041C043C00F0EBD00B587B00020CA
:101E5000ADF8000001A8142103F0CCFD80208DF81E
:101E6000000001208DF80100022300AA7221072042
:101E700000F01DFA002801D1002012E01022414993
:101E80000DF1050001F077FEA0208DF8040011236C
:101E900001AA7221072000F00AFA401E8041C043C7
:101EA000C00F07B000BD30B583B00020ADF804000E
:101EB0008DF806002F4C217A0FF2781000F081F98E
:101EC0000020FFF7FBFD002060736072FFF7BDFF8D
:101ED0008F208DF8040001ADA07B6870022301AA59
:101EE0007221072000F0E3F9002801D100203EBD57
:101EF00090208DF80400E07B6870022301AA722113
:101F0000072000F0D4F9002801D100203EBD802038
:101F10008DF80400207A6870022301AA722107203C
:101F200000F0C5F9002801D100203EBD012000903D
:101F30000DF10603E3227221072000F012FA401E81
:101F40008041C043C00F3EBD3C5F01207C63012047
:101F5000EF620120F0620120F1620120F2620120B3
:101F60007D6301207E630120489A0020D09A0020E2
:101F700070640120D4620120085401203C4F0120EC
:101F80008D66012090630120233E47452043552064
:101F9000257820257820257800000000233E47532F
:101FA000454C4600233E4753544552520000000022
:101FB000233E4C4947500000233E4C4348495020A3
:101FC0003078257800000000233E3E4C49474F0002
:101FD000233E4C49474F0000233E4C4947430000F5
:101FE0004D4244202564202564202564202564205A
:101FF00025642025640000004D6F6265616D2057E7
:10200000460000004D6F6265616D20486F7020468C
:1020100061696C004D4220486F70436F756E74208B
:10202000256400004D6F6265616D204C656E3D2535
:10203000640000004D4220436C6F736520256400EE
:102040000104104035100008A510000845110008D3
:10205000BD110008000000009B13000800000000F4
:10206000D9130008A3130008BF150008391600088B
:10207000D916000859170008000000005D17000875
:10208000000000000000000000000000BFF34F8FC0
:10209000DFF81807016801F4E061DFF84027114319
:1020A0000160BFF34F8FFEE710B5DFF834474FF400
:1020B0008E720021204601F02BF9204610BDDFF87A
:1020C0002007704710B5FFF7EFFF044600231A46BC
:1020D0001146084600F06FFAC046C04601F062FDA6
:1020E000204600F019F801F0B4FF204600F0D0F9C6
:1020F000204600F015F8204600F01FF800F093F994
:1021000000206072A072E0722073012060730020D2
:10211000E075A073012010BD0021C171017231E092
:1021200010B50446DFF8880601F0E8FDDFF8B406D4
:1021300001F0E4FD0120607110BD10B5044601F00E
:1021400048FE0120A07110BD38B50446012501F0FC
:10215000F3FE012804D12846E0700020A0700AE0B8
:10216000022804D10020E0702846A07003E000207F
:10217000E070A0700546284632BD80B502F05AF8DE
:10218000012002BD10B50446E07902F091F9012169
:10219000217010BD70B504460025E679E171FFF7A6
:1021A000F1FF002807D02046FFF7BAFF2046FFF7CF
:1021B000C4FF012503E0E6712046FFF7E3FF284650
:1021C00070BD0EB470B5C1B0054600A84FF4807163
:1021D00003F010FCFFF773FF044645AB2A464FF4AB
:1021E000807100A803F016FC00A803F031FC451C28
:1021F00000A82818002100F8011CDFF8EC653078F1
:10220000401C30707078F021084202D0992003F011
:102210003FFC03F0AAFC7078401C7070207E2818E8
:10222000FF2810DA207E002803D0207E00190A2122
:1022300001762A4600A9207E0019193001F09BFC86
:10224000207E2818207600A803F0F7FE7078F02191
:10225000084202D0992003F01BFC7078401E707079
:10226000C0B2002801D103F07AFC04F0D4FA41B0E6
:1022700070BC5DF810FB0428DFF8380503D8DFF8E0
:10228000301501607047DFF85C1501607047DFF8BA
:10229000281551F82000007F002807D0DFF84C05F2
:1022A00001784A1C0270032900D3EFE670472DE93C
:1022B000F84305460E4617464FF00208DFF828455A
:1022C0006078F021084202D0992003F0E1FB03F08E
:1022D0004CFC6078401C60709DF80000401E8DF83A
:1022E000000017F8019B2846FFF7C5FF00AB4A46E0
:1022F0003946304602F0F4F9002810D06078F02119
:10230000084202D0992003F0C3FB6078401E607041
:10231000C0B2002801D103F022FC01201FE05FFAC7
:1023200088F8424629460FF2D040FFF74AFF404660
:10233000A0F101080028D9D16078F021084202D02C
:10234000992003F0A5FB6078401E6070C0B20028A1
:1023500001D103F004FC2846FFF799FF0020BDE8F7
:10236000F2832DE9F04704460D4616461F460898AD
:10237000DFF8488488F80000DFF86C9499F80100D1
:10238000F021084202D0992003F082FB03F0EDFB1C
:1023900099F80100401C89F801002046FFF76BFF07
:1023A0004FF0020A434632463946284602F048FAC0
:1023B000002813D099F80100F021084202D099209A
:1023C00003F066FB99F80100401E89F80100C0B2D5
:1023D000002801D103F0C3FB012022E05FFA8AFA52
:1023E000524621460FF21C40FFF7EBFE5046A0F18B
:1023F000010A0028D6D199F80100F021084202D044
:10240000992003F045FB99F80100401E89F801006E
:10241000C0B2002801D103F0A2FB2046FFF737FF2E
:102420000020BDE8F08703F010BAF8B50446022793
:102430000025DFF884630DE039464F1EC9B200293C
:102440000AD1002804D120690121A94088432061D4
:1024500002276D1C162D10DA56F82500006E006854
:1024600080470128E8D121690122AA401143216156
:1024700056F8251001220A77E3E72069032803D0E4
:10248000022801D0012802D140F480502061F1BD22
:1024900002F01EBB02F077BB81B00022ADF8022033
:1024A000ADF80020C079042808D0062809D00828F3
:1024B0000AD009280BD00A280CD00EE04FF4C860CF
:1024C0000DE04FF448600AE04FF4C85007E04FF4C5
:1024D000FA5004E042F2107001E041F27070ADF881
:1024E00002200DE0BDF80020521CADF80020BDF820
:1024F00000208242F6DBBDF80220521CADF802201B
:10250000BDF802208A4203D20022ADF80020EEE797
:1025100001B07047417230B589B004F097FA0446B3
:10252000FFF7CDFD054600A8242103F063FA002043
:10253000ADF8220001900A208DF8080000208DF8E7
:1025400009008DF80A00687A00280DD0002C18D0F8
:1025500000208DF80000052001900B208DF8080068
:1025600000A806F0CBFA0CE0002C0AD001208DF870
:102570000000052001900B208DF8080000A806F04F
:10258000BDFA09B030BD02F01ABB02F022BB012136
:102590000846F8E701210846F7E702210120F2E7A3
:1025A00002210120F1E702F01FBB10B50446FFF73E
:1025B00086FD447510BD2DE9F843054617460E46C5
:1025C0004FF47A704FF03C0C4FF4616815FB08F43F
:1025D00016FB0C443C1900FB0434DFF8E4E19EF9DF
:1025E000009019FB08F89EF9019019FB0C8C9EF9DC
:1025F00002804CFA88FCBEF9038000FB0C809EF838
:1026000008C0BCF1000F20D141EA05001043184377
:1026100002D001208EF808008EF8005028460028CD
:1026200002D518308EF800008EF801108EF80220C6
:10263000AEF8033000933B4632469EF900100FF28D
:10264000F410FFF7BEFDBDE8F183A0420ED3A0EB6E
:10265000040CACF2D17CDFF89881C445DCD322466F
:1026600001460FF2AC10BDE8F843AAE5D4D2A4EBC2
:10267000000CACF2D178DFF87891C845CCD3634632
:10268000224601460FF2981001B0BDE8F04398E5EC
:1026900010B504002FD004F08FFA4949CA68002A07
:1026A00000D0841AB1F80320A218A1F8032012B2B6
:1026B000B2F57A7F06DBA2F57A72A1F803208A7858
:1026C000521C8A7091F902203C2A04DB3C3A8A7041
:1026D0004A78521C4A7091F901203C2A04DB3C3AAA
:1026E0004A700A78521C0A7091F90020182A01DBFE
:1026F00000220A70C86010BD3149052201F000BAFD
:102700000FB410B52DED028B2E4C104606F034FBA5
:102710002D4A2E4B06F048FB206161619FED2C8B0A
:10272000049806F029FB53EC182B06F03DFB2060C3
:102730006160059806F020FB53EC182B06F034FB83
:10274000A060E1609DF81C00207604F118009DF85F
:102750001D1041709DF81E1081709DF81F10C170F2
:102760009DF820100171BDF8210000EE100AB8EEAE
:10277000400A10EE100A06F0E9FB174A1D4B06F05E
:1027800013FB06F00BFCC4F81D00BDF82300A4F8F1
:1027900021009DF8250084F82300BDEC028B10BCBD
:1027A0005DF814FB0749242201F0AAB90CED00E002
:1027B000005400400C9B0020006000209166012026
:1027C000E063012010610120FCA9F1D24D62503F6D
:1027D0008DEDB5A0F7C6B03E3BDF4F8D0400FA0586
:1027E0000C43012000580040F89900209066012019
:1027F0005F4C2605976EA23F49574520256420254A
:102800006400000049524520256420256400000032
:1028100041542D53657454533120256420256400A0
:1028200041542D536574545332202564202564206F
:102830002564000041542D536574542025643A25C5
:10284000643A25642E25640000487047884D0120B5
:1028500000214FF0804200E092089042FCD3002A11
:1028600009D05318984203D3401A801A01EB420151
:1028700049089208F3E708467047002802D400F0A0
:102880007F0002E0404240F08000C0B2704700F09C
:102890007F01802800D349420846704730B404467F
:1028A0000D46A54200DA2C461546A54200DA2C4614
:1028B000A34200DA1C46204630BC704730B40446C0
:1028C0000D46AC4200DA2C461546AC4200DA2C46E6
:1028D0009C4200DA1C46204630BC70471849002252
:1028E0004A608A600861C860704770B50546144C3C
:1028F000A0682169626823689A4214DB91FBF3F6B1
:10290000266190FBF3F0FFF7A3FFA060072804DB2C
:102910002846FFF7E3FF002070BDE6602561002137
:102920006160A16070BD521C626069182161E1683C
:10293000491B01FB0100A060002070BD00000000E9
:10294000609A00200EB47FB5044608A80FC80C9DFD
:1029500005FB00F6009605FB01F6019605FB03F664
:10296000039605FB02F00290204600A9102201F018
:10297000D7F804B070BC5DF810FB10B40C181C192B
:10298000101910BC70470A7822EA000008707047DE
:102990000A7810430870704730B583B004460D467E
:1029A0000020ADF806000120009001AB2246722104
:1029B0000720FFF7D6FC002801D100203EBD01A969
:1029C0002846FFF7E5FF8DF806409DF804008DF8D6
:1029D000070002230DF1060272210720FFF767FCB2
:1029E000401E8041C043C00F3EBD30B583B0044699
:1029F0000D460020ADF806000120009001AB2246F4
:102A000072210720FFF7ADFC002801D100203EBD58
:102A100001A92846FFF7B7FF8DF806409DF804008E
:102A20008DF8070002230DF1060272210720FFF73F
:102A30003EFC401E8041C043C00F3EBDDFF8C808C9
:102A400000210170C17008214170817000F00FBD3C
:102A5000DFF8B4080078032801D101207047002076
:102A60007047DFF8A4080078042801D101207047DE
:102A70000020704710B5DFF89048217800290FD169
:102A80000F219F20FFF7B1FF06219F20FFF784FF52
:102A9000012020700020E07020710120607210BDC4
:102AA000012952D1617A002954D1217900291CD100
:102AB000E17802290BD062785208824207D30120C4
:102AC000E07000F023F9002840F0978062E00129CF
:102AD00060D0A178490881425CD20220E07000F009
:102AE00038F9002840F0898054E001291ED1E178AE
:102AF00002290AD062785208824206D30120E0708F
:102B000000F08EF9002878D10BE0012909D0A178D6
:102B10004908814205D20220E07000F0A4F90028A3
:102B20006BD1E078012859D000202071022020705C
:102B30000020E0700F219F20FFF757FF09219F2001
:102B4000FFF72AFF0120607210BD022955D1617A7A
:102B5000002902D00020607210BD217900291ED109
:102B6000E17802290AD062785208824206D3012015
:102B7000E07000F010F900283FD10BE0012909D0E6
:102B8000A1784908814205D20220E07000F026F9C0
:102B9000002832D10020E0700120207110BD0129F1
:102BA00021D1E17802290AD062785208824206D304
:102BB0000120E07000F079F900281ED10BE0012916
:102BC00009D0A1784908814205D20220E07000F0C6
:102BD0008FF9002811D1E078012802D10020E0709F
:102BE00010BD002020710F219F20FFF7FEFE032063
:102BF00020700020E0700120607210BD38B5002008
:102C0000ADF80000DFF804472078FFF740FE9D2173
:102C10008DF8001000ADFFF730FE6870022300AAA7
:102C200072210720FFF743FB00280ED06078FFF7E2
:102C30002EFE9E218DF80010FFF71FFE6870022304
:102C400000AA72210720FFF732FB31BD3FB581B0EA
:102C5000DFF8B4462078032856D101A80FC8FFF743
:102C60001DFE054601A80FC8FFF728FE217900299F
:102C700020D1E17802290BD06278AA4208DB01203A
:102C8000E07001A80FC800F055F900283CD10CE015
:102C900001290AD0A178814207DA0220E07001A858
:102CA0000FC800F0C4F900282ED10020E0700120E8
:102CB000207129E0012923D1E17802290BD0627823
:102CC000AA4208DB0120E07001A80FC800F027FA33
:102CD000002819D10CE001290AD0A178814207DA35
:102CE0000220E07001A80FC800F095FA00280BD16F
:102CF00000202071E078012802D10020E07003E07C
:102D0000042020700020E07005B030BD10B582B006
:102D10000020ADF80000DFF8F4452078FFF7B7FD9C
:102D200010F17B0F01DA002016BD9D218DF80010F7
:102D3000001FFFF7A2FD8DF801002070022300AAFA
:102D400072210720FFF7B3FA401E8041C043C00F35
:102D500016BD10B582B00020ADF80000DFF8AC451C
:102D60002078FFF794FD7C2801DB002016BD9D2113
:102D70008DF80010001DFFF780FD8DF80100207018
:102D8000022300AA72210720FFF791FA401E80411A
:102D9000C043C00F16BD10B582B00020ADF80000D2
:102DA000DFF868456078FFF772FD10F17B0F01DAFC
:102DB000002016BD9E218DF80010001FFFF75DFD5D
:102DC0008DF801006070022300AA72210720FFF72E
:102DD0006EFA401E8041C043C00F16BD10B582B0D0
:102DE0000020ADF80000DFF824456078FFF74FFDC4
:102DF0007C2801DB002016BD9E218DF80010001DEF
:102E0000FFF73BFD8DF801006070022300AA7221DC
:102E10000720FFF74CFA401E8041C043C00F16BD8B
:102E200010B582B00020ADF80000DFF8E044207853
:102E3000FFF72DFD10F17F0F01D1002016BD9D2160
:102E40008DF80010401EFFF718FD8DF8010020706E
:102E5000022300AA72210720FFF729FA401E8041B1
:102E6000C043C00F16BD10B582B00020ADF8000001
:102E7000DFF898442078FFF70AFD7F2801D1002071
:102E800016BD9D218DF80010401CFFF7F6FC8DF853
:102E900001002070022300AA72210720FFF707FA21
:102EA000401E8041C043C00F16BD10B582B0002047
:102EB000ADF80000DFF854446078FFF7E8FC10F14B
:102EC0007F0F01D1002016BD9E218DF80010401EFD
:102ED000FFF7D3FC8DF801006070022300AA722175
:102EE0000720FFF7E4F9401E8041C043C00F16BD24
:102EF00010B582B00020ADF80000DFF81044607813
:102F0000FFF7C5FC7F2801D1002016BD9E218DF85A
:102F10000010401CFFF7B1FC8DF801006070022327
:102F200000AA72210720FFF7C2F9401E8041C0436A
:102F3000C00F16BD3FB581B000252846ADF8000092
:102F4000DFF8C44301986178884217DA6079FFF7A7
:102F50009EFC10F17A0F11DBA4218DF80010001FE8
:102F6000FFF78BFC00A948706071022300AA722150
:102F70000720FFF79CF9002853D0012502986178BB
:102F8000884217DAA079FFF782FC10F17A0F11DB83
:102F9000A5218DF80010001FFFF76FFC00A94870F5
:102FA000A071022300AA72210720FFF780F90028F0
:102FB00037D0012503986178884217DAE079FFF766
:102FC00066FC10F17A0F11DBA7218DF80010001FAD
:102FD000FFF753FC00A94870E071022300AA722198
:102FE0000720FFF764F900281BD0012504986178B9
:102FF000884219DA207AFFF74AFC10F17A0F13DBC6
:10300000A9218DF80010001FFFF737FC00A94870B8
:103010002072022300AA72210720FFF748F9002836
:1030200001D1002001E00125284605B030BD3FB5A3
:1030300081B000252846ADF80000B34CA078019976
:10304000884216DA6079FFF722FC7B2811DAA42186
:103050008DF80010001DFFF710FC00A9487060718A
:10306000022300AA72210720FFF721F9002850D07F
:103070000125A0780299884216DAA079FFF707FCAB
:103080007B2811DAA5218DF80010001DFFF7F5FB54
:1030900000A94870A071022300AA72210720FFF73F
:1030A00006F9002835D00125A0780399884216DA60
:1030B000E079FFF7ECFB7B2811DAA7218DF80010EF
:1030C000001DFFF7DAFB00A94870E071022300AA97
:1030D00072210720FFF7EBF800281AD00125A0780D
:1030E0000499884218DA207AFFF7D1FB7B2813DA9B
:1030F000A9218DF80010001DFFF7BFFB00A9487043
:103100002072022300AA72210720FFF7D0F80028BE
:1031100001D1002001E00125284605B030BD3FB5B2
:1031200081B000252846ADF80000774C0198617801
:10313000884217DA6079FFF7AAFB10F17F0F11D0F0
:10314000A4218DF80010401EFFF797FB00A94870DE
:103150006071022300AA72210720FFF7A8F8002857
:1031600053D0012502986178884217DAA079FFF7D9
:103170008EFB10F17F0F11D0A5218DF80010401E9D
:10318000FFF77BFB00A94870A071022300AA7221FF
:103190000720FFF78CF8002837D0012503986178C5
:1031A000884217DAE079FFF772FB10F17F0F11D038
:1031B000A7218DF80010401EFFF75FFB00A94870A3
:1031C000E071022300AA72210720FFF770F800289F
:1031D0001BD0012504986178884219DA207AFFF71C
:1031E00056FB10F17F0F13D0A9218DF80010401E5F
:1031F000FFF743FB00A948702072022300AA722146
:103200000720FFF754F8002801D1002001E0012534
:10321000284605B030BD3FB581B000252846ADF841
:103220000000394CA0780199884216DA6079FFF7DE
:103230002EFB7F2811D0A4218DF80010401CFFF731
:103240001CFB00A948706071022300AA72210720AC
:10325000FFF72DF8002850D00125A0780299884268
:1032600016DAA079FFF713FB7F2811D0A5218DF87E
:103270000010401CFFF701FB00A94870A071022359
:1032800000AA72210720FFF712F8002835D0012587
:10329000A0780399884216DAE079FFF7F8FA7F28D8
:1032A00011D0A7218DF80010401CFFF7E6FA00A905
:1032B0004870E071022300AA72210720FEF7F7FF91
:1032C00000281AD00125A0780499884218DA207ABB
:1032D000FFF7DDFA7F2813D0A9218DF80010401CDC
:1032E000FFF7CBFA00A948702072022300AA7221CE
:1032F0000720FEF7DCFF002801D1002001E00125B6
:10330000284605B030BD0000EA6201207D6301203F
:1033100010B5044610460A460146204605F086FED2
:10332000204610BDDFF880070021C161DFF87C175F
:1033300000220A7701224A7700221046086381F8AA
:103340002000C87770470FB410B5DFF85C479DF8D0
:103350001D00411E8941C90F6177201D03A910225C
:1033600000F0DEFBDFF844079DF81E1041770021D6
:1033700080F8201001779DF80810002907D1217FDF
:103380004A1C227706290ED3012101770BE0002089
:103390002077607F00289DF8080002D100F030F906
:1033A00001E000F09DF810BC5DF814FB0FB438B5D7
:1033B000DFF8F4469DF82400411E8941C90FE177EA
:1033C000201D05A9102200F0ABFBDFF8E0569DF8A8
:1033D0002600687705A80FC8FFF770FA606168617A
:1033E000002085F820002877E07F002804D105A878
:1033F0000FC800F0AEF909E0A07F002805A80FC8AB
:1034000002D000F0DFF901E000F018FA31BC5DF8FD
:1034100014FBF0B50446DFF8985605F11C06DFF8FA
:103420008806C17F4A1E9241D20F7275407F411EAD
:103430008941C90FB175DFF87476387F307597F818
:1034400020002877284639461C2200F069FBB87F07
:10345000707005F12000DFF85C16102200F060FBB0
:10346000204629463422BDE8F04000F059BB10B593
:1034700082B00020ADF80000A0208DF8000000AC64
:1034800000206070DFF82C0600210174022300AADE
:1034900072210720FEF70BFF002801D1002016BD86
:1034A000A1208DF80000FF206070022300AA722185
:1034B0000720FEF7FCFE002801D1002016BD802168
:1034C000A320FFF769FA3C21A220FFF765FADFF895
:1034D000D80500218177DFF8D4050163012016BDEE
:1034E00010B50446DFF8C005807F0028204602D0D2
:1034F000BDE810400BE000F039F8DFF8B005C07F00
:10350000002803D12046BDE8104053E010BD10B59F
:10351000DFF89845E07F012827D1201DDFF89815B6
:10352000102200F0FDFA04202070A069C7280FD1F6
:10353000201D0FC8FFF7C2F9A17F814208DADFF82A
:103540007C05012101700FF28850FEF73AFE07E07A
:10355000DFF86805002101700FF28C50FEF731FE94
:10356000012084F820000020E07710BD10B5DFF8BE
:103570003C45E17F012909D100F0CBF8002802D0B9
:103580000420E07710BD0020E06210BD002909D1C1
:1035900000F0B6F8002802D00220E07710BD00202D
:1035A000E06210BDE06A411CE1620B2801DB0020F3
:1035B000E06210BD10B5044600F055F8204600F05A
:1035C0005DF8204600F065F8204600F06DF8DFF861
:1035D000D804416A01EB8102D100642291FBF2F12F
:1035E000826B436B9A4204DAC06A052290FBF2F0C8
:1035F00003E0806A142290FBF2F0BDE8104091E0F5
:1036000038B5044600F014F8204600F01AF8DFF848
:103610009854686A00EB8001C800642190FBF1F1C6
:1036200004EB8400400000F07DF80120687731BD94
:10363000DFF874144FF4FA620A62C8224A62FFF794
:103640004DB9DFF86414C82212FB00F28A623222FC
:1036500012FB00F2CA6200EB800252000A63486368
:103660008863C863704710B50146DFF83C4404F135
:1036700030020A2000F025F8E06310BD10B50146C5
:10368000DFF8244404F12C02322000F01AF8A06381
:1036900010BD10B50146DFF8104404F12802C8201F
:1036A00000F00FF8606310BD10B5FFF71EF964213C
:1036B00001FB00F4002C02D0204600F013F8204655
:1036C00010BD10B400EBD0735B101468091900FB37
:1036D0000131441C91FBF4F11160591891FBF0F099
:1036E00010BC704710B50146C82900DAC821DFF8C0
:1036F000B84304F120020A20FFF7E3FF606210BD27
:10370000DFF8A813496A814201DA012070470020DE
:103710007047DFF89813896A884201DA0120704700
:103720000020704740F2DD52904201DB40F2DC5055
:103730000A2901DA0A2102E0652900DB6421081860
:10374000401D0A2190FBF1F0C0B2D849486288625E
:10375000704780B500F004F8D3480121C17701BD5E
:103760000FB587B0C820019007A883B069460CC880
:103770000CC10CC80CC10EBC02A8FFF7E3F8D0487E
:1037800002A9102200F0CCF90A20019007A883B00A
:1037900069460CC80CC10CC80CC10EBC02A8FFF7CE
:1037A000D1F8C84802A9102200F0BAF9C64807A902
:1037B000102200F0B5F9C54807A9102200F0B0F9B1
:1037C0000BB000BD00BF1FB5B84CE07F002802D091
:1037D00001280ED01FBD0020A061201D00A91022CD
:1037E00000F09EF902202070012084F82000E0778C
:1037F0001FBD201D00A9102200F092F901202070A9
:10380000A069401CA061C72807D10121AB20FFF7A8
:10381000ECF80021AB20FFF7BFF8A069C82809DB4E
:103820000020A0610121AB20FFF7DFF80021AB20D1
:10383000FFF7B2F8012084F820001FBD1FB59B4C94
:10384000E07F002803D0012084F8200003E000A8D6
:103850000FC800F037F800A80FC800F00AF8607F22
:10386000002805D0206B292802DBBDE81F40D8E0E6
:103870001FBD1FB58D4CE07F012804D002280DD05C
:10388000042817D01FBD201D00A9102200F048F900
:1038900001202070A069401CA0611FBD0020A06114
:1038A000201D00A9102200F03BF902202070012009
:1038B000E0771FBD042020700020E077012084F80D
:1038C00020001FBDFFB585B07848016B491C01631E
:1038D00005A883B069460CC80CC10CC80CC10EBC4D
:1038E00001A800F025F805A883B069460CC80CC1F2
:1038F0000CC80CC10EBC01A800F040F8734C94E851
:103900000F00FFF73AF805466A4E6F4F97E80F0031
:10391000FFF733F88542304604DA2146102200F0E2
:10392000FFF803E03946102200F0FAF809B0F0BDC4
:103930000EB430B588B004460BAD0BA80FC885E8AF
:103940000F005F4802900BA882B069460CC80CC1FA
:103950000CC80CC10CBCC82103A800F035F85A4DA6
:10396000284603A9102200F0DBF820462946102241
:1039700000F0D6F808B030BC5DF810FB0EB430B5DE
:1039800088B004460BAD0BA80FC885E80F004D4862
:1039900002900BA882B069460CC80CC10CC80CC1BF
:1039A0000CBC0A2103A800F00FF8484D284603A9D3
:1039B000102200F0B5F820462946102200F0B0F899
:1039C00008B030BC5DF810FB0CB47FB504460D4662
:1039D00008AE08A80FC886E80F000C9E32460146C4
:1039E0002846FFF76EFE0090321D09992846FFF722
:1039F00068FE019006F10C020B992846FFF761FE64
:103A0000039006F108020A992846FFF75AFE029031
:103A1000204600A9102200F083F804B070BC5DF8C5
:103A20000CFB70B582B00020ADF80000214C94E88A
:103A30000F00FEF743FF401D1C4DFF2802DDFF2055
:103A4000A87700E0A877A0208DF8000000AE686A93
:103A5000707070782074022300AA72210720FEF78C
:103A600026FC002801D1002076BDA1208DF80000A1
:103A7000A87F7070022300AA72210720FEF717FCAE
:103A8000002801D1002076BD8021A320FEF7ADFFE4
:103A90003C21A220FEF7A9FF0348012181770020E5
:103AA0002863084676BD0000485D0120A45F012020
:103AB000D85F01206C6301204C5D01208E660120DF
:103AC000A0630120C0630120B0630120D063012006
:103AD000233E445F6C6F6E675F67657374757265D4
:103AE000203A202564000000233E525F6C6F6E6711
:103AF0005F67657374757265203A20256400000065
:103B000062B38B0708D0521E11F8013B00F8013B4D
:103B100000F024808B07F6D1830740F0208000BF9F
:103B2000103A07D330B4B1E83810103AA0E8381092
:103B3000F9D230BC530724BFB1E80810A0E8081040
:103B400044BF51F8043B40F8043BD20724BF31F88E
:103B5000022B20F8022B44BF0B7803707047083A01
:103B600007D3B1E80810083A40F8043B40F804CB0A
:103B7000F7D25307E4E710B50446FFF7C1FF20462C
:103B800010BD50F8041B61B150F8042BD30744BF9B
:103B9000A9F101039A18002342F8043B091FFAD146
:103BA000EFE7704730B583B00121032005F0D6FA66
:103BB000DFF8804C204605F06DFBDFF87C5C284682
:103BC00005F068FB01208DF8040000208DF8050049
:103BD00001208DF8060000208DF8070001212846FD
:103BE0000183C0460120009000A9284605F0AEFBE5
:103BF000022128460183C0460220009000A92846E1
:103C000005F0A4FB01208DF8040000208DF80500CC
:103C1000ADF806004FF48070009000A9284605F02A
:103C200095FB4FF4807128464183C04601208DF8F2
:103C3000040000208DF8050001208DF8060000200A
:103C40008DF807004FF48050009000A9204605F041
:103C50007DFB4FF4805120464183C046042206215B
:103C6000284605F0C1FB04220721284605F0BCFBCD
:103C700002208DF8040001208DF805008DF8060063
:103C800000208DF807004020009000A9284605F08C
:103C90005DFB8020009000A9284605F057FB042218
:103CA0000A21284605F0A0FB09220321284605F039
:103CB0009BFB02208DF8040001208DF805008DF893
:103CC000060000208DF807004FF48060009000A9E6
:103CD000284605F03BFB0820009000A9284605F087
:103CE00035FB286820F0300040F010002860206884
:103CF00020F0300040F01000206037BD1FB5DFF825
:103D00003C4BA04230D101214FF4001005F031FAB4
:103D10000121022005F022FA01214FF4001005F0E4
:103D200049FA00214FF4001005F044FA0020ADF8E4
:103D300004004BF6FF70ADF806004FF48060ADF85C
:103D40000A004FF48040ADF80C000A20ADF80800DE
:103D5000DFF8CC0C009000A9204605F088FB01217B
:103D6000204605F0E7FB1FBDDFF8B84CA0422FD17D
:103D700001214FF4800005F0FCF90121022005F03B
:103D8000EDF901214FF4800005F014FA00214FF401
:103D9000800005F00FFA0020ADF804004BF6FF702C
:103DA000ADF806004FF48060ADF80A004FF4804093
:103DB000ADF80C000A20ADF80800DFF8640C0090A4
:103DC00000A9204605F053FB0121204605F0B2FB77
:103DD0001FBD2DE9F04192B001214FF4805005F054
:103DE000D3F90121084605F0B9F901214FF480000B
:103DF00005F0B4F9DFF83C4A05221146204605F0EB
:103E0000F3FA05220721204605F0EEFA05220621E5
:103E1000204605F0E9FA05220421204605F0E4FADF
:103E200002208DF8040001208DF805000020ADF877
:103E300006002020009000A9204605F087FA802087
:103E4000009000A9204605F081FA4020009000A9CA
:103E5000204605F07BFA1020009000A9204605F0CE
:103E600075FADFF8C44B204605F0C6FBDFF8BC5BF3
:103E70000020288068600120288100206881E86097
:103E80000720288200206880DFF8A46B304605F008
:103E900023FCDFF8A07B384605F01EFC4FF4806061
:103EA000069000210D9103210E9100210F910A919E
:103EB0000890DFF8180C03900846109009900790BE
:103EC0004FF400300C9008460B904FF0C068CDF8CE
:103ED0000880402005900846049002A9304605F06D
:103EE0007FFC00200B90CDF80880059005F11400B0
:103EF000049002A9384605F073FC0020688029462A
:103F0000204605F0A8FB01220221204605F0D2FB45
:103F100001221146204605F0CDFB0121204605F087
:103F2000BDFB0021304605F082FC0021384605F03B
:103F30007EFC12B0BDE8F08130B589B001214FF0B0
:103F4000805005F016F9012005F0DAFC01214FF44C
:103F5000802005F003F90F2005F082FE04461020B2
:103F600005F07EFE0546012005F0F5F8002005F07D
:103F7000F2F821460F2005F066FE2946102005F0D4
:103F800062FE00214FF4802005F0E8F8012005F0E2
:103F900081F8412005F02FF90028FAD04FF4807005
:103FA00005F0C3F8012005F0D3F805F0FCFC3F2034
:103FB000069040F2FF1007900020059005A805F03C
:103FC000A9FC0020029002A905F00EFD00208DF84A
:103FD000070001208DF804008DF805008DF806001B
:103FE00001A9002005F079FD4FF4800005F018FFCD
:103FF0004FF48000039000208DF8100008208DF809
:10400000110001208DF8120003A805F0C7FE03205F
:104010008DF800000D208DF8010000208DF80200C1
:1040200001208DF8030000A805F007FF032005F02C
:10403000C8FD4FF4804005F07EFE4FF4800005F08F
:10404000EFFE01214FF4804005F03BFE012009B056
:1040500030BD10B586B00121084605F07FF801217A
:104060004FF4804005F090F800208DF810008DF896
:10407000130001200390DFF8BC4703A9204605F098
:1040800065F90420039003A9204605F05FF900219B
:10409000084605F00BFF0221002005F007FF002075
:1040A0008DF8080001208DF80A0001900C208DF891
:1040B000090001A805F072FE042001900C208DF883
:1040C000090001A805F06AFE042005F0A9FE2820D9
:1040D0008DF800000F208DF8010000208DF80200FF
:1040E00001208DF8030000A805F0A7FE06B010BD62
:1040F00010B586B00121084605F030F801214FF4D3
:10410000804005F041F800208DF810008DF8130074
:104110004FF40064039403A9DFF8180705F016F9BB
:104120000B21002005F0C2FE00208DF808000120C0
:104130008DF80A0001940C208DF8090001A805F003
:104140002DFE204605F06CFE28208DF800000F2083
:104150008DF8010000208DF8020001208DF8030089
:1041600000A805F06AFE06B010BD30B58DB004465B
:1041700001214FF4807005F007F800A805F020F940
:104180000A20009003208DF8040000208DF807001D
:1041900000A9DFF8A00605F0D9F805F09BFE02A8FB
:1041A00005F0DDFE4FF48030039002A805F0C9FE53
:1041B00006A805F0BCFEDFF8DC5A06A9284605F083
:1041C00096FE072301222146284605F0D9FE01214B
:1041D000284605F01AFF0121284605F0C6FE0DB05D
:1041E00030BD38B5DFF8AC4A204605F009FF4FF482
:1041F0007A750221204605F01FFF002803D12846CA
:10420000451E0128F5DA2046BDE8324005F008BF1A
:1042100080B50021DFF87C0A05F0A7FE00214FF4ED
:104220008070BDE8044004F0AFBFDFF8280B0068E1
:104230007047000038B5040040D0012005F060FB55
:10424000002005F0D8FC4FF40055042005F054FD83
:10425000012804D12846451E80B20028F5D100EE81
:10426000104AB8EE400ADFED800A80EE800AF0EED8
:10427000000A20EE200ADFED7D0A80EE800ABDEE06
:10428000C00A10EE100A401E80B205F0AAFC4FF4DE
:10429000804005F050FD4FF4800005F0C1FD012085
:1042A00005F0A9FCDFF8AC0A012181600460214619
:1042B0000FF22000BDE83440FDF783BFDFF8940A19
:1042C00000210160012005F01BFB0020BDE8324009
:1042D00005F091BC536574525443203D2025640081
:1042E00030B4014601200023DFF86C2A1C4694609C
:1042F000946814F00C0FFBD10C460B2C55D8DFE85A
:1043000004F02054545406192031383F464D946827
:1043100044F080049460DFF8444A4FF4C06525609F
:10432000146824F080741460DFF8B44ADFF8305A5F
:1043300025603BE00346DFF8A84ADFF8A85A25606D
:1043400034E094689460DFF8144A4FF4C065256047
:10435000146824F080741460DFF8844ADFF8885A07
:10436000256023E00223DFF8784ADFF8805A2560D1
:104370001CE00323DFF8684ADFF8745A256015E073
:104380000423DFF85C4ADFF8C45A25600EE00523F9
:10439000DFF84C4ADFF8B85A256007E00623DFF85B
:1043A000404ADFF8B05A256000E01846002B4AD09A
:1043B00003EBC3030FF2B8041B19946894601468EC
:1043C00024F080741460146824F0806414609C7875
:1043D0001D8844EA8514DD786D086D1E44EA0544A5
:1043E0001D7944EA05645460DC881D7A2D0745EA8E
:1043F0008414DFF8C05A2C60146844F08074146090
:104400001468A401FCD55B7943F4C063DFF84C4920
:1044100023609368936093689360052904D1916841
:1044200041F09001916005E00A2903D1916841F4BF
:1044300080519160916841F002019160916801F0B2
:104440000C010829FAD1DFF898190968DFF8682A01
:10445000914207D2DFF8F41A0A6822F4404242F48B
:1044600080420A6030BC704700007A440000004778
:10447000200110040F03020103F00010060F0102D7
:104480000103C00010080F01020103C00010060F55
:1044900001020103F00010060F01020103C8001021
:1044A000040F02020103A80010020F03020103001F
:1044B00016E7002800E0401EFDD170477CB50726B6
:1044C000DE4988426BD101208DF804008DF805008B
:1044D0008DF8060000208DF8070040200090DFF8DE
:1044E0008C5A00A9284604F031FF8020009000A9D2
:1044F000284604F02BFF402128464183C0460F2068
:10450000FFF7D7FF402128460183C0460F20FFF761
:10451000D0FF3046461E80B20028ECD180200090AB
:1045200000A9284604F012FF402128464183C046D6
:104530000520FFF7BEFF802128460183C0460520E5
:10454000FFF7B7FF402128460183C0460A20FFF746
:10455000B0FF402128464183C0460520FFF7A9FF50
:10456000802128464183C0460520FFF7A2FF022094
:104570008DF8040001208DF805008DF8060000205C
:104580008DF807004020009000A9284604F0DEFEC8
:104590008020009000A9284604F0D8FE73BDDFF803
:1045A000841488426AD101208DF804008DF805003A
:1045B0008DF8060000208DF807004FF48064009409
:1045C000DFF8A85900A9284604F0C0FE0820009092
:1045D00000A9284604F0BAFE214628464183C04679
:1045E0000A20FFF766FF214628460183C0460A20BD
:1045F000FFF75FFF3046461E80B20028ECD108204E
:10460000009000A9284604F0A1FE214628464183D7
:10461000C0460520FFF74DFF082128460183C0460C
:104620000520FFF746FF214628460183C0460A20A1
:10463000FFF73FFF214628464183C0460520FFF78C
:1046400038FF082128464183C0460520FFF731FF87
:1046500002208DF8040001208DF805008DF8060079
:1046600000208DF80700009400A9284604F06EFE93
:104670000820009000A9284604F068FE73BD10B51C
:10468000DFF8EC480121206804F08DFF206804F079
:10469000BFFE2068FFF732FB05E02068FFF70EFF42
:1046A0002068FFF72BFB4FF40031206804F086FFF1
:1046B0000028F2D110BD30B40022838A008BDFF8CD
:1046C000B048656843EA00400840000255EA1020FF
:1046D00060600840884200D10122104630BC70471B
:1046E0002DE9F84F04460D4616464FF420491F7831
:1046F000DFF87C884FF40031D8F8000004F05EFF4A
:10470000002808D04846A0F101090028F2D1FFF79F
:10471000B6FF00208CE0D8F8000001884FF6FF5269
:10472000114001800121D8F8000004F00FFF4FF480
:10473000805AD1460020C8F80400D8F800B0DFF84D
:1047400034185846FFF7B7FF002805D14846A0F1B6
:1047500001090028F1D163E0D146002221465846E4
:1047600004F00CFF0020C8F80400D8F80040DFF87F
:1047700008182046FFF79FFF002805D14846A0F102
:1047800001090028F1D14BE03146C9B2204601822F
:10479000C046D1460020C8F80400D8F80040DFF831
:1047A000DC172046FFF787FF002805D14846A0F117
:1047B00001090028F1D133E0012F15D129782046D5
:1047C0000182C046D1460020C8F80400DFF8B017C7
:1047D000D8F80000FFF76FFF002823D14846A0F16A
:1047E00001090028F2D11BE03846471EC0B200285C
:1047F00018D015F8011BD8F800000182C046D14638
:104800000020C8F80400DFF87817D8F80000FFF798
:1048100052FF0028E8D14846A0F101090028F2D152
:10482000002005E00121D8F8000004F09BFE0120E3
:10483000BDE8F28F00000240000402400054004036
:104840002DE9F54F81B00D461E464FF420483778CC
:10485000DFF81C474FF40031206804F0AFFE002859
:1048600008D04046A0F101080028F3D1FFF707FF68
:104870000020D3E0206801884FF6FF5211400180EC
:104880000121206804F062FE4FF48059C8460020E0
:104890006060DFF8E0A6D4F800B051465846FFF754
:1048A0000AFF002805D14046A0F101080028F2D1F6
:1048B00091E000229DF80410584604F05FFEC846BF
:1048C00000206060D4F800B0DFF8AC165846FFF75F
:1048D000F2FE002805D14046A0F101080028F1D1E0
:1048E00079E0BDF80810C9B258460182C046C846F2
:1048F000DFF89016206804F061FE002805D14046DC
:10490000A0F101080028F3D165E00121206804F03E
:104910001DFEC84600206060D4F800B051465846DD
:10492000FFF7C9FE002805D14046A0F10108002884
:10493000F2D150E001229DF80410584604F01EFE0A
:10494000022FC84639D2DFF84016206804F036FE40
:10495000002805D14046A0F101080028F3D13AE033
:104960000021206804F013FE2068018B012104F06F
:10497000F9FDC846DFF81416206804F01FFE002871
:1049800005D14046A0F101080028F3D123E02068BA
:10499000008AC0B228703078401E3070C846206847
:1049A0000188890505D54046A0F101080028F6D107
:1049B00011E0012104F0EBFD2BE000206060DFF846
:1049C000D0152068FFF777FE002806D14046A0F1F9
:1049D00001080028F3D1002020E0012616E0012F75
:1049E0000CD1012E0AD100263146206804F0CFFDFB
:1049F0002068818A018B012104F0B4FD2068818A3E
:104A0000490603D5008A05F8010B7F1EFFB2002F6F
:104A1000E5D10121206804F0BAFD0120BDE8FE8F38
:104A2000801A06000058004000300140EC60012070
:104A30008864024010640240DFF8580501680829C4
:104A400033D1DFF814130A6842F080720A604268BA
:104A5000B2F1806F03D10A6842F080620A600A688E
:104A60009201FCD58A6842F002028A608A6802F0EC
:104A70000C02082AFAD14268B2F1806F02D10A68AA
:104A80001201FCD5DFF858130968DFF82C24914295
:104A900007D2DFF8B8140A6822F4404242F4804298
:104AA0000A6000210160416070474168B1F1806F88
:104AB00009D1A9490A6842F080620A600A681201B5
:104AC000FCD5002141607047000000000C3001401F
:104AD000DFF8C404016841F080510160DFF86C0424
:104AE00001688908890041F001010160DFF8AC0428
:104AF0000FF205014160704738B5DFF8A444208803
:104B000040F004002080FDF7DAFA807A012803D112
:104B1000012004F0F8FE02E0002004F0F4FEDFF8CB
:104B200084548021DFF8800404F0CEFD002818D1E1
:104B300072B68948DFF85C14826802F00C020A60E1
:104B4000006800F080604860286840F00400286039
:104B500030BF62B6286820F004002860FFF76CFFC1
:104B60000CE0608840F004006080286820F00400B9
:104B7000286030BF286840F004002860608840F05A
:104B80000400608031BDDFF8140440680047DFF89E
:104B90001C14012806D010D3032809D005D30428FB
:104BA00009D00AE0DFF8C41307E0DFF8041404E0DA
:104BB000DFF8001401E0DFF800140846704710B574
:104BC0000C46FFF7E4FF214689B2BDE8104004F02F
:104BD00007BC10B50C46FFF7DAFF214689B2BDE8E5
:104BE000104004F0FFBB0000E0B500238DF8083052
:104BF00001238DF80A30002A03D10C228DF80920F8
:104C000002E008228DF8092004283CD8DFE800F0F3
:104C1000030D192222004FF40060019028208DF826
:104C200000000F208DF801001CE0184601901020B4
:104C30008DF8090006208DF800000E208DF8010087
:104C400010E00220019007208DF800000F208DF861
:104C5000010007E00420019008208DF800000F20DB
:104C60008DF8010000208DF80200012903D11846BB
:104C70008DF8030001E08DF8030001A805F08EF81F
:104C800000A805F0DAF807BD4FF40061C74804F04A
:104C9000A0BB00000020014010B5044601214FF4E4
:104CA000802004F05BFA2146102004F0CCFF0021A4
:104CB0004FF48020BDE8104004F050BA10B5012137
:104CC0004FF4802004F04AFA102004F0C9FF044693
:104CD00000214FF4802004F041FA7B2004F08BFA8D
:104CE000002802D09AA0FDF76CFA7A2004F083FA2B
:104CF000002802D097A0FDF764FA792004F07BFA2F
:104D0000002802D094A0FDF75CFA7C2004F073FA2E
:104D1000002802D091A0FDF754FA7D2004F06BFA30
:104D2000002802D08EA0FDF74CFA7E2004F063FA32
:104D3000002802D08BA0FDF744FA7F2004F05BFA34
:104D4000002802D088A0FDF73CFA04F06AFA204659
:104D5000C0B210BD7C64012000380240003C02401B
:104D600000127A003EB50C4615460422014602A800
:104D7000FEF701FF0422214601A8FEF7FCFE0422F3
:104D8000294600A8FEF7F7FE02A9002004F02CFE39
:104D900001A9002004F0A1FE04F09AFE0446874A0F
:104DA000002300981946101A63EB0101490241EAF9
:104DB000D051400205F06AF90090844205D2011BEF
:104DC0004FF0004004F059FF37BDA04207D2C4F5B0
:104DD0000070009909184FF0004004F04EFF37BDF5
:104DE000AC9A0020809698000024F40000366E01F2
:104DF0000048E8012DE9704384B004460D4616468C
:104E000002A9002004F03FFE01A9002004F0B5FE35
:104E100004F05EFE0090694AA2FB00894FEA582820
:104E200048EAC958A2EB08000090042202A92046D3
:104E3000FEF7A1FE042201A92846FEF79CFE0422EB
:104E400000A93046FEF797FEBDE87F83005A620254
:104E500080F0FA0200BD0105F0B4049C059D8E1E91
:104E6000012E01DA0C36401E3C216427B0FBF7F717
:104E7000C7EB90074FF4C87CB0FBFCFC674440F2E2
:104E80006F1C0CFB06F64FF00C0CB6FBFCF6F6198B
:104E9000921940F26D1606FB0020494A101800EBEB
:104EA000400203EBC20001FB004001FB0050F0BCDC
:104EB0007047000084380240018793031CB50C46FC
:104EC00001680191416800918368C2680169491CC9
:104ED000406900F26C70FFF7BFFF2060002016BD34
:104EE00010B58EB037480068C405E40D01A9002054
:104EF00004F0C9FD00A9002004F03FFE9DF8040065
:104F000006909DF8050005909DF8060004909DF818
:104F10000100401E08909DF8020007909DF80300D4
:104F20006430099002A904A8FFF7C8FF4FF47A7013
:104F300010FB04F0400AC0F57A700390029A4FF417
:104F40007A73C117E3FB02010EB010BD0070004080
:104F5000504F520050494E00424F520053465400A9
:104F600049574400575744004C5057000004024032
:104F70000C9B002001000300820007008000070056
:104F80008400070004000010020000104000001020
:104F90000200030084650120403802407C64012047
:104FA0001800024010ED00E0003001400000024017
:104FB00000080240000C02400010024000CA9A3B68
:104FC0007505F5FF282800405060026041600860C8
:104FD00070470A68F8E748600160704701684068F8
:104FE000F9E7F8B50600DFF8C05802D505F158001A
:104FF000F2BD05F158040020296F00E0096805F1B1
:105000007002914204D00C46A2689642F6D101206B
:10501000002840D1A86FD0F88070182005F0AEF8B5
:105020000446A660002F05D0B74203D2B6FBF7F0C6
:10503000784300E03046E060002F02D0B74200D253
:105040003E46266100202075DFF860683078401CFD
:1050500030707078F021084202D0992000F018FDDD
:1050600000F083FD7078401C707005F170012046DF
:10507000FFF7AFFF7078F021084202D0992000F0CE
:1050800007FD7078401E7070C0B2002801D100F09A
:1050900066FD01F0C0FB2046F2BD38B5044694F928
:1050A0001400002829D1DFF804582878401C287003
:1050B0006878F021084202D0992000F0E9FC00F065
:1050C00054FD6878401C68702046FFF787FF204633
:1050D00005F06CF86878F021084202D0992000F0C1
:1050E000D7FC6878401E6870C0B2002801D100F07B
:1050F00036FDBDE8314001F08EBB31BDF8B5044648
:1051000008466FF00045FFF76CFF064694F905006E
:1051100094F90410814214D1C01C800005F02EF8CF
:10512000074694F90500012807DB8200216838460C
:10513000FEF721FD206805F039F827606079C01C72
:10514000607194F90400411C2171216841F82060CC
:10515000DFF85C07864202D0307D401C30750020AD
:1051600008E0216851F820108A68954201DB154655
:10517000A160401C94F904108842F2DBF1BDF8B53F
:1051800004466FF00046DFF8202702F1580502F1CF
:1051900058004FF0FF33002704E0664501DB664608
:1051A00075467F1C94F904C067450DDAD4F800C039
:1051B0005CF827E0DEF808C0002BEED58C45ECD17A
:1051C00070463B465BB2ECE7002B11D4BCF1010FFB
:1051D0000EDB06E0216801EB8306766841F8236068
:1051E0005B1C94F904104E1EB342F3DB491E21717F
:1051F00002F15801884204D0017D491E0175FFF774
:105200004CFFA560F1BD10B4C26A836B406C9C6812
:10521000002C02D56FF0004300E01B698468002C6D
:1052200002D56FF0004000E00069984200DD1846AA
:10523000D2685143884201DB012000E0002010BC0D
:10524000704738B5DFF860168A6FD36E012490F985
:105250000850AC402343D36601F66C11FFF7B9FE4A
:10526000012032BD10B5DFF84016896FCA6E0123E8
:1052700090F90840A3409A43CA66FFF7AFFE0120A9
:1052800010BD012070472DE9FC4104460D4616462D
:105290001F4604F12400FFF731FF07EB470004EB42
:1052A0008008314608F13000FFF728FF019598F992
:1052B000340000903B46627A94F908100FF2F450E3
:1052C000FCF77FFFBDE8F3812DE9FC4104460D4664
:1052D00016461F4604F12400FFF751FF07EB470075
:1052E00004EB8008314608F13000FFF748FF0195D4
:1052F00098F9340000903B46627A94F908100FF256
:10530000C850FCF75EFFBDE8F381C16A8A68012AD4
:1053100009DB0969012906DA006D002801D50020A2
:105320007047022070470020704701EB410200EBFC
:105330008201896B8A68012A09DB0969012906DA79
:10534000006D002801D50020704702207047002022
:105350007047002900D5D8E7E7E7012900DA0121E5
:1053600013460A468FE7012900DA012113460A464F
:10537000AAE7DFF83405C06A417A481E8041C00FB1
:10538000704713464FF0FF3211467CE713464FF04B
:10539000FF32114698E780B5DFF80C050068417AC6
:1053A000002902D1006E40688047012002BD80B50F
:1053B000FFF758FFDFF8F0040068417A002902D1B6
:1053C000006E80688047012002BDB1F57A7F01DC64
:1053D0004FF47A7113460A464FF4FA7153E7B1F568
:1053E0007A7F01DC4FF47A7113460A464FF4FA7162
:1053F0006AE710B50446002922D5E06A81680129D0
:105400001CDB0069012819DA02212046FFF7FBFEA8
:10541000002813D194F954004FF0FF31884204D191
:10542000002084F85400012010BD002806D101207E
:105430006077084684F85400022010BD002010BD9B
:10544000BDE8104071E74FF0FF3280F85420F8E6D5
:10545000DFF85424926FD2F88020A03252420265C5
:10546000EFE600290AD5C06A8168012904DB0069DA
:10547000012801DA022070470020704755E7B5295E
:1054800000DAB42113460A463C21FCE6B52900DACD
:10549000B42113460A463C2116E710B504460029FC
:1054A00026D5E06A8168012920DB006901281DDA20
:1054B00003212046FFF7A7FE002817D194F95400D6
:1054C0004FF0FF31884204D1002084F854000120BD
:1054D00010BD002803D1012084F8540010BD01281C
:1054E00004D1084684F85400022010BD002010BDED
:1054F000BDE8104019E74FF0FF3280F85420DFF884
:10550000A823926FD2F88020B4325242026598E606
:10551000DFF89423926FD2F88020C832524202659D
:105520008FE613464FF0FF321146ACE613464FF0BC
:10553000FF321146C8E680B5FFF783FEFCF7BFFDDA
:1055400000210175012002BD80B5FFF78BFEFCF73D
:10555000B6FD00210175012002BD00002DE9F041DA
:105560000C46D14D55F82060307206F154070FF209
:105570006C313961152800F22E81DFE810F0160039
:105580002600330053004300620073008200B20023
:105590009200A200C200D200E000EC00F900070176
:1055A0001301200120012001200106F1080006213D
:1055B00041760A21817605F67411416040F2DC5192
:1055C00081600FF23430386105E106F108000621F0
:1055D00041760A21817605F6507141604FF496714B
:1055E0008160F8E006F108000C21417610218176F7
:1055F00005F5805190314160102181600FF24C30EF
:105600003861E8E006F10800072141760B21817638
:1056100005F58051843141600B2181600FF22C30FF
:105620003861D8E006F10800062141760A2181762A
:1056300005F5855141600A2181600FF21030386113
:10564000C9E006F10800062141760A21817605F5B8
:105650008051AC3141604FF4FA7181600FF2083033
:105660003861B8E006F108001421417618218176EE
:1056700005F595514160182181600FF25C30386169
:10568000A9E006F10800022141760621817605F5A0
:105690009051D4314160062181600FF204303861AD
:1056A00099E006F108000A2141760E21817605F580
:1056B0009051C43141600E2181600FF2C8203861E1
:1056C00089E006F10800012141760521817605F582
:1056D0009051DC314160052181600FF2E02038619A
:1056E00079E006F10800052141760921817605F56A
:1056F0009051B8314160092181600FF23420386146
:1057000069E006F10800062141760A21817605F557
:105710009051E43141600A2181600FF2F810386144
:1057200059E006F10800012141760521817605F551
:105730009051F031416040F2866181604BE006F1AA
:105740000800012141760521817605F5CC514160A3
:10575000052181603FE006F108000C21417610210F
:10576000817605F5C851883141601021816032E0B1
:1057700006F10800112141761521817605F5C85101
:105780009831416041F66631816024E006F10800FD
:10579000112141761521817605F55451416015217D
:1057A000816018E006F10800042141760821817625
:1057B00005F5C85178314160082181600BE006F1A0
:1057C0000800012141760521817605F580517C3163
:1057D00041600521816006F10800002101754175D5
:1057E00081750176C1600161417006F128080846A3
:1057F000C8F828004FF0FF3086F854007880062261
:1058000006F15800FDF784FD002010E000EB400198
:1058100006EB8101002281F8342034314A7005F111
:1058200058024A6006EB800100228A64401C02286C
:10583000ECDB002086F8280088F8010005F158000C
:10584000C8F80400FC60BDE8F08110B5164CFCF708
:10585000FBFFA067002006E0682111FB00417C31BE
:1058600044F82010401C1628F6DB4FF0FF3020666D
:1058700060660020A06605F05DFF06F0C2FD07F03F
:1058800066FAFBF7A5FB07F0E7FBFBF793FEFCF7D7
:1058900010F907F04BFC07F082FF07F04CFCBDE865
:1058A000104007F059BC000000600020F89900206B
:1058B0005860002041442025642025642025642070
:1058C00025642C2025640000524D20256420256489
:1058D00020256420256420256400000083520008F0
:1058E0004352000883520008655200085B530008C9
:1058F00067530008535300087353000843520008CD
:1059000073530008655200085B5300086753000892
:10591000535300089753000843520008835200086D
:10592000AF530008835300088D53000853530008F9
:10593000835200084754000883520008655200084B
:10594000CB530008DF530008F353000883520008CC
:105950005154000883520008655200085B53000848
:10596000675300086354000883520008F754000886
:1059700083520008655200087F5400088D540008C7
:105980009B540008835200081155000883520008F8
:10599000655200085B530008675300085353000822
:1059A0008352000837550008835200084955000803
:1059B000235500082D550008535300088352000852
:1059C0004352000883520008655200085B530008E8
:1059D00067530008535300088352000843520008DD
:1059E0008352000865520008235500082D55000811
:1059F00053530008002207F06FBF8268521C826078
:105A0000426832B10268531C036011704168491E3C
:105A10004160704708B584B00023029311B9009328
:105A2000019302E00090481E019004AB00A90748D2
:105A30007844183007F06AFF009909B100220A7013
:105A4000002858BF029805B000BD00BFAFFFFFFFA0
:105A500000F10103810704D010F8011B89B181070F
:105A6000FAD10268B2F10131914311F0803F04BFD5
:105A700050F8042FF6E710F8011B11B110F8011BC4
:105A8000FBE7C01A70470268531C0360117070472F
:105A900000B585B002460FF2140100A808F09EFD83
:105AA00000A800F093FB05B000BD00004F45256441
:105AB0000000000030488168002904BF08B008E0F9
:105AC000EFF30982A2F12802036882E8F84F8368A5
:105AD0005A6000F047FD816859B14A6892E8F84F72
:105AE000036002F1280282F3098813F47F4F36D055
:105AF0007047224822490968401A80F308884FF00D
:105B00008071C1611F4981617FF0060E704701BC41
:105B10002046DFF874E000BDFEE71C480068184925
:105B20000968401A203820F0070080F308884FF0F9
:105B3000000181F3118862B600F00DF8FEE74FF026
:105B4000000181F311881249124A0A604FF0800166
:105B500081F3118870470E490E4A0A6070474FF072
:105B6000000181F31188704700BF4FF0800181F37D
:105B70001188704700BF0000F8990020E05F002006
:105B8000784B030829E90008195B000800000008A9
:105B900004ED00E000000010EFF303807047BFF356
:105BA0004F8FDFF86C06016801F4E061DFF86426CE
:105BB00011430160BFF34F8FFEE770B582B0064618
:105BC0000C462046FFF744FF0546202D05D1042250
:105BD000314600A8FDF7CFFF06E0102D16D10222B6
:105BE000314600A8FDF7C7FF002000E0401CA84296
:105BF0000EDA015D7829F9D0009A2B465B1E1B1A3C
:105C0000DA4002F0010230398A42EFD0002076BD3E
:105C1000012076BDDFF80016016006207047A0F174
:105C20000060DFF8F81588428041C00F7047F8B572
:105C300004460D46002000902068FFF7F0FF002882
:105C40001AD000A8FFF7E6FF0646002700E07F1CF9
:105C5000B74211D2009850F8371000EBC7004068E7
:105C600040422268520810EB4200FFF7A6FF0028CE
:105C7000EDD02F600120F2BD0020F2BDF8B50C463A
:105C8000DFF89C150A6D4B6D002559082E465F1BE9
:105C9000062F11D3482707FB01273F6C874200D20C
:105CA0000D46B84200D20B46E918490837467E1C1B
:105CB0001F2FECD300E06D1C9D4211D2482707FB3B
:105CC00005210E6CB042F6D34E6C8642F3D34022CF
:105CD000204608F09DFC002084F840000120F2BD21
:105CE00040220FF20861204608F092FC0020F2BD2D
:105CF000F0B591B0044600250EE032590FF2F8518C
:105D000000A808F06BFC00A8FFF7A2FE024600A95D
:105D1000381D08F07DFC6D1C05EBC500C600305930
:105D200000280BD0371900A9FFF7A8FF0028E4D0FE
:105D3000402200A9381D08F06BFCECE711B0F0BD63
:105D4000F8B507460C461546002630460090002F51
:105D50001ED0002C09D1F2BD06EBC600C00057F8DA
:105D6000041B490849004151761C0C2E0FD200A992
:105D70003846FFF75CFF002807D13868FFF74FFF70
:105D8000002802D13F1DBC42F1D2BC42E4D23046D1
:105D9000F2BD70B5DFF88C140A460B68D21A13688E
:105DA000DFF88444A34201D0002070BDDFF87044C6
:105DB000121D22650968091F4822B1FBF2F16165D5
:105DC00010F1030F02D010F1130F0AD1DFF85C5469
:105DD000A86808F053FC0646A86808F05BFC811927
:105DE00005E008F065FC054608F064FC4119DFF8A1
:105DF0004054A069286005F14802A06AFFF7A0FF9F
:105E00002846FFF775FF012070BD0EB430B5CCB049
:105E1000044600A84FF49671FFF7ECFD00254FAB48
:105E200022464FF4967100A8FFF7F4FD00A8FFF793
:105E30000FFE044609E0DFF8E813C86D421CCA658E
:105E400000A9695C08F09EFC6D1CA542F3D34CB020
:105E500030BC5DF810FB38B50024DFF8C453E865AA
:105E60000FF29C40FFF7D1FFDFF8C80301680FF283
:105E7000B440FFF7CAFFA86C0090AB6B6A6B296B4C
:105E80000FF2B840FFF7C1FFE96C0FF2E840FFF7EF
:105E9000BCFF6A69A9690FF2F040FFF7B6FF0FF285
:105EA0000050FFF7B2FF06E01018021D0FF2085075
:105EB000FFF7ABFF641C04EBC400C200DC481158C0
:105EC0000029F1D10FF2FC40FFF79FFFA86D441E9F
:105ED000002505E00918BCA0FFF797FF641E6D1CA4
:105EE0003C2D09D2002C00D53B24322000FB04F1CC
:105EF000D1480A5C002AEDD131BDD048D0490A68AA
:105F000002604A6842608A688260CA68C2600A6940
:105F100002614A6942610A7E8261097F8161C949E1
:105F20000A7882614A6842628A688262CA68C2628A
:105F30000A6902634A6942638A698263CA69C26301
:105F40008A6EC0F88820C04A9369C0F89830D36838
:105F5000C0F88C301369C0F890305369C0F89430A1
:105F60000B6FC0F89C304B6FC0F8A0308B6FC0F83F
:105F7000A430C96FC0F8A810B4490968C0F8AC10C3
:105F8000B3490B68C0F8CC304B68C0F8D0308B6890
:105F9000C0F8D430CB68C0F8D8300969C0F8DC103C
:105FA0005168C0F8E8101168C0F8E410704770B587
:105FB00006460C469A4D6FF01E01401A14D0083860
:105FC00012D0001F05D0001F0ED008380CD0001FC3
:105FD00010D104F120002862EFF3148040F0020099
:105FE000E862286AA86205E004F120002862EFF365
:105FF0001480E862EFF308806862EFF3058028639D
:10600000EFF300806863FFF7C7FDA863EFF310802C
:10601000E863EFF311802864EFF313806864F1EE16
:10602000100AA864EE64002004E054F8201045F83B
:106030002010401C0828F8D370BD70B5784CA16DB5
:106040003C2901D30021A165A56D32217A4A01FBCB
:1060500005260A4601463046FDF78DFD002086F8EC
:106060003100681CA06570BD70B5014674462046BD
:10607000FFF79DFFFFF741FF2046FFF78AFE00F084
:106080009AF8002832D100F034F808F01BFBF32016
:1060900008F092FB6F484FF00054002505E021788E
:1060A000641C08F06FFB30466D1C461CB5F5C03F04
:1060B000F5D3532108F066FB5221304608F062FB0D
:1060C000741C4121204608F05DFB641C4D212046D4
:1060D00008F058FB6048C046C04604F10D00FFF7C9
:1060E000BAFE08F0F8FA5D4800F01FF8BDE870400D
:1060F00055E510B508F0E6FAF32008F05DFB584CC2
:106100003820206002E020680830206020684028A5
:1061100007D2002108F0E5FA0928F4D0FFF73FFD87
:10612000FCE7BDE8104008F0D6BA38B5044608F0E0
:10613000C9FAF32008F040FB3E480168204608F009
:1061400005FB241DFF21204608F01CFB641C424D6A
:106150006979204608F016FB641CE978204608F0AF
:1061600011FB641C2979204608F00CFB641C29787B
:10617000204608F007FB641C6978204608F002FB03
:10618000641CA978204608F0FDFAF521601C08F08F
:10619000F9FABDE8314008F09EBA80B508F092FAED
:1061A000F32008F009FBAA212E4808F0EBFABDE81D
:1061B000014008F090BA00202A490978F52900D159
:1061C000012070470000000025730A0010B5044646
:1061D000FFF73EFCC0B2142800D31320024621462C
:1061E0002148FDF7C8FC4FF0AC30007810BD80B5F9
:1061F00000F04BF8BDE80140D1E480B5FFF7CDFFDA
:106200004FF4C83213490020BDE8084001F03FBCFC
:106210000CED00E00400FA059899002001F8020056
:1062200010560120FC4F0508FECAFECAF89900204E
:106230003C1E01202C9B002010E60020244501205C
:1062400000ED00E020ED00E004E000E0A0ED00E063
:1062500034EF00E0000006087C650120F4FF070829
:106260000C660120FFFF0708F462012010B500F062
:106270001BF80FF270142046FFF7EAFB0246214696
:106280000020BDE8104001F002BC80B501214FF4B0
:10629000802002F063FF012003F032FB94210F20E5
:1062A000BDE8044003F0CFBC80B501214FF480204D
:1062B00002F054FF012003F023FB00210F20BDE872
:1062C000044003F0C0BC10B5002401214FF480202D
:1062D00002F044FF012003F013FB0F2003F0C0FC89
:1062E000942800D10124204610BD00004E6F205399
:1062F000796D626F6C0000003078253038780000CE
:106300000A0A0A0A3D3D2043726173682044756D94
:106310007020496E666F726D6174696F6E203D3DCD
:106320000A0000004669726D7761726520566572D9
:1063300073696F6E203A2025640A00000A495053A1
:1063400052203D20307825782C2041505352203D5A
:1063500020307825782C2078505352203D203078FA
:1063600025782C205046534352203D203078257804
:106370000A0000000A6661756C74206D6F64652008
:106380003D203078257800000A5043203D203078A9
:1063900025782C204C52203D20307825780A0000AA
:1063A0000A3C43726173682043616C6C20537461D2
:1063B000636B3E0A000000003078257820202573AA
:1063C0000A0000000A0A3D3D20526563656E742094
:1063D0004C6F67204D65737361676573203D3D0A9F
:1063E00000000000534E414D590000000000000025
:1063F00038B5FFF7BAFBDFF830068468DFF8280607
:1064000000210171FFF7ABFB002C2CD02068002885
:1064100029D0607C2168497CC0B2814223D12568A3
:1064200000E00D002968002903D04A7CC0B28242F6
:10643000F7D0FFF79AFBDFF8F0050069A04203D11F
:10644000DFF8E40521680161E06921680160C86145
:10645000E56129682160002900D0CC612C6095F8A5
:10646000410085F84000FFF77AFB31BD10B5FFF71A
:106470007CFBDFF8B8050468DFF8AC05006A201A79
:10648000012832DADFF8A005046A04E0DFF8980595
:106490000462FFF764FBDFF898050078C00722D597
:1064A000FFF763FBDFF8880500788007EED5DFF89B
:1064B0008005007810F0FD00DFF874150870FFF714
:1064C0004EFBDFF86405006A8442FAD0DFF8580515
:1064D0000462DFF858050068401CDFF850150860BA
:1064E000DFF844154862FFF740FB10BD38B50400E3
:1064F0000020A071206A10F57A606062E0690028CF
:1065000002D02000E1698847FFF729FBE56809E030
:10651000E868616A401A002801D5E8686062FFF700
:106520001EFB2D68002D1AD0FFF71FFB20690028E5
:1065300004D0687C2169497C884212D3287C4007BA
:10654000EDD5E868216A401A0128E1DA280000F058
:106550009EF9FFF70AFB287C0028D9D101E0FFF75C
:1065600004FB31BD70B50400002060700120207074
:1065700008F09EF80078C0B2CD2802D07D20FFF749
:1065800087FAA06800280CD0A068406C002808D0CA
:10659000A068406C01680800002802D0A06840682C
:1065A000884794F8290000280BD0A06894F8281098
:1065B00080F84010DFF870040079002801D0FFF760
:1065C00017FFDFF870040078002823D0DFF8680494
:1065D0000068DFF85414096A401A002804D5DFF86F
:1065E00054040021017015E0FFF7BFFA08F0A9F983
:1065F0000500FFF7B4FAA068002808D0A068406B37
:106600002818DFF838140968401AA1684863DFF8D1
:106610002C040560A068002808D0A068007C002831
:1066200004D1A068006B401CA168086320690028A1
:106630002BD003E030682061FFF791FAFFF795FA5D
:106640002669002E27D0357CEDB2002D23D06807B7
:1066500010D5F068216A411A012906DA300000F0ED
:1066600016F9307C002805D10FE0616A411A002933
:1066700000D56062EDB215F0FB001028DAD1B068E9
:1066800080684068007C0028D4D1FFF76EFA02E0F1
:106690002000FFF72BFFA0790028F9D1DFF8900345
:1066A0000078C00701D5FFF7E1FE00206071206986
:1066B000002839D02069007C002805D02069806836
:1066C00080684068A06001E02069A060A06890F840
:1066D0004C00642802D08020FFF7DAF9A068806AB5
:1066E0000078CD2802D07820FFF7D2F9A068406C5E
:1066F000002808D0A068406C41680800002802D03B
:10670000A06840688847A06890F8400084F8280096
:1067100084F82900DFF810038068C06A401CDFF8A5
:1067200008138968C8620BE0002084F82900002063
:1067300084F828000020A06000202070FFF70FFAE6
:10674000200070BD80B508F029F9DFF8F41209784F
:10675000002806D0022810D009D3042815D010D361
:1067600014E0002902D0A320FFF792F911E00029DC
:1067700002D1A420FFF78CF90BE0A620FFF788F9DF
:1067800007E0A720FFF784F903E002E0A820FFF765
:106790007FF901BD10B508F001F90400DFF8A0028F
:1067A0000078002802D0A020FFF772F9002C05D055
:1067B000022C08D003D3032C09D00CE00EE0A42057
:1067C000FFF766F90AE0A620FFF762F906E0A720C6
:1067D000FFF75EF902E0A820FFF75AF910BD80B577
:1067E00008F0DCF8002805D0022808D006D30328DA
:1067F00009D00CE0A320FFF74BF90BE00AE0A6203C
:10680000FFF746F906E0A720FFF742F902E0A820CB
:10681000FFF73EF901BD80B5DFF80C0200780028D3
:1068200002D19720FFF734F9DFF8FC010078401E11
:10683000DFF8F4110870C0B2002827D1DFF8E801B2
:106840004068002822D0FFF790F9DFF8DC014068AB
:1068500000280BD0DFF8D00101210170DFF8C8015A
:10686000FFF76DF9DFF8C00100210170DFF8B80112
:106870004078F021084202D09920FFF709F9DFF8AB
:10688000A8014078002801D1FFF769F901BD10B5D2
:10689000816800290CD0DFF89011096AC160816815
:1068A0000A684968002A00D051600A6000218160AE
:1068B000017C11F003010174C9B2002945D1DFF850
:1068C00068110969002929D1DFF85C110861DFF836
:1068D0005801007800280CD1DFF84C01012101702B
:1068E000DFF84401FFF72BF9DFF83C0100210170CC
:1068F00003E0DFF8340101214171DFF82C01407819
:10690000F021084202D09920FFF7C2F8DFF8180101
:106910004078002801D1FFF722F916E0427C4B7C39
:10692000D2B29342D0D38142D1D04B7CD2B29A42E0
:106930000BD10300FFE71B68002BDED05C7CD2B2DA
:10694000A242DAD18B42F6D1BEE710BD10B50400E9
:10695000627C35480078401C33490870394800E0B3
:1069600008000168002903D04B7CD2B29A42F7D3C9
:106970002160E061046000290AD0CC61487CD2B279
:10698000904202D194F8410000E0002084F84000D9
:10699000207C002812D1FFF7E8F82000FFF777FFEE
:1069A00021484078F021084202D09920FFF770F882
:1069B0001D484078002801D1FFF7D1F8FFF72BFFE1
:1069C00010BD10B51848047817480078401C1649C7
:1069D00008701548FFF7B3F8134804701248407860
:1069E000F021084202D09920FFF752F80E48407873
:1069F000002801D1FFF7B3F810BD10B507F0D4FFA0
:106A000009480121017007F053FE04006846C046A2
:106A1000021B203A012A03DBCD212000FCF778FC81
:106A200009480121017010BDF8990020606601201D
:106A3000B3660120B46601207866012064660120F7
:106A4000B5660120049A0020B7660120DFF8B4067D
:106A5000007870472DE9F0418AB0FBF7F5FE044657
:106A6000DFF8A4562E6842E096F9080007283DD0CA
:106A70000B283BDA062839D006F10807B86C002845
:106A800003D5D4F880100818B8644FF0FF313046B1
:106A9000FA6D926990478046B8F1010F04D197F8DA
:106AA0004C00B96D09698847B8F1020F0BD1797EA6
:106AB00038697A688018BA6D52699047002802D008
:106AC000304608F02FF800213046FA6D9269904761
:106AD000022801D10120B87501213046FA6D926972
:106AE0009047022802D1304608F0C8F83668AE4216
:106AF000BAD1D4E91C01002901D100280CD00A2008
:106B00008DF8080002208DF80000D4F88000ADF860
:106B1000220000A801F0F2FF01200AB0BDE8F081D8
:106B200030B585B004460D46CA208DF8000028888F
:106B3000ADF801000220ADF80300BDF80100001D12
:106B400003F01CFBCDF8090002220DF10301FDF753
:106B500012F802222946DDF80900801CFDF70BF827
:106B60002A882146DDF80900001DFDF704F8002001
:106B7000288000A9DFF8E40D08F092FB05B030BDD5
:106B800042F23411081A322801DA0120704700203D
:106B9000704780B5FBF793FA407B002804D007F0DC
:106BA0002FFFDFF8941E086001BD80B507F028FFB5
:106BB000DFF8881E086001BDDFF8800E00687047AE
:106BC00010B582B000F10C03D96A896800910422E3
:106BD00000A95C7DDB68C06818182018FCF7CBFFA3
:106BE00013BD30B41488651C1580052565541488C0
:106BF000651C1580635413885C1C1480007A5854FB
:106C000030BC704732B515461C4621884A1C22808C
:106C100037224A5521884A1C2280007A4855022290
:106C200000A920884019FCF7A6FF2088801C20803E
:106C300031BDF8B517461D4600F10C06069CA4B2FE
:106C4000B27D6243C06809182888C019FCF793FF19
:106C50002888B17D614311FA80F02880F1BD30B4FD
:106C600000F110039B7C914203D1006990FBF3F08B
:106C70000DE00C46154603D2281B90FBF3F006E00E
:106C80000069001B90FBF3F095FBF3F1081880B24C
:106C900030BC704700F110018A688B7CD2188A6082
:106CA0000069824201D1002088600020887370470B
:106CB000F8B504460D461E46069F92B289B2FFF70C
:106CC000CEFF00903B46324629462046FFF7B1FFF3
:106CD000F1BDF8B5044615461E462269002D00D1C7
:106CE0001546069F0097FFF7E3FF2069854206DA05
:106CF000009733462A4600212046FFF7D9FFF1BD11
:106D00002DE9FC4104460D461646A169606900283C
:106D100015D500270A4692B289B22046FFF79FFF99
:106D2000804633462A4641462046FFF76BFFA2695C
:106D300000962B4611462046FFF7CBFF2EE08142FE
:106D400016DA01270A4692B2014689B22046FFF7B9
:106D500086FF804633462A4641462046FFF752FFCB
:106D600000962B46A26961692046FFF7B2FF15E045
:106D700002270A4692B2014689B22046FFF76FFF0A
:106D8000804633462A4641462046FFF73BFF0096A1
:106D90002B46A26961692046FFF78AFFA06901902E
:106DA000606900903B46424694F908100FF20800D3
:106DB000FBF707FABDE8F3815061636B203D256462
:106DC000202564202564202564202564000000001F
:106DD00070B582B004460D461646A06C012811DA43
:106DE000A07F012811D133462A4601212046FFF712
:106DF00009FF0120009033462A46A1692046FFF78B
:106E000018FF02E02046FFF77BFF012332462946A8
:106E10002046FFF7E6FEA0696061A36CE26C94F97E
:106E200008100FF20C00FBF7CCF9A06CE06473BD06
:106E3000666C757368202564202564202564000035
:106E40002DE9F84304460D461646FBF7FDFC814646
:106E5000FBF735F9804604F10807B87D002802D019
:106E60002046FFF7ADFE386C0128C0F2898098F803
:106E70000E00002844D0B87D002800F0C580786C52
:106E8000D9F88010401A7864B87E3969FA68531AC4
:106E9000834205D0002A2FD1BA68511A81422BD1E2
:106EA00094F90820397E0FF26410FBF78AF9397ED5
:106EB00000291ED094F908200FF26810FBF781F921
:106EC0003869B97E421892B2F96889B22046FFF754
:106ED000C6FE33462A4601462046FFF793FE00963B
:106EE0002B463869B97E4218F9682046FFF7F1FE53
:106EF00002E04FF0FF30F8602046BDE8F243C9E6FB
:106F000098F80E00002840F07F80786CD9F8801047
:106F1000401A786401282CDA386C7864386BD0F821
:106F20000C8094F908308268396C0FF21410FBF76A
:106F300048F9B868B97E90FBF1F0396C91FBF8F133
:106F4000814202DB4FF0FF30F860B87D00280AD0A4
:106F50002046FFF79FFE324629462046FFF7D0FE27
:106F60003869F86050E0324629462046BDE8F843CB
:106F7000C6E6B87D002847D02046BDE8F24389E642
:106F8000B87D002840D094F9080098F80A1000292C
:106F90001BD0072803D00D2801D015282FD1334648
:106FA0002A4601212046FFF72DFE0120009033469E
:106FB0002A4639692046FFF73CFE7A7894F9081092
:106FC0000FF29000FBF7FDF819E0092809D194F8B9
:106FD0005E10012905D10FF28C00BDE8F443FBF7E8
:106FE000F0B833462A4601212046FFF70BFE012068
:106FF000009033462A4639692046FFF71AFE20469C
:10700000FFF748FE3869F860BDE8F1837375737067
:10701000656E64206669666F2066756C6C202564F9
:107020002025640073757370656E64206669666FF1
:107030002066756C6C2032202564202564000000D9
:107040006669666F2066756C6C3320256420256444
:107050002025640041502053757320256420256449
:1070600000000000233E6C75785F73617420256416
:1070700000000000F8B504460D46234E376805E0D1
:107080002A4621463846FFF7DBFE3F68B742F7D174
:10709000F1BD2DE9F04104460D46DFF82C6DF7698E
:1070A00007F10C0898F81510D8F80C00FA68801849
:1070B000D8F854205269904700280AD0012088F857
:1070C0001200787A002804D02A4621463846FFF775
:1070D000B7FEB66906F10C07797DF868F26880188A
:1070E0007A6D52699047002809D00120B874707AEF
:1070F000002804D02A4621463046FFF7A1FE012091
:10710000BDE8F081AF6601206C6900200288D21CC6
:1071100002800A80704780B50B889B1AADF800305A
:10712000BDF80030002B09D01018012100F8031C15
:10713000022200A9801EFCF71EFD01BD0888C01EAA
:10714000088001BD2DE9F04FADF68C2D04460D46AB
:10715000FBF77AFB8046FAF7B2FF074610A840F625
:107160004821FEF747FC00208DF8020006A82821E0
:10717000FEF740FC01A81421FEF73CFC0020ADF80E
:1071800000000646D8E91C01002902D1002800F0C1
:10719000E18397F9090008F095FD002800F0DA83F3
:1071A00000A92846FFF7B2FF37461BE00120314611
:1071B0003A4608F0B1FFD8E91C231040194001D12C
:1071C00000280ED007EB8700DFF8001C01EBC0029F
:1071D00092F90900012804D10DF1020110A8126AE8
:1071E00090477F1C2D2FE1DB37461AE02888411C91
:1071F000298099F8021001552888FFF7C1FC002862
:107200000DD0BDF8002029462046FFF784FF29460F
:107210002046FFF785FC00A92846FFF777FF7F1C73
:107220007FB29DF80200874280F28C832988481C37
:10723000288040F2491010FB07F010AA825C0A5522
:1072400029884A1C2A8010AA00EB020898F801003D
:1072500008552888411C298008F1010999F8011076
:10726000015599F80100032821D0092800F04C812C
:107270000C2800F026811A2800F04A821B2800F012
:1072800059811C2800F078821D2800F066811E2894
:1072900000F06282252800F0A182262800F0DB821F
:1072A000282800F0B6822C2800F0E5829EE798F8A6
:1072B0000100032805D12888411C298099F8021073
:1072C00001552888411C298099F80310015599F827
:1072D0000300C0280DD1B8F83020D8F83210288823
:1072E0000019FCF748FC2888B8F8301008182880E6
:1072F00082E7711C00064ED401A808F104025278FE
:107300003254C9B298F806200A54491CC9B2002266
:107310000A544A1C08F20601D2B24B781354521C8C
:10732000B8F80E30D2B21E0A1654521CD2B2135400
:10733000521C08F20E03D2B29E781654521CD2B2DE
:10734000DB781354521CD2B298F812301354521CEA
:10735000D2B298F813301354521CD2B28B78135413
:10736000521CD2B2C9781154511CC9B298F80A20E3
:107370000A54491CC9B298F80B200A544E1CF6B2A4
:10738000324601A928880019FCF7F5FB288850FA35
:1073900086F0288030E7D8F8052006A8130C33546F
:1073A000C9B2130A0B54491CC9B20A54491CD8F873
:1073B0000920C9B2130C0B54491CC9B2130A0B544F
:1073C000491CC9B20A54491CD8F80D20C9B2130C83
:1073D0000B54491CC9B2130A0B54491CC9B20A54B4
:1073E000491CD8F81120C9B2130C0B54491CC9B25E
:1073F000130A0B54491CC9B20A54491CD8F8272057
:10740000C9B2130C0B54491CC9B2130A0B54491CC2
:10741000C9B20A544A1C08F22701D2B20B7913549C
:10742000521CD2B24B791354521CCB88D2B21E0AD2
:107430001654521CD2B21354521CD2B2097A1154AF
:10744000511CD8F81520C9B2130C0B54491CC9B2F1
:10745000130A0B54491CC9B20A54491CD8F8192004
:10746000C9B2130C0B54491CC9B2130A0B54491C62
:10747000C9B20A54491CD8F81D20C9B2130C0B54C8
:10748000491CC9B2130A0B54491CC9B20A54491CFD
:10749000D8F82120C9B2130C0B54491CC9B2130AE5
:1074A0000B54491CC9B20A544E1CF6B2324606A906
:1074B00028880019FCF75FFB288850FA86F028809E
:1074C0009AE608F20301B1F90300C0F3072242EA89
:1074D0000020A1F80300B1F90700C0F3072242EA37
:1074E0000020A1F80700B1F90500C0F3072242EA25
:1074F0000020A1F80500092228880019FCF73BFBB1
:1075000028880930288077E698F8010003280AD1F6
:10751000022208F1030128880019FCF72CFB2888B7
:10752000801C288068E62888411C298099F8021070
:10753000015561E62888411C298099F802100155FF
:1075400098F8010005287FF457AE2888411C29804F
:1075500008F10401497801554EE608F2030998F84C
:107560000100012840F0C4802888411C298099F836
:10757000041001554FF0000AA1E0CAEB4A1000EBDD
:10758000090BDBF81800010221F0FF11000A00F0DE
:10759000FF100843CBF818004FEA3040CBF8180032
:1075A00004220BF1180128880019FCF7E4FA288856
:1075B000001D2880DBF80800010221F0FF110012F5
:1075C00000F0FF100843CBF80800C0F30F4141EA78
:1075D0000040CBF8080004220BF1080128880019AC
:1075E000FCF7C9FA2888001D2880DBF80C0001028E
:1075F00021F0FF11001200F0FF100843CBF80C003F
:10760000C0F30F4141EA0040CBF80C0004220BF11B
:107610000C0128880019FCF7AEFA2888001D288084
:10762000DBF81000010221F0FF11001200F0FF1042
:107630000843CBF81000C0F30F4141EA0040CBF8FB
:10764000100004220BF1100128880019FCF793FAAE
:107650002888001D2880DBF81C00010221F0FF11A2
:10766000000A00F0FF100843CBF81C004FEA30403E
:10767000CBF81C0004220BF11C0128880019FCF730
:107680007AFA2888001D2880BBF81600010A41EA12
:107690000020ABF8160002220BF116012888001911
:1076A000FCF769FA2888801C2880411C298080B258
:1076B000DBF8201001550AF1010A5FFA8AFA99F8FD
:1076C00004008245FFF659AFB8F84321D8F84511B8
:1076D00028880019FCF74FFA2888B8F843110818D1
:1076E0002880B8F843110FF27820FAF76AFD83E595
:1076F00005287FF481AD2888411C298099F8021063
:1077000001552888411C298099F80310015573E51B
:1077100008F2030198F80100032805D12888421CCB
:107720002A8098F80A200255D1F80100020222F0BE
:10773000FF12000A00F0FF101043C1F801004FEAE9
:107740003040C1F80100072228880019FCF713FA1D
:107750002888C01D28804FE508F203010888020A26
:1077600042EA00200880022228880019FCF703FA68
:107770002888801C28803FE508F2030098F8011053
:1077800001297FF439AD99F80210012918D129880F
:107790004A1C2A8000780855B8F80420D8F806104A
:1077A00028880019FCF7E7F92888B8F804100818A9
:1077B0002880B8F804100FF2BC10FAF702FD1BE5A0
:1077C00002297FF419AD29884A1C2A8002780A55BB
:1077D00029884A1C2A80C07908550DE52888411C53
:1077E0002980B9F8021001552888411C2980B9F96F
:1077F000021009120155B9F90220D8F8051028889D
:107800000019FCF7B8F92888B9F90210081828807F
:10781000F2E42888411C2980B9F802100155288813
:10782000411C2980B9F90210091201552888411C10
:10783000298008F1040149780155B9F90220D8F8E6
:10784000061028880019FCF796F92888B9F9021063
:1078500008182880D0E408F203010888020A42EAE6
:1078600000200880022228880019FCF784F9288863
:10787000801C2880C0E408F203082988084698F88C
:10788000002013072AD5491C298098F800100155BB
:107890002888411C298098F8071001552888411C28
:1078A000298098F808100155D8F80900010221F044
:1078B000FF11000A00F0FF100843C8F809004FEA62
:1078C0003040C8F80900042208F10901288800198D
:1078D000FCF751F92888001D28808DE4520724D533
:1078E000491C298098F8001001552888411C2980DE
:1078F00098F801100155D8F80300010221F0FF119A
:10790000000A00F0FF100843C8F803004FEA3040B7
:10791000C8F80300042208F1030128880019FCF7C5
:107920002AF92888001D288066E498F80220D8F8F3
:107930000D100019FCF71FF9288898F8021040185C
:10794000288059E4BDF8002029462046FFF7E3FBD4
:1079500008F0E5F90DF68C2DBDE8F08F689D00204C
:107960004F4A483A20415442442073697A653A208C
:10797000256400004F4A483A204150445220736920
:107980007A653A20256400002DE9F04105460E464F
:10799000FAF795FB0746DFF838442078401C207042
:1079A0006078F021084202D09920FEF771F8FEF7C6
:1079B000DCF86078401C607097F81880B8F1010F0F
:1079C00026DB3088404480B2FFF7DAF8002803D085
:1079D00031462846FFF7A4F83088411C3180032146
:1079E00041553088411C318000F80580424607F13E
:1079F000190130884019FCF7BEF8308840443080C7
:107A0000FF22002107F11900FBF782FC00203876E5
:107A10006078F021084202D09920FEF739F86078AA
:107A2000401E6070C0B2002801D1FEF798F8BDE892
:107A3000F041FEF7F0BE00003C66012040660120E8
:107A400038B504460D46FAF73AFB817A002909D188
:107A5000417B002906D129884A1C2A8006220A5522
:107A60000121417331BD38B504460D4628880028F0
:107A70000CD02046FFF788FF29462046FFF7E0FF9D
:107A800029462046BDE83440FFF74AB831BD14B559
:107A900085B0049101A90022134614461CC10A2195
:107AA000ADF8001004218DF804108DF805000A4689
:107AB00005A90DF10600FCF75EF8042204A90DF1FA
:107AC0000A00FCF758F800A901A8FFF729F806B04A
:107AD00010BD80B5FAF7F3FA4FF49671FAF7DCFCB3
:107AE00007208DF802000120ADF8000000A90DF17B
:107AF0000200FFF715F801BD2DE9F041DFF88C4DCC
:107B00006068002828D0218888421FD002F036FB08
:107B1000054666682788A6EB07081FFA88F84246DC
:107B2000381900F108012846FCF725F83A4604F117
:107B3000080108EB0500FCF71EF83246294604F15F
:107B40000800FCF718F8284602F030FB626804F1E0
:107B500008010520FFF79BFF002060602080BDE842
:107B6000F08180B5FAF770FE062180F88410843029
:107B7000417007218170C170017101BD2DE9FC4187
:107B800005460F469046FAF79AFA0026D5F80910EE
:107B90000C1D2A781146012962D00F2933D03529CE
:107BA00037D0802900F08A80812900F091808229D5
:107BB00000F08E80852900F08B80862900F0888077
:107BC000882900F085808A2900F08A808B2900F0BE
:107BD000A3808C2900F0AF808D2900F0B780DD29CB
:107BE00000F0C180DF2900F0DB80F0291AD0F429F1
:107BF00023D0F62929D0F82947D0F92935D0FF29F3
:107C000000F0A98061E0807D2070FFF7AAFF0120CD
:107C10005CE00120FAF7CBF83046FAF7CCF8012007
:107C2000207053E00422DFF8681C2046FBF7A3FF16
:107C30000120FDF731F8012048E0042200F1100195
:107C40002046FBF798FF012040E003222146304602
:107C5000DFF8403C9B681B6E1B6A9847012035E0AB
:107C6000204608F089FA012030E0B5F80120B5F887
:107C70000300C010C0EB0011D5F8050000EB811126
:107C80002046FBF778FF012020E03046ADF80400E5
:107C90000120D5F80510C9B2012900D10320FCF755
:107CA00064FAFCF79EFAADF80400FCF7B1FA022280
:107CB00001A92046FBF75FFF012007E0D5F805008A
:107CC00020702146304607F097F83046BDE8F6812F
:107CD00030462070214602F07F0007F08DF8F4E76F
:107CE00001202070DFF8AC0B45683746287F00285C
:107CF00001D13046EAE7687A002803D1286E40684F
:107D0000804707462046296EC9698847002FDCD086
:107D1000286E80688047D8E70120B5F80310C1F3CA
:107D2000C101091D884040F0020020702146012059
:107D300007F062F8C9E701782170C1786170417974
:107D4000A1708079E07001202071BFE7204608F023
:107D500027FA0646B9E704F10802211D2046FDF77F
:107D600049F80120B2E76879DFF8281B51F8205064
:107D7000687A002810D0424639462846FFF728F88E
:107D8000DFF8140B01210170DFF8101B082008F048
:107D9000C9FA0120207001E030462070012095E7EB
:107DA0006879DFF8F01A51F82050286995F8221008
:107DB00090FBF1F0401E0090042200A92046FBF742
:107DC000DAFE012082E7000000600020C8F10020F8
:107DD000F8990020F0B593B00646FAF770F9054619
:107DE000FAF732FDD6F809100C1D317800220892FE
:107DF0004FF0FF32099217460A46312A00F01E81E1
:107E0000322A00F02581332A00F03181342A00F033
:107E10003881372A74D0A12A00F06081A22A00F0AC
:107E20007F81A42A00F08A81B12A00F03483B22A2B
:107E300000F0CF84B82A00F09C81C12A00F0CA81EA
:107E4000CD2A00F08B80CE2A00F0A180D02A37D036
:107E5000D12A2BD0D22A38D0D32A3FD0D42A41D00D
:107E6000D62A58D0D72A56D0D82A5CD0D92A5AD068
:107E7000DB2A00F01E81DC2A00F02281F12A5AD090
:107E8000F22A00F09D80F52A00F0B180F72A00F078
:107E9000C480FA2A00F0DD84FB2A00F0DD84FD2A8C
:107EA00000F0B080FE2A00F0E784C4E000212846FC
:107EB000FAF730FB0020A873FFF71EFE0120BBE09D
:107EC0000020FCF7E9FE0120B6E001212846FAF780
:107ED00021FB012008F076FA0120ADE00020A87215
:107EE0000120A9E00120A872002068730120A87376
:107EF000E87A002802D1012008F064FA01209BE012
:107F0000002221461046DFF88C391B681B6E1B6A65
:107F10009847012090E0D62901D1012000E00020FF
:107F2000E872012088E0D92901D1012000E0002079
:107F30002873012080E000210CE00A180B5D82F814
:107F40008430022905D10A5D80F887200A5D80F817
:107F50008820491C0329F0DB01206DE0002512E098
:107F6000DFF83009466806EB4506022204EB4501BE
:107F700006F15800FBF7FFFDB6F95810DFF82009AD
:107F8000FAF71FF96D1C032DEADB012054E00025F0
:107F900012E0DFF80009066806EB4506022204EB52
:107FA000450106F15800FBF7E6FDB6F95810DFF879
:107FB000F408FAF706F96D1C032DEADB01203BE01B
:107FC000297C090601D4012036E02178A0F88A1026
:107FD0006178A0F88C1002212046DFF8B828D26919
:107FE000126E92699047002825D0012024E00322D8
:107FF00021460120DFF89C389B681B6E1B6A98475E
:10800000012019E01B2221460720DFF888389B68F1
:108010001B6E1B6A984701200EE0DFF8780886691E
:10802000306E80688047002805D001222146052057
:10803000336E1B6A9847002013B0F0BDF9F7BFFEFE
:10804000012801D10120F7E72046F9F7E3FDF2E727
:10805000F9F7B5FE012801D10120EDE72046F9F737
:108060005EFE20780028E6D0F9F78AFEE3E7F9F70C
:10807000A6FE012801D10120DEE72078F9F787FE6E
:10808000D9E7F9F79CFE012801D10120D4E74FF48C
:1080900080510020FAF777FA0120F9F70FFD01204F
:1080A000F9F789FE2078F9F78DFEF9F77AFD0120BE
:1080B000C2E7D6F80510DFF8F007FAF782F8BAE75A
:1080C000FEF779F8002802D0FEF797F8B3E7FEF73D
:1080D000FAF80028AFD0FEF7C9F8ACE794F90050E1
:1080E0000422611C08A8FBF746FDB6F8010006282B
:1080F00006D30422611D09A8FBF73DFD94F9097020
:10810000042D04D1DFF88C070069A17A81720097F1
:10811000099B00220899284606F0CEFE20708AE7C7
:1081200094F900500422611C08A8FBF724FD0023E9
:108130001A460899284606F029FF7DE794F9005071
:108140000422611C08A8FBF716FDB6F801000628FA
:1081500006D30422611D09A8FBF70DFD94F90970EF
:108160000097099B00220899284606F061FF2070BD
:1081700061E720780146032908D01A2913D0252960
:1081800015D0282917D02C2919D01CE060788DF83B
:108190000A00012805D1A0788DF80B00204600F0D8
:1081A00044FC012048E7204600F03FFCF9E7204668
:1081B00000F03BFCF5E7204600F037FCF1E72046F5
:1081C00000F033FCEDE794F9011040B207F047FEF0
:1081D000C0B231E7207801460E3908D0091F0329C3
:1081E0001CD9091F3DD0491E00F09B803DE10E20A7
:1081F0008DF8080060788DF80A00A1788DF80B10D2
:10820000E2788DF80C200023ADF80D3052B249B25F
:1082100040B2FAF7D0F900F0FFFB26E18DF8080034
:10822000122802D160788DF80A009DF80800132802
:1082300002D160788DF80B009DF80800142802D157
:1082400060788DF80C009DF80800152802D1607840
:108250008DF80A0062782178DFF85006F9F7B1FF4F
:1082600003E16078A178090401EB0060E17800EB9C
:10827000012021794018CDF80A006179A279120411
:1082800002EB0161E27901EB0221227A8918CDF833
:108290000E10627AA37A1B0403EB0262E37A02EB0C
:1082A0000322237BD218CDF81220637B8DF8163081
:1082B000A37B8DF81730E37B8DF81830237C8DF885
:1082C0001930637C8DF81A30A37CE57C15EB032311
:1082D0001BB21D46ADF81B50257D03EB0523657DC4
:1082E0005B19ADF81D30A37D8DF81F30002803D138
:1082F000002901D1002A09D00DF10A0184B0684695
:108300001622FBF7FDFB0FBCFAF7FAF90DF10A0193
:1083100084B068461622FBF7F3FB0FBC00F0C4FBE9
:10832000A3E060788DF809001D283DD1A0788DF874
:108330001300A07801280DD1E078217911EB0021FC
:10834000ADF80A1089B20A461D21DFF86405F9F775
:1083500038FF8AE002280BD1E078217911EB002167
:10836000ADF80C1089B2DFF84C05F9F72AFF7CE074
:1083700003280BD1E078217911EB0021ADF814101E
:1083800089B2DFF83405F9F71CFF6EE004286CD1E0
:10839000E078217911EB0021ADF8161089B2DFF8F1
:1083A0001C05F9F70EFF60E0262809D1A0788DF8AA
:1083B0000E00A078012858D1E0788DF80D0054E027
:1083C0001C2823D1A0788DF80D00A078012807D1B2
:1083D000E1788DF80A10DFF8E804F9F7F2FE44E0DE
:1083E000022807D1E1788DF80B10DFF8D804F9F7EF
:1083F000E8FE3AE0032838D0052836D1E1788DF838
:108400000C10DFF8C404F9F7DCFE2EE02C282CD188
:10841000A0788DF81400A078012803D1E0788DF8B9
:108420000E0022E0022806D1E078217911EB00202D
:10843000ADF8150019E0032806D1E078217911EB99
:108440000020ADF8170010E0042806D1E07821796B
:1084500011EB0020ADF8190007E0052805D1E07800
:10846000217911EB0020ADF81B0006208DF82800C3
:1084700020780B900DF1310002A91822FBF740FB88
:108480000B208DF830000020ADF84A000AA800F05B
:1084900035FBC0B2D0E594F9000006F050FF01288A
:1084A00040F0698120780146032928D0062965D04B
:1084B00009292BD00C2945D00D2951D0192900F0BC
:1084C00090801A2967D01B2900F0A0801C2900F099
:1084D000DB801D2900F0B3801E2900F0E2802529F1
:1084E00000F0FB80262900F0EA80272900F0FC80BC
:1084F000282900F020812C2900F0218136E1032277
:10850000611C0DF10A00FBF736FB34E10722611C08
:108510000DF10A00FBF72FFBBDF80A00010A41EA42
:108520000020ADF80A00BDF80C00010A41EA002065
:10853000ADF80C00BDF80E00010A41EA0020ADF8CC
:108540000E0018E10322611C0DF10A00FBF713FB7A
:10855000BDF80B00010A41EA0020ADF80B000AE16A
:108560000322611C0DF10A00FBF705FBBDF80B00AF
:10857000010A41EA0020ADF80B00FCE00122611C79
:108580000DF10A00FBF7F7FA9DF80A100FF24030E0
:10859000F9F717FEEFE00B22611C0DF10A00FBF763
:1085A000EAFADDF80B00010221F0FF11000A00F0E9
:1085B000FF100843CDF80B004FEA3040CDF80B0018
:1085C000BDF81000010A41EA0020ADF810000023B8
:1085D0009DF914209DF913109DF91200F9F7EBFF96
:1085E000C9E00622611C0DF10A00FBF7C4FABDF8D0
:1085F0000A00010A41EA0020ADF80A00BDF80E00A9
:10860000010A41EA0020ADF80E00B4E00422611C2A
:108610000DF10A00FBF7AFFABDF80A00010A41EAC2
:108620000020ADF80A00BDF80C00010A41EA002064
:10863000ADF80C000FF2A420F9F7C3FD9BE009226E
:10864000611C0DF10A00FBF796FABDF80A00010A59
:1086500041EA0020ADF80A00BDF80C00010A41EA29
:108660000020ADF80C00BDF80E00010A41EA002020
:10867000ADF80E0000239DF912209DF911109DF90F
:108680001000F9F798FF76E060788DF80A00A0787E
:108690008DF80B00A27861780FF24C20F9F791FD6C
:1086A00069E00322611C0DF10A00FBF764FABDF8D2
:1086B0000B00010A41EA0020ADF80B005BE0052247
:1086C000611C0DF10A00FBF756FABDF80B00010A18
:1086D00041EA0020ADF80B004DE00922611C0DF1CC
:1086E0000A00FBF748FA46E00A22611C0DF10A0075
:1086F000FBF741FABDF90A00C0F3072141EA002067
:10870000ADF80A00BDF90C00C0F3072141EA0020D2
:10871000ADF80C00BDF90E00C0F3072141EA0020BE
:10872000ADF80E00BDF91000C0F3072141EA0020AA
:10873000ADF810001FE060788DF80A001BE00822F9
:10874000611C0DF10A00FBF716FABDF80C00010AD6
:1087500041EA0020ADF80C0000239DF911209DF99D
:1087600010109DF90F00F9F726FF04E08DF80800BE
:1087700060788DF809002078052807D15348012139
:108780000170687A00280ED1084655E418280AD1ED
:108790008DF8080060788DF80900A0788DF80A003F
:1087A000E0788DF80B0000208DF8280020780B90E1
:1087B0000DF1310002A91822FBF7A2F90B208DF868
:1087C00030000020ADF84A000AA800F097F9C0B2C6
:1087D00032E42078052804D13C48002101700120B2
:1087E0002AE41A281CD10822611C0DF10A00FBF7AB
:1087F000C2F9DDF80B00010221F0FF11000A00F0C0
:10880000FF100843CDF80B004FEA3040CDF80B00C5
:10881000BDF81000010A41EA0020ADF8100004E0A4
:108820002C2802D160788DF80A0001208DF82800EC
:1088300020780B900DF1310002A91822FBF760F9A6
:108840000B208DF830000AA800F058F9C0B2FFF7ED
:10885000F3BB0120FFF7F0BB2078002802D00528E9
:1088600005D006E00FF29000FDF7B0FC01E0FFF745
:1088700043F90120FFF7E0BB04F10802211D204667
:10888000FCF770FA0120FFF7D7BB0000CC240120D1
:108890002C9B002000600020AE660120B8D4002090
:1088A000004803080C480308184803082448030834
:1088B0003448030844480308504803085C48030848
:1088C000684803087C48030890480308AF66012005
:1088D00050443A2053432025640000004C54205358
:1088E000532041444400000041504452204144443C
:1088F000202564202564000041505F5245515545B4
:10890000535400007C4870472DE9F04182B00C467A
:108910001646012500282DD106EB8600764901EB8D
:10892000C007284600FA04F8F86810EA080F08D0D3
:108930002346FA6831460FF25030F9F742FC022024
:1089400046E04FF0FF30009003462A467968204603
:1089500006F0B2FA00280BD02346FA6831460FF22F
:108960003830F9F72EFCF86848EA0000F8602EE08D
:1089700002202DE001282AD106EB86005E4901EB9A
:10898000C007284600FA04F8F86810EA080F08D172
:108990002346FA6831460FF21030F9F712FC03252E
:1089A00015E04FF0FF332A467968204606F0EEFACC
:1089B000002807D02346FA6831460FF2FC20F9F769
:1089C00000FC00E00325F86820EA0800F86028466B
:1089D000BDE8F68107F04FBA02B58AB00021ADF8C4
:1089E000221001910A218DF8081000218DF809103C
:1089F0008DF80A1005218DF80010019004220AA9B3
:108A00000DF10900FBF7B7F80020ADF8220000A82F
:108A100000F074F80BB000BD80B508F087FA0FF2D3
:108A2000A820BDE80240F9F7CCBB38B5447885787A
:108A30000078032822D01A2802D02C282AD031BD51
:108A4000012C0CD1012009F065FE012322461A21D8
:108A50000FF2802001B0BDE83040F9F7B2BB022C24
:108A600021D1022009F056FE022322461A210FF2DC
:108A7000742001B0BDE83040F9F7A3BB012C12D13E
:108A8000284608F05EFA29460FF26C20BDE8344013
:108A9000F9F797BB012C06D129460FF26820BDE8F3
:108AA0003440F9F78EBB31BD0FB480B5002805D135
:108AB0000846002802D11046002804D00AF07BFBAB
:108AC000C046C04601E00AF05FFB01BC5DF814FB44
:108AD0000022C0B22D280CD240B200EB8003064821
:108AE00000EBC300C068012303FA01F1084200D083
:108AF0001A46104670470000C8F1002030B585B016
:108B00000446012594F90000062800F2A880DFE859
:108B100000F004284B667D9EA20004F1090182B09A
:108B200068461822FAF7ECFF0CBC94F9081060684C
:108B300040B206F0ABFD02280AD1606800B206F030
:108B4000B8FF002561680FF2C410F9F73AFB8CE01A
:108B5000032840F08A8061680FF2B810F9F731FB02
:108B600083E060681A280BD104F1090007F061FA6C
:108B7000237CE268E17A0FF2A410F9F722FB05E00A
:108B80002C2803D104F1090007F053FA94F90810D6
:108B9000606840B206F094FE032866D161680FF267
:108BA0009410F9F70EFB60E0618C00A806F09BFFC3
:108BB0009DF9040002280AD1009800B206F079FF5E
:108BC000002500990FF27410F9F7FBFA4DE0032825
:108BD0004BD100990FF26C10F9F7F3FA45E00AF067
:108BE000F7FB02280AD1606800B206F062FF002598
:108BF00061680FF25810F9F7E4FA36E0032834D12F
:108C000061680FF25010F9F7DCFA2EE06068052871
:108C10000CD128460AF0A3FC02280DD0032824D149
:108C200061680FF24010F9F7CCFA1EE002281CD15F
:108C30000AF099FD0228F1D1606800B206F039FF10
:108C4000002561680FF21410F9F7BBFA0DE0204619
:108C500006F0AFFF09E0204607F06EF905E0616815
:108C60000FF20810F9F7ADFA0025284605B030BD1F
:108C7000012070470FB4022004B0704701207047F4
:108C80000020704770470000534D41432025642069
:108C90002564202564000000534D412025642025D3
:108CA0006420256400000000534D524320256420B9
:108CB0002564202564000000534D522025642025A2
:108CC0006420256400000000504420536574535410
:108CD0000000000041542052492D256420256420C5
:108CE00025640000415420524920426174202D2502
:108CF000642025642025640050442055542D2564AB
:108D000000000000534C4D2025640000414C4F46AC
:108D100020256400414C4346202564004F4A4820EA
:108D2000454C2030782578203078257820307825FB
:108D300078000000524C434620256400504C4F46BA
:108D400020256400504C43462025640050414F4686
:108D500020256400504143462025640050504F4672
:108D60002025640050504346202564004558204C7F
:108D70004D454C2025640000010040F10980F44677
:108D8000404200F005F851F000416047010000BF8B
:108D900009D0B0FA80F18840C91CC1F58461090589
:108DA00001EBD02140057047B0B581EA030C0CF00F
:108DB000004C40F2FF7515EA11541DBF15EA135718
:108DC000AC42AF4239E0E41923EA455343F480133F
:108DD000C90241F0004141EA505EC7021100A7FB01
:108DE000020200284FF00000EEFB01204FF00001CE
:108DF000E3FB072118BF42F001024018002149415E
:108E0000E3FB0E01A4F580640F0302D2520040413F
:108E1000494154F101046CDD470872F1004250F100
:108E2000000051EB0451A1F580115CBF41EA0C0137
:108E3000B0BD4CEA05510020B0BD05EA1357AC4265
:108E400014BFAF4241E050EA410E1CBF52EA430E4C
:108E500002E061460020B0BD24423C441BD15FEAE1
:108E6000070EF6D0090302BF01460020AEF1140E32
:108E7000B1FA81F7AEEB070401FA07FE0C37C7F130
:108E8000200100FA07F7C8404EEA000E23EA4553D6
:108E900043F48013A2E733F00043B3FA83F704BF2F
:108EA000B2FA82FE77440B3FE41BB7F1200E2FBFCE
:108EB00002FA0EF3BB40C7F1200E22FA0EFE38BFB5
:108EC00043EA0E03BA40641C82E750EA410E14BF25
:108ED00052EA430E6FF000014FF4001717EB430FF7
:108EE0008ABF194617EB410FB5E74CEA0551002040
:108EF000B0BDD4F10104B4F120070FDAC4F12007AA
:108F0000520828BF42F0010210FA07F501FA07F7EC
:108F1000E1BF2A43E0403843E1400FE0352C98DCC4
:108F2000C7F1200452EA400220FA07F218BF42F0CB
:108F3000010231FA07F0A1400A43002172F1004218
:108F400050F1000051EB0C01B0BD00005FF0FF0CD0
:108F50001CEAD05114BF614506E0C110400721F062
:108F6000E04101F16051704779B900F00041000221
:108F70000AD0B0FA80FC00FA0CF001F16051A1EBCC
:108F80000C5101EBD0214005704741020CBF40F469
:108F9000E0016FF000010020704700004FEAF17C13
:108FA000BCF1E04C2CBFBCF5001F11E05FEA4C0C9B
:108FB00034BFBCF17F5F2EE05FEA9C0C4FEA0C1CD3
:108FC0004FEA3C0CC10071F100414CEB507070470E
:108FD000C90241EA5051C00218BF41F0010141F0FD
:108FE00000414FEA6C50C0F10900212810D240EA3C
:108FF000CC7CCCF1200C11FA0CF070F10040CCF1DB
:10900000200C21FA0CF00CF0004C40EB0C007047E7
:109010004FEACC707047490011F5001F04D84FEAA1
:10902000CC10FF30C0057047C817704762F30F229D
:1090300062F31F42401810F0030308D0C91A1FD36F
:10904000DB0748BF00F8012D28BF20F8022D1300D0
:1090500030B414461546103928BF20E93C00FAD830
:10906000490728BF20E90C0048BF40F8042D8900BB
:1090700028BF20F8022D48BF00F8012D30BC7047F2
:10908000C91818BF00F8012DCB0728BF00F8012D23
:1090900070470000DFF8B01100220A700A70012842
:1090A00002D0042803D070470120087070470520C3
:1090B0000870704765490860704710B464494A6891
:1090C00002F00C02644B082A12D10A680C6804F002
:1090D0003F04B3FBF4F30A68C2F388125A430B68E7
:1090E000C3F301435B1C5B00B2FBF3F2026000E0E0
:1090F00003604A6802F0F003584A1B099B5C04684D
:1091000024FA03F343604C6804F4E054A40AA45C1A
:10911000E3408360496801F46041490B895C42681F
:1091200022FA01F1C16010BC70474A4900F4407254
:10913000B2F5407F06D10A6822F4F812484B03408A
:109140001A430A608A6E000552EA1050886670471A
:10915000444908607047444908607047434A002901
:10916000116802D008431060704721EA00001060C7
:1091700070473F4A0029116802D0084310607047C9
:1091800021EA0000106070473A4A0029116802D0B5
:1091900008431060704721EA000010607047364AAB
:1091A0000029116802D008431060704721EA0000CE
:1091B00010607047314A0029116802D008431060DE
:1091C000704721EA0000106070472D4A002911689D
:1091D00002D008431060704721EA00001060704719
:1091E000284A0029117802D008431070704721EAFC
:1091F00000001070704700214209124B012A01D172
:109200001A6804E0022A01D11A6F00E05A6F0123A4
:1092100000F01F0003FA00F0024200D01946084691
:1092200070471948016841F0807101607047002162
:10923000164A1268024200D00121084670471449BC
:10924000087070470038024070380240800E474274
:1092500004380240083802400024F400E09A00205C
:10926000FFFCFF0F3C0E4742400E474230380240A1
:109270004038024044380240103802402038024052
:10928000243802400D380240743802400C38024045
:109290000E38024080B52749884209D1012108468D
:1092A000FFF77DFF00210120BDE80440FFF777BFF5
:1092B0002149884209D101210220FFF770FF0021D6
:1092C0000220BDE80440FFF76ABF1C49884209D16B
:1092D00001210420FFF763FF00210420BDE80440C2
:1092E000FFF75DBF1649884209D101210820FFF729
:1092F00056FF00210820BDE80440FFF750BF114988
:10930000884209D101211020FFF749FF00211020D8
:10931000BDE80440FFF743BF0B49884209D1012152
:109320008020FFF73CFF00218020BDE80440FFF7CC
:1093300036BF01BD000002400004024000080240A8
:10934000000C024000100240001C0240F0B4002259
:1093500032E0012393400C681C409C422BD1540006
:109360000325A540ED4306682E40066006680F7988
:10937000A7403E4306600E79012E01D0022E11D186
:1093800086682E40866086684F79A7403E43866097
:10939000466826EA0303436043688E799640B6B276
:1093A00033434360C3682B40C360C368CD7905FA7B
:1093B00004F42343C360521C102ACAD3F0BC704784
:1093C0004FF6FF7101600021017141718171C1711E
:1093D000704700220069084200D001221046704701
:1093E000018370474183704710B4CB1000EB8300BA
:1093F00001F007018900036A0F248C40A343036234
:10940000036A02FA01F11943016210BC70470000BF
:1094100080B5434988420BD101214FF40010FFF77A
:10942000C9FE00214FF40010BDE80440FFF7C2BEA2
:109430003C4988420BD101214FF48000FFF7BAFE6E
:1094400000214FF48000BDE80440FFF7B3BE364969
:1094500088420BD101214FF40000FFF7ABFE002141
:109460004FF40000BDE80440FFF7A4BE01BD7FB586
:1094700004460D46A68800A8FFF71FFE02992B4858
:10948000B1FBF0F04FF6C07232400243A280228856
:109490004FF6FE731A4022802A68254B9A420AD260
:1094A0005200B1FBF2F10A4692B2042A00D2042122
:1094B000401C208421E0EB884BF6FF76B34204D1B8
:1094C00002EB4202B1FBF2F106E019235A43B1FB71
:1094D000F2F141F4804189B20A0502D141F0010163
:1094E00089B241F4004180B24FF4967250434FF478
:1094F0007A7290FBF2F0401C2084A183208840F017
:109500000100208020884FF6F5310840A9880843E3
:10951000698908432080A8892989084320817FBD63
:109520000054004000580040005C004040420F00E2
:10953000A18601000029018803D041F001010180CA
:1095400070474FF6FE721140018070470029018874
:1095500003D041F48071018070474FF6FF621140E3
:10956000018070470029018803D041F40071018017
:1095700070474FF6FF52114001807047002A02D019
:1095800041F0010101E001F0FE0101827047002974
:10959000018803D041F48061018070474FF6FF32AB
:1095A0001140018070470029018803D041F4004137
:1095B000018070474904490C0180704782B002461F
:1095C000002003460193009300920A0F01920902C2
:1095D000090A019A002A03D0009A1432009203E08B
:1095E000090C009A18320092009A12680A4200D0C0
:1095F000012002B07047000080B5254988420BD198
:1096000001214FF48050FFF7E0FD00214FF480501E
:10961000BDE80440FFF7D9BD1E4988420BD10121A6
:109620004FF48040FFF7C6FD00214FF48040BDE8B5
:109630000440FFF7BFBD184988420BD101214FF408
:109640000040FFF7B7FD00214FF40040BDE80440A3
:10965000FFF7B0BD01BD028802F441520B881A43E6
:109660004B881A438B881A43CB881A430B891A43B9
:109670004B891A438B891A43CB891A430280828B08
:109680004FF2FF731A408283098A018270470000FB
:109690000030014000380040003C004000290188B3
:1096A00003D041F04001018070474FF6BF72114076
:1096B00001807047002A828802D011438180704760
:1096C00022EA01018180704700220089084200D00F
:1096D00001221046704700000168490849000160F6
:1096E0000021016041608160C1600161212141610F
:1096F0006A49884203D16A483D210160704769493F
:10970000884204D166484FF474610160704766492D
:10971000884204D162484FF4741101607047634974
:10972000884204D15E484FF074610160704760491F
:10973000884203D15A485F49416070475E49884278
:1097400003D157485D49416070475D49884203D164
:1097500053485C49416070475B49884204D1504896
:109760004FF03D51416070475849884203D15848F5
:109770003D21016070475749884204D154484FF455
:109780007461016070475449884204D150484FF4D5
:109790007411016070475149884204D14C484FF020
:1097A0007461016070474E49884203D1484841497D
:1097B000416070474B49884203D145483F49416069
:1097C00070474949884203D141483E49416070474A
:1097D0004649884203D13E484FF03D5141607047B1
:1097E0000268434B1A400B681A43CB681A434B6913
:1097F0001A438B691A43CB691A430B6A1A434B6AA3
:109800001A438B6A1A434B6B1A438B6B1A430260E1
:109810004269D208CB6A53EAC2020B6B1A43426117
:109820000A6942604A6882608968C160704700299D
:10983000016803D041F00101016070474908490007
:1098400001607047002A01D001617047C160704714
:10985000006800F00100704700221C4B984201D2C2
:10986000244800E024488B0001D5406800E00068EF
:1098700008402249084200D0012210467047134A8E
:10988000904201D21B4800E01B481C4A0A40890054
:1098900001D5C260704782607047000010600240CE
:1098A0000860024028600240406002405860024068
:1098B000706002403D00002088600240400F0020A0
:1098C000A060024000003D20B860024010640240E9
:1098D0000864024028640240406402405864024028
:1098E0007064024088640240A0640240B864024090
:1098F0003F801CF000600240006402407D0F7D0F3D
:1099000002490860704702490860704720000E4213
:1099100024000E4270B504460026DFF83854CA20F1
:10992000E8615320E86100F018F8002811D0286899
:1099300020F0400028602868216808432860A0685B
:10994000A860A868616840EA0140A86000F024F8B7
:109950000126FF20E861304670BD81B000200090F4
:10996000DFF8F4030168490613D44FF0FF310160BA
:10997000016801F04001009A521C0092009AB2F571
:10998000803F01D00029F3D00068800900F0010079
:1099900000E0012001B07047DFF8BC03016821F04E
:1099A00080010160704781B000200090DFF8A813AB
:1099B000CA20886153208861086820F0A0000860F0
:1099C000086800F02000009A521C0092009AB2F53C
:1099D000003F01D00028F3D00868400900F00100E2
:1099E000FF228A6101B07047F8B507460E46002491
:1099F000DFF85C53002FA86804D140060AD4204643
:109A0000F07007E0400603D5307800F0BEF901E0C1
:109A10002046F0703078002F09D07178090241EAB1
:109A20000040B1780843F17840EA01460FE000F0C9
:109A3000A1F90746707800F09DF9000240EA074757
:109A4000B07800F097F93843F17840EA0146CA202F
:109A5000686253206862FFF780FF00280FD0DFF8AC
:109A6000FC0230402860FFF797FFA868800605D405
:109A7000FFF799FF002802D0012400E00124FF2015
:109A800068622046F2BD10B50C46DFF8C4120968C2
:109A9000DFF8C82211400A0C02F03F0323700B0AC2
:109AA00003F07F03637001F07F01A17002F04001B9
:109AB000E17000280BD1207800F067F92070607801
:109AC00000F063F96070A07800F05FF9A07010BD3D
:109AD000DFF88C12486A0968704770B506460D4673
:109AE0000024002E06D16878C10603D500F0EF00EF
:109AF0000A306870002E05D0687800F046F9A87822
:109B000000F043F9E878002E09D06978090241EAAB
:109B10000040A9780843297840EA41360FE000F078
:109B200029F90646687800F025F9000240EA064661
:109B3000A87800F01FF93043297840EA4136DFF871
:109B40002052CA20286253202862FFF706FF00280F
:109B50000FD0DFF8100230402860FFF71DFF686863
:109B6000800605D4FFF71FFF002802D0012400E083
:109B70000124FF202862204670BD10B50C46DFF896
:109B8000E0110968DFF8DC2111400A0CE2700A0AD2
:109B900002F01F02627001F03F02A270490B01F057
:109BA0000701217000280BD1E07800F0EEF8E0709A
:109BB000607800F0EAF86070A07800F0E6F8A07035
:109BC00010BDDFF89011CA22CA615322CA610A6827
:109BD000D208D2000A600A6810430860FF20C861FA
:109BE0007047DFF88411CA220A6153220A610860B3
:109BF000FF200861704781B000210091DFF8541107
:109C0000CA22CA615322CA610028086804D040F4FD
:109C100080600860012012E020F4806008604868DD
:109C200000F00400009A521C0092009AB2F5803FA6
:109C300001D00028F3D04868800800F00100FF221E
:109C4000CA6101B0704781B000220092474A009279
:109C5000009A02EB800000900098016001B070470C
:109C600081B00021009141490091009901EB8000F1
:109C700000900098006801B0704738B50024224673
:109C8000344DCA23EB615323EB616B681B0701D48E
:109C900006E0521C6B681B0702D5B2F5805FF8D155
:109CA0006A68120709D42A68D20606D40843686293
:109CB000FFF779FE002800D00124FF20E86120464C
:109CC00032BD244ACA23D3615323D36100F0040375
:109CD00020F004000029116805D008431060906B43
:109CE0001843906305E021EA00001060906B9843F0
:109CF0009063FF20D06170470021174A12681C4B07
:109D00001A40024200D001210846704710B40021D9
:109D1000104A936B03F004031468044003EAD03341
:109D20002343526802EA101002D0000400D001213F
:109D3000084610BC704708490003000C40F0800042
:109D40000A6802F0800262EA0000086070470000C2
:109D500000280040082800400C2800407F7F7F003A
:109D6000042800403FFFFF00142800405028004016
:109D70007F3F0100002101E0491C0A38C0B20A28D7
:109D8000FAD240EA0110C0B27047010901EB81022A
:109D900000F00F0000EB4200C0B2704730B4016821
:109DA000CB4321498279002A27D00A4614682340F0
:109DB000136053680468A34353600379CC18236885
:109DC00005682B43236093680468A3439360D368BA
:109DD0000468A343D36043790568102B07D19168C9
:109DE00029439160D16800680843D0600AE051FAC5
:109DF00083F420682843206004E000790C18206870
:109E00001840206030BC70470021074A13680340A7
:109E10005269024202D0002B00D00121084670474F
:109E20000249086070470000003C0140143C0140BA
:109E30001949084319490860704770B403781A46F5
:109E40000121C478002C1DD0144B1B6803F4E0637F
:109E5000C3F5E0631B0A4478C3F10405AC40857880
:109E60000F2646FA03F32B4023431B010C4C1355DA
:109E7000007842110B4B00F01F0001FA00F043F88C
:109E8000220006E05011084A03F01F03994042F8EF
:109E9000201070BC704700000000FA050CED00E0D7
:109EA00000E400E000E100E080E100E030B401F017
:109EB0000302920021F00301054BCC580F25954079
:109EC000AC43CC50CC5890402043C85030BC704775
:109ED0000838014080B501214FF48070FFF775F913
:109EE00000214FF48070BDE80440FFF76EB942686E
:109EF0004D4B1A400B7942EA03220B681A43426029
:109F000082684A4B1A400B691A43CB681A438B6824
:109F10001A434B7942EA43028260C26A22F4700219
:109F2000097D491EC9B242EA0151C1627047002150
:109F30000160017141718160C160016101210175A0
:109F400070473B490A683B4B1A4003681A43436811
:109F50001A4383681A43C0681043086070470021A1
:109F6000016041608160C16070470029816803D051
:109F700041F00101816070474908490081607047E4
:109F800070B407240A290BD3C568A1F10A0606EBB1
:109F90004606B44025EA0404B3402343C36008E006
:109FA000056901EB4106B44025EA0404B3402343AC
:109FB00003611F23072A0AD2446B521E02EB82025E
:109FC000934024EA030391401943416316E00D2AAC
:109FD0000AD2046BD21F02EB8202934024EA0303ED
:109FE00091401943016309E0C46A0D3A02EB820211
:109FF000934024EA030391401943C16270BC704747
:10A00000816841F08041816070470029816803D0F8
:10A0100041F480618160704721F480618160704704
:10A02000C06C80B270470000FFFEFFFCFDF7FFC070
:10A0300004230140E030FCFF00220068084200D009
:10A04000012210467047000013F0004C03D55B421C
:10A05000524263F100039CEA210C00F0178010B516
:10A06000644603D34942404261F1000100F00EF81A
:10A07000640004D34942404261F10001244203D507
:10A080005B42524263F1000310BD00001B4213D13A
:10A09000094236D12AB18446B0FBF2F002FB10C26D
:10A0A000704709F0C1BBFCD30022002370470B00AE
:10A0B0000200002100207047904271EB030CF6D3A0
:10A0C00070B5B1FA81F4B3FA83F52C1BA340C4F147
:10A0D000200532FA05F63343A2405FF00046E64021
:10A0E00002E05B085FEA3202841A71EB030524BFC9
:10A0F000204629467641F4D302000B0030000021AF
:10A1000070BD012ACFD970B5140C20D0B1FA81F4FA
:10A11000B2FA82F5C4F120046419B4F12006D6D352
:10A12000B2405FF00044F440002502E052085FEACC
:10A130003303C61A71EB020E24BF304671466441E8
:10A140006D41F3D302000B002000290070BD0C46C6
:10A15000B1FBF2F102FB11452D0445EA1045B5FBB8
:10A16000F2F402FB145580B240EA0545B5FBF2F06B
:10A1700002FB105240EA044070BD000010B504001C
:10A1800010480078002805D10F4809F074FB0D48ED
:10A19000012101700C4809F0A4FB20000AF020FA0C
:10A1A0000400094809F0D1FB200010BD10B50400DF
:10A1B000054809F096FB20000AF05EFB024809F012
:10A1C000C4FB10BDB866012058630120BFF34F8F58
:10A1D000DFF8B40C006810F4E060DFF8B01C08434E
:10A1E000DFF8A41C0860BFF34F8FFEE700B583B013
:10A1F0000020ADF8040000208DF8060000208DF846
:10A200000700012000900DF106037622D0210020E6
:10A21000F8F7A7F8002801D1002044E076208DF857
:10A2200004009DF8060050F020008DF80500022380
:10A2300001AAD0210020F8F73AF8002801D1002027
:10A2400031E0012000900DF107034922D0210020C8
:10A25000F8F787F8002801D1002024E049208DF884
:10A2600004009DF8070050F001008DF8050002235E
:10A2700001AAD0210020F8F71AF8002801D1002007
:10A2800011E076208DF804009DF806008DF8050099
:10A29000022301AAD0210020F8F709F8002801D1F3
:10A2A000002000E001200EBD38B50400F7F707FFDD
:10A2B0000500DFF8040D0078401CDFF8FC1C087076
:10A2C000DFF8F40C4078F021084202D09920FBF727
:10A2D000DFFBFBF74AFCDFF8E00C4078401CDFF8BE
:10A2E000D81C4870210089B22800F8F7D5F8DFF8AB
:10A2F000C80C4078F021084202D09920FBF7C8FB37
:10A30000DFF8B40C4078401EDFF8AC1C4870C0B2D7
:10A31000002801D1FBF723FCFCF77DFA31BD10B515
:10A3200082B00020ADF80000F7F7C9FE04006B20F2
:10A330008DF8000080208DF80100022300AAD021B2
:10A340000020F7F7B4FF002801D1002094E0642139
:10A350002000F8F7A1F8FFF749FF002801D10020FD
:10A360008AE06B208DF8000000208DF801000223A8
:10A3700000AAD0210020F7F79AFF002801D1002081
:10A380007AE028212000F8F787F819208DF80000DE
:10A3900004208DF80100022300AAD0210020F7F745
:10A3A00086FF002801D1002066E01A208DF8000009
:10A3B00003208DF80100022300AAD0210020F7F726
:10A3C00076FF002801D1002056E01B208DF8000008
:10A3D00008208DF80100022300AAD0210020F7F701
:10A3E00066FF002801D1002046E01D208DF8000006
:10A3F00003208DF80100022300AAD0210020F7F7E6
:10A4000056FF002801D1002036E06A208DF80000B8
:10A4100000208DF80100022300AAD0210020F7F7C8
:10A4200046FF002801D1002026E06C208DF80000B6
:10A430003F208DF801009DF80110DFF8500DF7F76F
:10A44000C0FE022300AAD0210020F7F730FF002829
:10A4500001D1002010E06B208DF8000040208DF825
:10A460000100022300AAD0210020F7F720FF0028D6
:10A4700001D1002000E0012016BD0178407850EAAB
:10A48000012000B2704780B502200090DFF8003D47
:10A490006B22D0210020F7F764FF002801D10020B3
:10A4A0005BE001200090DFF8EC3C1A22D021002074
:10A4B000F7F757FF002801D100204EE0012000905F
:10A4C000DFF8D43C1B22D0210020F7F74AFF0028F8
:10A4D00001D1002041E001200090DFF8C03C1C22A7
:10A4E000D0210020F7F73DFF002801D1002034E003
:10A4F00001200090DFF8A83C1D22D0210020F7F7B2
:10A5000030FF002801D1002027E001200090DFF873
:10A51000943C6A22D0210020F7F723FF002801D1C4
:10A5200000201AE001200090DFF87C3C3822D02186
:10A530000020F7F716FF002801D100200DE00120D0
:10A540000090DFF8683C1922D0210020F7F709FFBE
:10A55000002801D1002000E0012002BD80B50020CC
:10A56000ADF800001A208DF80000DFF8240C007907
:10A570008DF80100022300AAD0210020F7F797FEF2
:10A58000002801D1002090E01B208DF80000DFF8AA
:10A59000000C40798DF80100022300AAD021002090
:10A5A000F7F785FE002801D100207EE01C208DF801
:10A5B0000000DFF8DC0B80798DF80100022300AA8F
:10A5C000D0210020F7F773FE002801D100206CE0B5
:10A5D0001D208DF80000DFF8B80BC0798DF8010060
:10A5E000022300AAD0210020F7F761FE002801D144
:10A5F00000205AE06A208DF80000DFF8940BC07844
:10A600008DF80100022300AAD0210020F7F74FFEA9
:10A61000002801D1002048E019208DF80000DFF863
:10A62000700B80788DF80100022300AAD021002051
:10A63000F7F73DFE002801D1002036E038208DF8E4
:10A640000000DFF84C0B007A8DF80100022300AA0D
:10A65000D0210020F7F72BFE002801D1002024E0B4
:10A660006B208DF80000DFF8280B00788DF80100D2
:10A67000022300AAD0210020F7F719FE002801D1FB
:10A68000002012E06C208DF80000DFF8040B407809
:10A690008DF80100022300AAD0210020F7F707FE61
:10A6A000002801D1002000E0012002BD10B582B0D9
:10A6B0000020ADF80000DFF8D80A0078400612D577
:10A6C0006B208DF8000000208DF80100022300AA05
:10A6D000D0210020F7F7EBFD002801D10020C9E0D0
:10A6E0003220FFF7E1FD6C208DF80000DFF8A00AB2
:10A6F000407810F0F8008DF80100022300AAD02164
:10A700000020F7F7D4FD002801D10020B2E06A2034
:10A710008DF8000000208DF80100022300AAD0214E
:10A720000020F7F7C4FD002801D10020A2E000249A
:10A7300000E0641C062C10DA14F113008DF8000000
:10A7400000208DF80100022300AAD0210020F7F795
:10A75000AEFD0028EDD100208CE019208DF800001E
:10A7600000208DF80100022300AAD0210020F7F775
:10A770009EFD002801D100207CE01A208DF8000009
:10A7800003208DF801004FF4FA642000FA281DD050
:10A79000B0F5FA7F13D0B0F57A7F09D0B0F5FA6F33
:10A7A00019D19DF8010050F018008DF8010016E055
:10A7B0009DF8010050F010008DF801000FE09DF8A9
:10A7C000010050F008008DF8010008E09DF801003C
:10A7D0008DF8010003E09DF801008DF801000223CF
:10A7E00000AAD0210020F7F762FD002801D1002047
:10A7F00040E0FA2C14D0B4F5FA7F0DD0B4F57A7F8E
:10A8000006D0B4F5FA6F0FD103208DF801000EE0E9
:10A8100002208DF801000AE001208DF8010006E019
:10A8200000208DF8010002E000208DF801001B20BF
:10A830008DF800009DF80100C0008DF80100022392
:10A8400000AAD0210020F7F732FD002801D1002016
:10A8500010E038208DF8000000208DF80100022360
:10A8600000AAD0210020F7F722FD002801D1002006
:10A8700000E0012016BD00B583B00020ADF8060051
:10A8800000208DF804006B208DF8060001208DF863
:10A89000070002230DF10602D0210120F7F707FD82
:10A8A000002801D1002023E02820FFF7FDFC012033
:10A8B000009001AB6C22D0210120F7F752FD002857
:10A8C00001D1002014E06C208DF806009DF80400F2
:10A8D00010F0C0008DF8070002230DF10602D02110
:10A8E0000120F7F7E4FC002801D1002000E001205E
:10A8F0000EBD2DE9F04F85B004000D0016001F00BD
:10A900000020ADF8040002A80021002206C008388B
:10A9100006208DF8060038208DF8040000208DF800
:10A920000500022301AAD0210120F7F7C0FC00286E
:10A9300002D15FF0FF3070E123208DF80400002089
:10A940008DF80500022301AAD0210120F7F7AFFC02
:10A95000002802D15FF0FF305FE16A208DF804002B
:10A9600000208DF80500022301AAD0210120F7F76D
:10A970009EFC002802D15FF0FF304EE16A208DF886
:10A98000040004208DF80500022301AAD021012033
:10A99000F7F78DFC002802D15FF0FF303DE11A206F
:10A9A0008DF8040001208DF80500022301AAD021B2
:10A9B0000120F7F77CFC002802D15FF0FF302CE18A
:10A9C00019208DF8040000208DF80500022301AA4B
:10A9D000D0210120F7F76BFC002802D15FF0FF3097
:10A9E0001BE11B208DF804008DF80540022301AA0D
:10A9F000D0210120F7F75BFC002802D15FF0FF3087
:10AA00000BE1FFB2002F0FD01C208DF804008DF851
:10AA10000540022301AAD0210120F7F748FC0028B5
:10AA200002D15FF0FF30F8E064B2002C02D0C82001
:10AA3000FFF73AFC6A208DF8040044208DF80500E9
:10AA4000022301AAD0210120F7F731FC002802D10E
:10AA50005FF0FF30E1E023208DF80400FFB2002F0B
:10AA600003D008208DF8050002E070208DF8050065
:10AA7000022301AAD0210120F7F719FC002802D1F6
:10AA80005FF0FF30C9E00A20FFF70EFC002408E069
:10AA9000E4B2002045F82400E4B2002046F8240087
:10AAA000641CE4B2032CF3D35FF00009B9F1320F58
:10AAB0006EDA0A20FFF7F8FB0220009002AB722248
:10AAC000D0210120F7F74DFC002802D15FF0FF30C4
:10AAD000A3E002A8FFF7D1FC9DF8061090FBF1F867
:10AAE000B8F1070F02DA7FF0010096E000241AE0C7
:10AAF0005FFA8AFA55F82AB05FFA8AFA02A810EBD0
:10AB00004A00FFF7BAFC0BFA80F05FFA8AFA45F8C0
:10AB10002A001AF1010A5FFA8AFABAF1030FE7D3A1
:10AB200019F10109641CE4B24445BFDAB9F1320FEE
:10AB3000BCDA9DF80600009002AB7422D0210120FF
:10AB4000F7F70FFC002802D15FF0FF3065E0FFB29D
:10AB5000002F1AD05FF0000A5FFA8AFABAF1030FE9
:10AB6000DED25FFA8AFA56F82AB05FFA8AFA02A8A9
:10AB700010EB4A00FFF781FC0BFA80F05FFA8AFACB
:10AB800046F82A001AF1010AE6E75FF0000AC2E778
:10AB900023208DF8040000208DF80500022301AA6F
:10ABA000D0210120F7F783FB002802D15FF0FF30AE
:10ABB00033E05FF0000A0FE05FFA8AFA55F82A00E6
:10ABC0004FF47A714843322190FBF1F05FFA8AFA30
:10ABD00045F82A001AF1010A5FFA8AFABAF1030F5E
:10ABE000EAD3FFB2002F17D05FF0000A0FE05FFA40
:10ABF0008AFA56F82A004FF47A714843322190FBC2
:10AC0000F1F05FFA8AFA46F82A001AF1010A5FFAAF
:10AC10008AFABAF1030FEAD3012005B0BDE8F08F3C
:10AC20002DE9F04389B004000D00160000275FF005
:10AC3000010801A8002101605FF0000903200090D5
:10AC400001AB0D22D0210120F7F78BFB002801D1A9
:10AC50005FF0FF385FF0000905E005A8002140F82B
:10AC6000291019F10109B9F1030F11DA01A819F836
:10AC700000000028F1D001A819F80000DFF8C81A78
:10AC800011EB400030F8020C05A941F82900E8E773
:10AC90005FF000091FE002A850F82900DFF8AC1AA5
:10ACA000884207DADFF8A80AF7F78BFA012010FAD2
:10ACB00009F0074302A850F82900DFF8981A8842E3
:10ACC00007DBDFF8940AF7F77CFA012010FA09F0A5
:10ACD000074319F10109B9F1030F2BDA55F82900DF
:10ACE00056F82910401A0AF03FF802A941F8290045
:10ACF00005A850F829000028CDD002A850F8290056
:10AD000005A951F8291090FBF1F0B0F57A700AF01E
:10AD10002BF824F8190034F9190040F2F511884293
:10AD2000D7DBDFF8380AF7F74CFA012010FA09F000
:10AD30000743CEE7B4F904000090B4F90230B4F947
:10AD400000203900DFF8180AF7F73BFA002F05D08A
:10AD5000DFF8100AF7F735FA7FF00208404640B2F4
:10AD600009B0BDE8F08338B505000020ADF800005B
:10AD70000020ADF80200F7F7A2F9040038208DF8A2
:10AD8000000000208DF80100022300AAD02100203D
:10AD9000F7F78DFA002801D1002074E000F029FBBC
:10ADA000002801D100206EE01F208DF800004B200C
:10ADB0008DF80100022300AAD0210020F7F777FACE
:10ADC000002801D100205EE01E208DF80000062042
:10ADD0008DF80100022300AAD0210020F7F767FABE
:10ADE000002801D100204EE069208DF80000C0202D
:10ADF0008DF80100022300AAD0210020F7F757FAAE
:10AE0000002801D100203EE0012201210320F7F7B4
:10AE1000CAFB0020F7F7C9FB38208DF8000040205E
:10AE20008DF80100022300AAD0210020F7F73FFA95
:10AE3000002801D1002026E0012028702000407D5C
:10AE4000C046012810D001212000F7F725FBBDF8EE
:10AE50000200401CADF80200BDF802003228EDD31C
:10AE6000DFF80409F7F7ADF9012200210320F7F715
:10AE70009AFB0020F7F799FB00F0B1FB002801D105
:10AE8000002000E0012032BD0CED00E00400FA05D6
:10AE900070B58EB0040000A80021002206C008385A
:10AEA000012500260BA80021002200230EC00C382B
:10AEB00008A80021002200230EC00C3805A800219C
:10AEC000002200230EC00C3802A80021002200231B
:10AED0000EC00C38FFF7D7FA002801D1002056E049
:10AEE000FFF7E4FB002806D00126FFF7C4FC00288A
:10AEF00003D100204BE0002049E0012302AA08A969
:10AF00000020FFF7F6FC05006DB2012D04D0DFF83C
:10AF10005408F7F756F91CE0012305AA0BA97FF0A6
:10AF20001F00FFF7E6FC05006DB2012D04D0DFF82D
:10AF30002C08F7F746F90CE005AA02A900A8FFF7CC
:10AF40006FFE05006DB2012D03D0DFF80408F7F79E
:10AF500038F92670BDF800006070BDF900000012DD
:10AF6000A070BDF80200E070BDF90200001220716F
:10AF7000BDF804006071BDF904000012A071E57114
:10AF8000FFF7ECFA002801D1002000E001200EB00C
:10AF900070BD80B5DFF8D4070078002809D1FFF72D
:10AFA000BEF9002801D1002004E0DFF8C00701212C
:10AFB0000170012002BD0000F89900201CB500209E
:10AFC0008DF806000020ADF80400F7F778F80400CB
:10AFD000012000900DF106036B22D0210020F7F72D
:10AFE000C0F9002801D1002088E09DF8060060210A
:10AFF000084216D06B208DF804009DF8060010F072
:10B000009F008DF80500022301AAD0210020F7F748
:10B010004EF9002801D1002070E014212000F7F73C
:10B020003BFA012000900DF106036C22D021002094
:10B03000F7F797F9002801D100205FE06C208DF828
:10B0400004009DF8060010F0C7008DF805000223EB
:10B0500001AAD0210020F7F72AF9002801D1002009
:10B060004CE00A212000F7F717FA1D208DF80400A4
:10B0700043208DF80500022301AAD0210020F7F714
:10B0800016F9002801D1002038E01C208DF80400BA
:10B0900000208DF80500022301AAD0210020F7F737
:10B0A00006F9002801D1002028E020208DF80400B6
:10B0B00080208DF80500022301AAD0210020F7F797
:10B0C000F6F8002801D1002018E01F208DF80400B8
:10B0D00080208DF80500022301AAD0210020F7F777
:10B0E000E6F8002801D1002008E0DFF884060078A7
:10B0F00050F00100DFF878160870012016BD00B589
:10B1000083B000208DF806000020ADF80400012077
:10B1100000900DF106036C22D0210020F7F721F9F1
:10B12000002801D1002030E06C208DF804009DF84B
:10B13000060050F038008DF80500022301AAD02146
:10B140000020F7F7B4F8002801D100201DE0DFF857
:10B150002006007880070FD46B208DF80400402073
:10B160008DF80500022301AAD0210020F7F79FF8EF
:10B17000002801D1002008E0DFF8F405007810F085
:10B18000FE00DFF8EC15087001200EBD104A030820
:10B19000406401204464012045640120466401208C
:10B1A0004764012043640120486401204264012077
:10B1B00000B583B000208DF804000020ADF8060033
:10B1C0000120009001AB6C22D0210020F7F7C9F8D4
:10B1D000002801D1002014E06C208DF806009DF8B5
:10B1E000040050F038008DF8070002230DF106022C
:10B1F000D0210020F7F75BF8002801D1002000E003
:10B2000001200EBD2DE9F04186B004000D0004A818
:10B210000021002206C008380020ADF80C000126ED
:10B22000DFF850050768F6F74AFF8046DFF8480563
:10B230000068401CDFF8401508600120009004AB56
:10B240006B22D0210020F7F78CF8002801D10020D4
:10B25000CCE09DF8100040061AD56B208DF80C004C
:10B260009DF8100010F0BF008DF80D00022303AA16
:10B27000D0210020F7F71BF8002801D10020B5E00D
:10B2800014214046F7F708F9DFF8F004F6F799FFC4
:10B290000120009004AB6C22D0210020F7F761F868
:10B2A000002801D10020A1E09DF8100038210842BB
:10B2B0001ED06C208DF80C009DF8100010F0C70017
:10B2C0008DF80D00022303AAD0210020F6F7EFFF2E
:10B2D000002801D1002089E005214046F7F7DCF87D
:10B2E000DFF89C04F6F76DFFDFF898040121016098
:10B2F000EDB2009504AB3B22D0210020F7F731F8E6
:10B30000002805D1DFF88004F6F75BFF00206DE030
:10B310009DF8110020709DF8100060709DF81300DA
:10B32000A0709DF81200E0709DF8150020719DF846
:10B3300014006071002000E0401C062806D2015D68
:10B34000DFF84824825C9142F6D00026F6B2012E46
:10B3500018D1DFF83C040068401CDFF834140860A2
:10B36000DFF82C040068132804D1DFF82804F6F76E
:10B3700028FF0BE0DFF818040068142806D1FEF758
:10B3800025FF03E0DFF80804002101600622210008
:10B39000DFF8F803F8F7EFFBDFF8DC030068C821FB
:10B3A00090FBF1F201FB120000281ED1F86AC06880
:10B3B0000290F86A80680190B4F904000090B4F932
:10B3C0000230B4F90020DFF8BC030168DFF8C803DD
:10B3D000F6F7F7FEDFF8A0030068DFF8C013884235
:10B3E00003DBDFF8940300210160012006B0BDE813
:10B3F000F08130B583B001240020ADF806000020B4
:10B400008DF80400F6F75BFE05000120009001AB0B
:10B410006B22D0210020F6F7A4FF002801D10020E4
:10B420008BE09DF8040040061AD56B208DF80600CD
:10B430009DF8040010F0BF008DF8070002230DF105
:10B440000602D0210020F6F732FF002801D10020AB
:10B4500073E014212800F7F71FF8D148F6F7B1FE82
:10B460001D208DF8060008208DF8070002230DF13D
:10B470000602D0210020F6F71AFF002801D1002093
:10B480005BE00120009001AB6C22D0210020F6F798
:10B4900068FF002801D100204FE06C208DF80600E5
:10B4A0009DF8040050F080008DF804009DF8040021
:10B4B00050F007008DF804009DF8040010F0C7005C
:10B4C0008DF804009DF804008DF8070002230DF1AB
:10B4D0000602D0210020F6F7EAFE002801D1002064
:10B4E0002BE00120009001AB6B22D0210020F6F769
:10B4F00038FF002801D100201FE06B208DF80600E6
:10B500009DF8040010F0BF008DF804009DF80400C1
:10B5100050F020008DF804009DF804008DF807001D
:10B5200002230DF10602D0210020F6F7C0FE00280C
:10B5300001D1002001E02000C0B23EBD80B5002056
:10B54000ADF80000FFF755FF002801D1002045E0CD
:10B550001F208DF800004B208DF80100022300AA67
:10B56000D0210020F6F7A3FE002801D1002035E00D
:10B570001E208DF8000006208DF80100022300AA8D
:10B58000D0210020F6F793FE002801D1002025E00D
:10B5900069208DF80000C0208DF80100022300AA68
:10B5A000D0210020F6F783FE002801D1002015E00D
:10B5B000012201210320F6F7F6FF38208DF8000064
:10B5C00040208DF80100022300AAD0210020F6F7C8
:10B5D0006EFE002801D1002000E0012002BD80B5F0
:10B5E0000020ADF80000012200210320F6F7DBFF68
:10B5F00038208DF8000000208DF80100022300AAF9
:10B60000D0210020F6F753FE002801D1002058E099
:10B610006B208DF8000000208DF80100022300AAA5
:10B62000D0210020F6F743FE002801D1002048E099
:10B630001D208DF8000000208DF80100022300AAD3
:10B64000D0210020F6F733FE002801D1002038E099
:10B650006C208DF8000046480078032803D10020B4
:10B660008DF8010012E042480078022803D138200A
:10B670008DF801000AE03E480078012803D1072038
:10B680008DF8010002E03F208DF80100022300AA9E
:10B69000D0210020F6F70BFE002801D1002010E099
:10B6A00069208DF8000000208DF80100022300AA17
:10B6B000D0210020F6F7FBFD002801D1002000E09A
:10B6C000012002BD80B50178012905D1FFF74BFBB0
:10B6D00000280AD1002009E00178022905D1FFF7EE
:10B6E000D7FB002801D1002000E0012002BD80B579
:10B6F0000020ADF800001D208DF80000087800281B
:10B7000006D140208DF801002648F6F75AFD05E0E5
:10B7100043208DF801002448F6F753FD022300AAC8
:10B72000D0210020F6F7C3FD002801D1002000E061
:10B73000012002BD80B51D490020F9F70FFF1C490B
:10B740000B20F9F70BFF01BD8C310308003E4900C7
:10B75000E04A030801EFE700E84A0308D84A030873
:10B76000B8490308F04A0308F84A03087F63012038
:10B770008C6601200060002094650120004B0308C6
:10B78000084B0308F8650120104B0308746501207D
:10B79000FC650120944A0308284A0308A186010099
:10B7A000184B0308B44A0308C04A0308940303086B
:10B7B0003C49030810B50024DFF8540C0078002839
:10B7C0000AD1FEF7ACFD002801D1002007E0DFF828
:10B7D000400C0121017000E001242000C0B210BD26
:10B7E0001CB500208DF806000020ADF80400F6F727
:10B7F00066FC0400012000900DF106036B22D021AD
:10B800000120F6F7AEFD002801D1002068E09DF888
:10B8100006006021084216D06B208DF804009DF8C8
:10B82000060010F09F008DF80500022301AAD02128
:10B830000120F6F73CFD002801D1002050E01E2138
:10B840002000F6F729FE012000900DF106036C227E
:10B85000D0210120F6F785FD002801D100203FE02E
:10B860006C208DF804009DF8060010F0F8008DF8AB
:10B870000500022301AAD0210120F6F718FD0028B7
:10B8800001D100202CE00A212000F6F705FE1B2044
:10B890008DF8040008208DF80500022301AAD021AC
:10B8A0000120F6F704FD002801D1002018E01A203D
:10B8B0008DF8040003208DF80500022301AAD02191
:10B8C0000120F6F7F4FC002801D1002008E0DFF8A1
:10B8D000440B007850F00200DFF8381B087001209C
:10B8E00016BD00B583B000208DF806000020ADF82D
:10B8F0000400012000900DF106036C22D0210120EC
:10B90000F6F72FFD002801D1002030E06C208DF8E3
:10B9100004009DF8060050F007008DF80500022392
:10B9200001AAD0210120F6F7C2FC002801D1002095
:10B930001DE0DFF8E00A0078C0070FD46B208DF817
:10B94000040040208DF80500022301AAD021012027
:10B95000F6F7ADFC002801D1002008E0DFF8B40ABA
:10B96000007810F0FD00DFF8AC1A087001200EBD61
:10B9700000B583B000208DF804000020ADF806006B
:10B980000120009001AB6C22D0210120F6F7E9FCE8
:10B99000002801D1002014E06C208DF806009DF8ED
:10B9A000040050F007008DF8070002230DF1060295
:10B9B000D0210120F6F77BFC002801D1002000E017
:10B9C00001200EBD7FB5040002A80021002206C0A0
:10B9D000083800260020ADF80400F6F770FB0500DB
:10B9E0000120009002AB6B22D0210120F6F7B9FCB8
:10B9F000002801D1002083E09DF80800400625D5ED
:10BA00006B208DF804009DF8080010F0BF008DF841
:10BA10000500022301AAD0210120F6F748FC0028E6
:10BA200001D100206CE032212800F6F735FDDFF867
:10BA3000E809F6F7C6FB002603E0F6B20020305511
:10BA4000761CF6B2062EF8D3012059E001200090B2
:10BA500002AB6C22D0210120F6F783FC002801D133
:10BA600000204DE09DF808000721084225D06C20F9
:10BA70008DF804009DF8080010F0F8008DF805001E
:10BA8000022301AAD0210120F6F711FC002801D1E0
:10BA9000002035E00A212800F6F7FEFCDFF87C09DB
:10BAA000F6F78FFB002603E0F6B200203055761C37
:10BAB000F6B2062EF8D3012022E00620009002AB59
:10BAC0004322D0210120F6F74CFC002805D1DFF8F5
:10BAD0005009F6F776FB002012E09DF8090020706F
:10BAE0009DF8080060709DF80B00A0709DF80A009A
:10BAF000E0709DF80D0020719DF80C006071012030
:10BB000004B070BD2DE9F64FADF63C6D0500002088
:10BB1000ADF8080003A81421F9F76CFF002608A867
:10BB20000021002200230EC00C385FF0000940F60F
:10BB30008C1068444FF49661F9F75CFFFFA8E03081
:10BB40004FF49661F9F756FF0BA84FF49661F9F799
:10BB500051FF5FF00008002700240020070000E0EC
:10BB60007F1C032F80F2BA806B208DF80800781CB0
:10BB70008DF80900022302AAD0210120F6F797FBD5
:10BB8000002801D1002099E13220FEF78DFB6A20C8
:10BB90008DF8080044208DF80900022302AAD02164
:10BBA0000120F6F784FB002801D1002086E1012462
:10BBB00009E019EB060608A850F8270019EB000069
:10BBC00008A941F827002000441E012875DB232026
:10BBD0008DF8080070208DF80900022302AAD021F8
:10BBE0000120F6F764FB002801D1002066E14B201C
:10BBF000FEF75AFB23208DF8080000208DF809007D
:10BC0000022302AAD0210120F6F751FB002801D11E
:10BC1000002053E10220009003AB7222D0210120CA
:10BC2000F6F79FFB002801D1002047E103A8FEF7AB
:10BC300024FC00EE100AB8EEC00A10EE100AFDF760
:10BC400085F9DFF8E027DFF8E037FDF7ADF809F018
:10BC50008FF88146B9F148000128B4DB5FF0000895
:10BC60001DE003A8FEF709FC18EB060140F68C1254
:10BC70006A4422F811000DF10E00FEF7FEFB18EBEE
:10BC80000601FFAAE03222F8110004A8FEF7F5FB36
:10BC900018EB06010BAA22F8110018F10108C8459B
:10BCA00087DA0620009003AB7422D0210120F6F73A
:10BCB00058FB0028D5D1002000E123208DF8080092
:10BCC00000208DF80900022302AAD0210120F6F7F6
:10BCD000EEFA00287FF444AF0020EFE0002E01D000
:10BCE000340000E001245FF0000800200021C5E9D5
:10BCF000000100200021C5E9020100200021C5E962
:10BD0000040122E0D5E9000140F68C126A4432F9C0
:10BD10001820D31780185941C5E90001D5E902015F
:10BD2000FFAAE03232F91820D31780185941C5E92B
:10BD30000201D5E904010BAA32F91820D3178018A3
:10BD40005941C5E9040118F10108B045DADBD5E92C
:10BD500000012200E317FEF777F9C5E90001D5E9F4
:10BD600002012200E317FEF76FF9C5E90201D5E9E8
:10BD700004012200E317FEF767F9C5E904015FF04B
:10BD80000008DDF83C0E00220023C0E90023DDF8A6
:10BD90003C0E00220023C0E90223DDF83C0E002205
:10BDA0000023C0E9042382E0DDF83C2ED2E9000143
:10BDB000CDE9000140F68C10684430F91800C11735
:10BDC000D5E90023801A994140F68C126A4432F971
:10BDD00018A05FEAEA7BD5E90023BAEB02027BEB0D
:10BDE0000303A2FB00AB02FB01BB03FB00BBDDE9CD
:10BDF000000110EB0A0051EB0B01DDF83C2EC2E90B
:10BE00000001DDF83C2ED2E90201CDE90001FFA8D6
:10BE1000E03030F91800C117D5E90223801A9941A2
:10BE2000FFAAE03232F918A05FEAEA7BD5E90223E3
:10BE3000BAEB02027BEB0303A2FB00AB02FB01BBEC
:10BE400003FB00BBDDE9000110EB0A0051EB0B0125
:10BE5000DDF83C2EC2E90201DDF83C2ED2E90401F6
:10BE6000CDE900010BA830F91800C117D5E904236A
:10BE7000801A99410BAA32F918A05FEAEA7BD5E94A
:10BE80000423BAEB02027BEB0303A2FB00AB02FB31
:10BE900001BB03FB00BBDDE9000110EB0A0051EB25
:10BEA0000B01DDF83C2EC2E9040118F10108B04590
:10BEB000FFF67AAFDDF8400E066001200DF6446D06
:10BEC000BDE8F08F2DE9F04389B004000D001600A5
:10BED00001275FF0000801A8002101600320009005
:10BEE00001AB0022D0210120F6F73BFA002801D156
:10BEF0005FF0FF375FF0000907E04FFA89F905A806
:10BF0000002140F8291019F101094FFA89F9B9F116
:10BF1000030F17DA4FFA89F901A819F80000002871
:10BF2000EBD04FFA89F901A819F80000DFF8FC14EA
:10BF300011EB400030F8020C4FFA89F905A941F8DD
:10BF40002900E0E75FF0000925E04FFA89F902A82F
:10BF500050F82900DFF8D814884208DADFF8D40452
:10BF6000F6F72FF9012010FA09F050EA08084FFA05
:10BF700089F902A850F82900DFF8BC14884208DBD0
:10BF8000DFF8B804F6F71DF9012010FA09F050EABD
:10BF9000080819F101094FFA89F9B9F1030F3CDAE0
:10BFA0004FFA89F955F829004FFA89F956F82910FE
:10BFB000401A08F0D9FE4FFA89F902A941F8290080
:10BFC0004FFA89F905A850F829000028BDD04FFA8A
:10BFD00089F902A850F829004FFA89F905A951F802
:10BFE000291090FBF1F0B0F57A7008F0BDFE4FFA21
:10BFF00089F924F819004FFA89F934F9190040F247
:10C00000F5118842C5DBDFF83804F6F7DAF80120CD
:10C0100010FA09F050EA0808BBE74FFA88F8B8F1BF
:10C02000000F05D0DFF81C04F6F7CBF87FF002070D
:10C03000380040B209B0BDE8F0832DE9F0479CB06C
:10C0400004005FF0010801250CA81821F9F7D2FCC3
:10C0500006A81821F9F7CEFC02A80021016000A86B
:10C060000021002206C008385FF0000A18A800214D
:10C07000002200230EC00C3815A800210022002346
:10C080000EC00C3812A80021002200230EC00C386C
:10C0900003A80021002200230EC00C380026DFF880
:10C0A000A803D0F80490FEF7EEF9002801D1002093
:10C0B00049E1FEF7FBFA80465FFA88F8B8F1010F14
:10C0C0000AD15FF0010A02AA06A90CA8FFF71AFD1F
:10C0D000002805D1002036E1FEF740FA002032E1C9
:10C0E000FEF7C9FB002801D100202CE1002303AAA0
:10C0F00015A90020FEF7FDFB05006DB2012D03D050
:10C10000761CD248F6F75DF8002312AA18A97FF032
:10C110001F00FEF7EEFB05006DB2012D03D0B61C2B
:10C12000CB48F6F74EF818AA15A900A8FFF7CAFEE3
:10C1300005006DB2012D03D0361DC648F6F741F853
:10C14000DDE90601002901D100280BD0DDE9080155
:10C15000002901D1002805D0DDE90A01002905D117
:10C16000002803D1BC48F6F72CF8083600273AE03F
:10C17000FFB20CA810EBC700D0E9002340F2411039
:10C1800000218B420FDB01DC82420CD31036FFB260
:10C190000CA810EBC702D2E900010200FFB239007F
:10C1A000AE48F6F70EF8FFB206A810EBC702D2E9C8
:10C1B0000001029AD317FDF747FF002912DB02DCCA
:10C1C000B0F5C85F0ED34036FFB206A810EBC70229
:10C1D000D2E90001029990FBF1F2FFB23900A048C8
:10C1E000F5F7EFFF7F1CFFB2032FC1D336B2002E4D
:10C1F0001AD100220CE0D2B219EB4203D2B20CA841
:10C2000010EBC206D6E900018000A3F85800521CCA
:10C21000D2B2032AEFD3B9F95C30B9F95A20B9F98F
:10C2200058109048F5F7CDFF84F800A0BDF8000045
:10C230006070BDF900000012A070BDF80200E0704F
:10C24000BDF9020000122071BDF804006071BDF953
:10C2500004000012A071E571029820720298001289
:10C26000607202980014A07202980016E072DDE974
:10C270000C012073DDE90C0100B200126073DDE9EE
:10C280000C010014A073DDE90C010016E073DDE978
:10C290000E012074DDE90E0100B200126074DDE9C8
:10C2A0000E010014A074DDE90E010016E074DDE952
:10C2B00010012075DDE9100100B200126075DDE9A2
:10C2C00010010014A075DDE910010016E075DDE92C
:10C2D00006012076DDE9060100B200126076DDE994
:10C2E00006010014A076DDE906010016E076DDE91E
:10C2F00008012077DDE9080100B200126077DDE96E
:10C3000008010014A077DDE908010016E077DDE9F7
:10C310000A0184F82000DDE90A0100B2001284F865
:10C320002100DDE90A01001484F82200DDE90A0198
:10C33000001684F82300FEF711F9002801D100202F
:10C3400001E04046C0B21CB0BDE8F08730B583B014
:10C3500004000020ADF8040000203B494D68697AD4
:10C36000002907D1286E40688047F5F7A8FE0A210A
:10C37000F6F792F80220009001AB4122D021012073
:10C38000F5F7EFFF002801D1002017E09DF8050028
:10C390009DF8041050EA0120032110FB01F04FF436
:10C3A0007A7190FBF1F01530207000206070687A8F
:10C3B000002802D1286E8068804701203EBD80B5EC
:10C3C0000178002905D1FFF738FE00280AD10020A6
:10C3D00009E00178012905D1FFF7B8FF002801D154
:10C3E000002000E0012002BD80B5C0B2062806D1C1
:10C3F0000800FFF7ABFF002801D1002000E001207A
:10C4000002BD80B518490120F9F7A8F801BD000068
:10C410007F6301208C660120204B0308284B030812
:10C42000304B03082D211FF46C56C53F8C33030895
:10C4300030FD1300404B030879E2D100484B03085C
:10C44000384B0308504B030800600020584B03088A
:10C45000604B0308684B0308A44A0308D849030843
:10C46000404A0308804A030860490308DFF87C0556
:10C47000704730B583B00020ADF806008DF8040099
:10C480000120009001AB002218210220F5F769FF7E
:10C4900004469DF8040048281FD131208DF806007D
:10C4A0000DF106050120687002230DF10602182126
:10C4B0001846F5F7FCFE00280DD031208DF8060057
:10C4C0000020687002230DF1060218211846F5F7C6
:10C4D000EEFE002802D100203EBD002418220021DB
:10C4E000DFF80805F6F714FF20463EBD70B582B0B0
:10C4F0000020ADF8000008F06CFC0446DFF8F00402
:10C500008168497AC268527A51180069407A0818DD
:10C51000012801DB012076BDDFF8D85468780128B6
:10C520001CD032208DF8000000AE01207070022374
:10C5300000AA18211846F5F7BAFE00280CD03120C1
:10C540008DF8000001207070022300AA18211846FF
:10C55000F5F7ADFE002803D1002076BD012028703C
:10C56000281D61698847012076BD38B50020ADF8E7
:10C57000000008F02EFC0446DFF874048168497A54
:10C58000C268527A51180069407A0818022801DB03
:10C59000012032BDDFF85C542878012812D0312008
:10C5A0008DF8000000208DF80100022300AA182158
:10C5B0001846F5F77CFE002801D1002032BD00208E
:10C5C000687001E000202870281D2169884701203B
:10C5D00032BD80B50020ADF8000031208DF800009C
:10C5E00000208DF80100022300AA18211846F5F753
:10C5F0005EFE401E8041C043C00F02BD7CB50446B4
:10C600000020ADF806008DF804000120009001AB79
:10C61000002218210220F5F7A4FE05469DF804002B
:10C62000482829D131208DF806000DF106061F207B
:10C63000707002230DF1060218211846F5F737FE37
:10C64000002817D0032000902346602218210220E2
:10C65000F5F787FE00280DD031208DF80600002068
:10C66000707002230DF1060218211846F5F71FFE1F
:10C67000002802D1002076BD0025284676BD002185
:10C68000DD4A02E00B5C8B54491C1B29FADBDB48BA
:10C69000C0F8D423012070472DE9F04387B0044649
:10C6A0000D4616461F464FF000084046ADF8040000
:10C6B00002A841460A460B460EC04FF0050906C0C7
:10C6C0000120009002AB102218210220F5F749FE4C
:10C6D0009DF80810C9070ED501280CD1082000903C
:10C6E0000DF10903112218210220F5F73AFE002866
:10C6F00007D140467AE04846A0F1010980B20028FF
:10C70000DED1BF489DF80810017002A90A7A427074
:10C71000CA7982704A78C2708A780271CA78427186
:10C720000A7982714A79C271897901720AE002A894
:10C7300000EB48008178407810EB012024F81800C5
:10C7400008F10108B8F1030FF1DBA948D0F80C801B
:10C7500008F10C0999F815202146D9F80C00D8F8F1
:10C760000C30C018F7F707FA404602F0DBF999F8E9
:10C770001520D9F80C00D8F80C1041182046F7F70E
:10C78000FAF9DFF8788205AA2146404608F074FDE0
:10C7900098F9F4023860B8F8EE00288008F2EE004C
:10C7A000418869808188A98081892180C1896180CF
:10C7B000008AA08020882988401A30806088698893
:10C7C000401A7080A088A988401AB08031208DF866
:10C7D000040001208DF80500022301AA1821184643
:10C7E000F5F765FD401E8041C043C00F07B0BDE8AE
:10C7F000F08330B585B004460020ADF8040002A8EF
:10C8000000210A460B460EC005250120009002AB10
:10C81000102218210220F5F7A4FD9DF80810C90781
:10C820000ED501280CD1082000900DF1090311222A
:10C8300018210220F5F795FD002806D1002028E0F8
:10C840002846451E80B20028DFD16D489DF80810AB
:10C85000017002A90A7A4270487820708878607066
:10C86000C878A0700879E070487920719DF80E00B2
:10C87000607131208DF8040001208DF8050002233D
:10C8800001AA18211846F5F712FD401E8041C04349
:10C89000C00F05B030BD2DE9F04104460025F5F785
:10C8A000D3FF0746FFF7E2FD06465148D0F8108057
:10C8B000F86E40070BD406F1140306F10C02B11D0B
:10C8C0003046FFF7E9FE002801D1284651E098F8EC
:10C8D0000A00012848D14A480178217041786170E6
:10C8E000C178A1700179E17041792171817961711B
:10C8F000C179A171007AE0714048818D2172B0F94F
:10C900002C100912617200F12C014A88A272B1F94F
:10C9100002201212E2728A882273B1F904100912FD
:10C920006173B0F8F410A173B0F9F4100912E17357
:10C93000F43041882174B0F90210091261748188C1
:10C94000A174B0F904000012E074284620750FE0CD
:10C9500006EB4500C18804F8151004EB4501B0F959
:10C960000600001248706D1C032DF1DB7069A07188
:10C970000120BDE8F081F8B504460025F5F764FF15
:10C980000746FFF773FD0646F86E000705D52046FB
:10C99000FFF72FFF002826D109E006F1140306F166
:10C9A0000C02B11D3046FFF777FE002814D128464F
:10C9B000F2BD36F8150004F8150004EB450036F911
:10C9C00015100912417006EB45018A898271B1F98F
:10C9D0000C100912C1716D1C032DEADB18223146BF
:10C9E0000248F7F7C8F80120F2BD00002C620120D0
:10C9F0000060002008630120D8610120880901201F
:10CA0000646401207CB504460020ADF806008DF872
:10CA10000400F5F754FB05460120009001AB00220D
:10CA200018210220F5F79DFC9DF80410482932D109
:10CA300031208DF806000DF106061F2070700223CC
:10CA40000DF1060218211846F5F731FC00281BD01D
:10CA500031208DF806000020707002230DF10602CF
:10CA600018211846F5F723FC00280DD0012128468F
:10CA7000F5F712FD0120009001AB312218210220B0
:10CA8000F5F76FFC002801D1002076BD9DF8040069
:10CA90002070012076BDFF21217076BD2DE9F04781
:10CAA0008AB0044604A800210A460B460EC0084678
:10CAB000ADF80C0007A806C04FF00509F5F7FFFA1E
:10CAC00005460220009004AB00221821F5F749FC2E
:10CAD00006469DF81000482840F01D819DF8100082
:10CAE000207004AF7878607031208DF80C000DF163
:10CAF0000C081F2088F80100022303AA18211846F9
:10CB0000F5F7D5FB002800F007810320009004AB67
:10CB1000602218210220F5F724FC002800F0FC8098
:10CB20009DF81000A0707878E070B87820713120FE
:10CB30008DF80C00002088F80100022303AA1821B8
:10CB40001846F5F7B4FB002800F0E68001200090BD
:10CB500004AB312218210220F5F703FC002800F075
:10CB6000DB809DF81000607531208DF80C000120ED
:10CB700088F80100022303AA18211846F5F797FB4D
:10CB8000002800F0C9801E212846F5F785FC012009
:10CB9000009004AB102218210220F5F7E2FB0646B4
:10CBA0009DF81000C0070DD5012E0BD10820009074
:10CBB0000DF11103112218210220F5F7D2FB0028F4
:10CBC00006D16AE04846A0F1010980B20028DED112
:10CBD000B87902907879019038790090FB78BA782A
:10CBE00079780FF29010F5F7ECFAB878797811EBC4
:10CBF0000020ADF81C000DF11C0A3879F97811EB12
:10CC00000020AAF80200B879797911EB0020AAF87F
:10CC10000400BDF91C0000126071BDF81C00A07179
:10CC2000BAF902000112E1712072BAF9040001128E
:10CC30006172A0729DF81000E072387A2073312082
:10CC40008DF80C00102088F80100022303AA182197
:10CC50001846F5F72CFB00285ED01E212846F5F774
:10CC60001BFC4FF005090120009004AB1022182195
:10CC70000220F5F776FB06469DF81000C0070ED59A
:10CC8000012E0CD1082000900DF111031122182162
:10CC90000220F5F766FB002807D100203DE048465A
:10CCA000A0F1010980B20028DDD1B879029078792D
:10CCB000019038790090FB78BA7879780FF2D0003B
:10CCC000F5F77FFAB878797811EB0020ADF81C0001
:10CCD0003879F97811EB0020AAF80200B87979794F
:10CCE00011EB0020AAF80400BDF91C0000126073CB
:10CCF000BDF81C00A073BAF902000112E1732074A0
:10CD0000BAF9040001126174A0749DF81000E07477
:10CD1000387A207500E0002630460AB0BDE8F0877A
:10CD200018B404460B4611460020032C04D0042CF2
:10CD300005D0072C06D008E0184614BC5EE418465F
:10CD400012BC5FE6184612BC99E412BC704710B5DD
:10CD50000FF2580421460220F8F700FC0FF2700190
:10CD60000420F8F7FBFB21460320BDE81040F8F74C
:10CD7000F5BB0000474D53312D25642C2025642C34
:10CD80002025642C2025642C2025642C202564007B
:10CD9000474D53322D25642C2025642C2025642CEE
:10CDA0002025642C2025642C2025640073C40008F1
:10CDB000EDC400086BC50008D3C5000800000000E2
:10CDC00077C90008000000009DCA000821CD0008B6
:10CDD00073C40008EDC400086BC50008D3C5000883
:10CDE0000000000097C80008000000009DCA00086D
:10CDF00021CD00087CB500242046ADF80400F5F7ED
:10CE00005EF9054620208DF8040001AE20467070C2
:10CE1000022301AABA210520F5F749FA002801D119
:10CE2000204676BD01212846F5F736FB641C01201B
:10CE3000009001AB2122BA210520F5F792FA0028D3
:10CE400001D1002076BD40F2F510A4B2844205D392
:10CE50000FF21020F5F7B5F9002076BD9DF804001B
:10CE60000006DFD420208DF80400022070700346F5
:10CE700001AABA210520F5F71AFA401E8041C043E5
:10CE8000C00F76BD1CB504460020ADF8040001209B
:10CE9000009001AB0F22BA210520F5F762FA0028B5
:10CEA00001D1002016BD9DF80400BD2833D100F04B
:10CEB00034F8002801D1002016BD032001E0401EF7
:10CEC00040B2002807D40FF2B41151F830108C4250
:10CED00001D20028F3D120208DF8040001ACA42059
:10CEE0006070022301AABA210520F5F7E0F90028B5
:10CEF00001D1002016BD10208DF804007F20607045
:10CF0000022301AABA210520F5F7D1F9401E80417C
:10CF1000C043C00F16BD002016BD80B50020ADF87F
:10CF2000000020208DF8000000208DF80100022371
:10CF300000AABA210520F5F7BAF9002805D10FF2A9
:10CF40002C10F5F73EF9002002BD012002BD80B58E
:10CF50008F20FFF797FF401E8041C043C00F02BDE6
:10CF600080B5FFF747FF002805D10FF20810F5F74D
:10CF700028F9002002BD012002BD80B5FFF7E7FFC0
:10CF8000401E8041C043C00F02BD80B5FFF7C5FF02
:10CF9000401E8041C043C00F02BD012070470120E8
:10CFA00070471FB5044601A800210A460B460EC073
:10CFB0000120009001AB0F22BA210520F5F7D1F92D
:10CFC000002821D09DF80400BD281DD10520009027
:10CFD00001ABA822BA21F5F7C4F9002801D100203D
:10CFE00013E09DF80400207001A8417861708178F9
:10CFF000A1700021E170C178217100796071E01C9D
:10D0000000F006F8012000E0002004B010BD000090
:10D010004178007840EA01204FF4F07190FBF1F084
:10D0200000EE100AB8EEC00ADFED070A30EE200A63
:10D03000BDEEC00A10EE100A80B204490870000A62
:10D04000487001207047000000002A4288660120D5
:10D0500001207047012070470FF240010520F8F7CA
:10D060007DBA000042522D524600000042522D432C
:10D070004600000042522D504600000028000000EB
:10D080007000000050000000600000008F000000F1
:10D0900050000000E80300001000000061CF00080D
:10D0A0007BCF00088BCF00089BCF00089FCF0008E4
:10D0B000A3CF00080000000051D0000855D00008A0
:10D0C00000207047012070470120704738B50446A2
:10D0D0000D46F4F7F4FF0521F5F7DEF900201049BD
:10D0E00004E00A680255521C0A60401CA842F8DBA2
:10D0F000012032BD012070470120704709480268B5
:10D100000A704A70511C01600120704706490A6884
:10D1100002704270501C086001207047000000003F
:10D12000249B002004660120086601200FF23401D0
:10D130000820F8F713BA10B50FF228042146122080
:10D14000F8F70CFA21461320F8F708FA21461420C4
:10D15000BDE81040F8F702BA0FF208011520F8F701
:10D16000FDB90000C1D00008C5D00008C9D0000832
:10D17000C9D00008F9D00008CDD00008F5D00008CB
:10D180000DD10008FDD0000810B50024F4F797FF7A
:10D19000007CC00700D50124204610BD00B589B031
:10D1A00000A82421F8F726FC0020ADF822000A2070
:10D1B0008DF8080000208DF809008DF80A008DF820
:10D1C00000001F20019000A8FBF798FC012009B087
:10D1D00000BD00B589B000A82421F8F70BFC0020A1
:10D1E000ADF822000A208DF8080000208DF8090013
:10D1F0008DF80A0001208DF800001F20019000A882
:10D20000FBF77CFC012009B000BD00B589B000A887
:10D210002421F8F7EFFB0020ADF822000A208DF85A
:10D22000080000208DF809008DF80A0001208DF813
:10D2300000001F20019000A8FBF760FC012009B04E
:10D2400000BD0120704710B50024F4F738FF007CC2
:10D25000C00700D50124204610BD00B589B000A844
:10D260002421F8F7C7FB0020ADF822000A208DF832
:10D27000080000208DF809008DF80A008DF80000E4
:10D280002020019000A8FBF739FC012009B000BD67
:10D2900000B589B000A82421F8F7ACFB0020ADF858
:10D2A00022000A208DF8080000208DF809008DF872
:10D2B0000A0001208DF800002020019000A8FBF753
:10D2C0001DFC012009B000BD00B589B000A82421D3
:10D2D000F8F790FB0020ADF822000A208DF8080036
:10D2E00000208DF809008DF80A0001208DF800005B
:10D2F0002020019000A8FBF701FC012009B000BD2F
:10D300000120704710B50024F4F7D9FE007C800797
:10D3100000D50124204610BD00B589B000A8242105
:10D32000F8F768FB0020ADF822000A208DF808000D
:10D3300000208DF809008DF80A008DF800002120EA
:10D34000019000A8FBF7DAFB012009B000BD00B591
:10D3500089B000A82421F8F74DFB0020ADF8220089
:10D360000A208DF8080000208DF809008DF80A00C9
:10D3700001208DF800002120019000A8FBF7BEFBE2
:10D38000012009B000BD00B589B000A82421F8F73C
:10D3900031FB0020ADF822000A208DF808000020A3
:10D3A0008DF809008DF80A0001208DF80000212079
:10D3B000019000A8FBF7A2FB012009B000BD0120ED
:10D3C000704710B50024F4F77AFE007C00F00300EB
:10D3D000032800D10124204610BD00B589B000A863
:10D3E0002421F8F707FBDFF83C03017841F0020144
:10D3F00001700020ADF822000A208DF808000120FD
:10D400008DF809008DF80A1000208DF80000222008
:10D41000019000A8FBF772FB012009B000BD00B528
:10D4200089B000A82421F8F7E5FADFF8F8120878A7
:10D4300010F0FD00087014D10020ADF822000A2081
:10D440008DF8080001208DF8090000208DF80A00F1
:10D4500001208DF800002220019000A8FBF74EFB70
:10D4600002E040B208F0CCFB012009B000BD012071
:10D4700070470120704710B50024F4F720FE007CAF
:10D4800000F00700072800D10124204610BD00B598
:10D4900089B000A82421F8F7ADFAA248017841F03C
:10D4A00001010170032905D1032008F0A9FB08F050
:10D4B000C3FB11E00020ADF822000A208DF808001F
:10D4C00000208DF809008DF80A108DF80000222048
:10D4D000019000A8FBF712FB012009B000BD00B5C8
:10D4E00089B000A82421F8F785FA8E49087810F051
:10D4F000FE00087013D10020ADF822000A208DF83C
:10D50000080000208DF809008DF80A0001208DF830
:10D5100000002220019000A8FBF7F0FA04E040B2DE
:10D5200008F06EFB08F08DFB012009B000BD012062
:10D5300070470120704710B50024F4F7C0FD007C4F
:10D54000C00700D50124204610BD00B589B000A851
:10D550002421F8F74FFA0020ADF822000A208DF8B8
:10D56000080000208DF809008DF80A008DF80000F1
:10D570002320019000A8FBF7C1FA012009B000BDEB
:10D5800000B589B000A82421F8F734FA0020ADF8DE
:10D5900022000A208DF8080000208DF809008DF87F
:10D5A0000A0001208DF800002320019000A8FBF75D
:10D5B000A5FA012009B000BD00B589B000A824215A
:10D5C000F8F718FA0020ADF822000A208DF80800BC
:10D5D00000208DF809008DF80A0001208DF8000068
:10D5E0002320019000A8FBF789FA012009B000BDB3
:10D5F0000120704770B58AB004460E46FBF782F9E9
:10D600000546002000900422214600A8F6F7B3FA50
:10D6100001A82421F8F7EEF9009A31460FF2C01064
:10D62000F4F7CFFD30460C3809284ED8DFE800F07B
:10D63000051118253C0C4D4D4D481420C5F8DC044F
:10D64000207001200AB070BD1420C5F87C05207040
:10D65000F7E705F2DC403C21816208462070F0E7E4
:10D6600005F2DC4021783C2904D13C21217021784D
:10D670000165E6E700990165E3E72A480078C107FC
:10D6800012D50021ADF826100A218DF80C100021CA
:10D690008DF80D108DF80E0001208DF80400222069
:10D6A000029001A8FBF72AFA0099304640B200F038
:10D6B00012F80090206005F2DC4000998167C0E715
:10D6C0001420C5F8BC062070BBE70FF22410F4F755
:10D6D00078FD0020B6E710B4134AD36B126C114CDE
:10D6E0002478002C1AD00F2802D010280BD015E077
:10D6F000507A002812D0906B806800280ED488429F
:10D700000DDD08460BE0587A002807D0986B80683A
:10D71000002803D4884202DD084600E0084610BC19
:10D72000704700008F6601200060002012B589B0AC
:10D7300001460C3909292CD8DFE801F0051F212307
:10D74000231D2B2B2B291F240020ADF82200019034
:10D750000A208DF8080005208DF8000001940422AD
:10D7600009A90DF10900F6F706FA00A8FBF7C6F9BA
:10D7700001200AB010BD2324E6E72024E4E7212499
:10D78000E2E722240999FFF7A6FF0990DCE72B24A2
:10D79000DAE70FF26400F4F714FD0020E9E780B542
:10D7A0000FF25C010C20F7F7D9FE0FF2780111207F
:10D7B000F7F7D4FE0FF290010D20F7F7CFFE0FF22E
:10D7C000AC010E20F7F7CAFE0FF2C4010F20F7F7E5
:10D7D000C5FE0FF2E0011020BDE80440F7F7BEBE21
:10D7E0004D52322044523D25642C25640000000037
:10D7F0004D523220534446004D523220524346008F
:10D8000089D100089DD10008D3D100080BD20008AF
:10D810000000000043D20008F5D500080000000019
:10D820000000000037D500084BD5000881D500085E
:10D83000B9D5000800000000F1D50008F5D50008B2
:10D84000000000000000000047D200085BD2000882
:10D8500091D20008C9D200080000000001D30008DE
:10D86000F5D50008000000000000000005D3000806
:10D8700019D300084FD3000887D300080000000028
:10D88000BFD30008F5D5000800000000000000002C
:10D89000C3D30008DBD300081FD400086FD40008EE
:10D8A0000000000073D40008F5D500080000000057
:10D8B0000000000077D400088FD40008DFD40008EF
:10D8C0002FD500080000000033D50008F5D500086A
:10D8D000000000000000000000B500BF13009646E5
:10D8E0009446103928BFA0E80C50FAD85FEA417C72
:10D8F00028BF0CC048BF40F8042BC90728BF20F838
:10D90000022B48BF00F8012B00BD00002DE9F04FAD
:10D91000A1B0804617461D46029102AE00207062FB
:10D9200011AC6FF000490AE017F8011B0298C047DC
:10D930000290002800F06A82706A401C7062387899
:10D9400008B9706A64E22528EED10020F0603061E9
:10D950007061B061F061306201E040F0010017F8E1
:10D96000011F2029F9D023290DD02B2904D02D29DE
:10D9700006D030290AD00CE040F0020080B2EEE779
:10D9800040F00400FAE740F00800F7E740F010002C
:10D99000F4E72A290DD129680A1D2A600968F16275
:10D9A000002904D54942F16240F0040080B27F1C96
:10D9B00012E00021F16209E0F16A494505D001EB6E
:10D9C000810302EB43013039F1627F1C3A78A2F106
:10D9D0003001C9B20A29EFD339782E2903D04FF08C
:10D9E000FF31B1621DE017F8011F2A2906D129680D
:10D9F0000A1D2A600968B1627F1C12E00021B16231
:10DA000009E0B16A494505D001EB810302EB43010E
:10DA10003039B1627F1C3A78A2F13001C9B20A29CB
:10DA2000EFD3308639780FF6983008F041F908B115
:10DA300017F8010B8DF83A009DF83A00682804D1D8
:10DA4000387868280AD1622005E06C2804BF38784D
:10DA50006C2803D171208DF83A007F1C11A8B060AA
:10DA60003978B1F1250023D01C3871D0001F02286D
:10DA70006ED9133800F09680093869D0801E00F006
:10DA80002781401E00F0D180401E022860D9001F6F
:10DA900000F0CB80401F30D0401E00F08380401E3D
:10DAA00020D0C01E09D0801E7CD0C01E7AD017E1C5
:10DAB000F068411CF16025211BE12868011D2960E7
:10DAC00000687060B26A002A02D5F7F7C1FF07E06C
:10DAD000002108F0F9F800281ABF7168401AB06AEE
:10DAE000306107E12868011D296000680021CDE947
:10DAF000000111A870607821E6E09DF83A006228E4
:10DB000018D0682806D06A280BD06C2819D0712844
:10DB100007D016E02868011D2960716A006801803D
:10DB2000E8E02A68101D2860706AC1171268C2E90F
:10DB30000001DFE02868011D2960716A006801703A
:10DB4000D8E02868011D2960716A00680160D1E091
:10DB50002868C01D20F00700286000F108022A6034
:10DB6000D0E90023CDE90023002B04D5F068421C46
:10DB7000F2602D220DE0308E820704D5F068421C41
:10DB8000F2602B2205E0C00704D5F068421CF26069
:10DB900020220255F06811AA8018706000A800F0D9
:10DBA000C5F9A7E09DF83A006C2808BF2A6811D093
:10DBB000712808BF2A6802D06A282A680AD1D21DB3
:10DBC00022F007022A6094460CF108022A60DCE980
:10DBD000002303E0131D2B6012680023CDE900230E
:10DBE000682808BF92B207D0622808BFD2B203D01B
:10DBF000742818BF7A2802D10023CDE9002396F8B3
:10DC0000300000075CD5DDE90023002B08BF002AA7
:10DC100056D041F02000782852D1F06830220255C9
:10DC2000401C421CF26001554AE09DF83A0062280F
:10DC30000CD0682810D06A281AD06C2823D07128FC
:10DC400016D074281FD07A280CD01CE02868021D3A
:10DC50002A6090F900201AE02868021D2A60B0F9B5
:10DC6000002014E02868021D2A60026800230FE0EB
:10DC70002868C01D20F00700286000F108022A6013
:10DC8000D0E9002304E02868021D2A600268D31747
:10DC9000CDE90023002B04DAF068421CF2602D224B
:10DCA0000DE0308E820704D5F068421CF2602B2212
:10DCB00005E0C00704D5F068421CF260202202553E
:10DCC000F06811AA8018706000A800F0A4F811E0B4
:10DCD000F068411CF16029680A1D2A60096808E0A3
:10DCE000F068421CF2602522025519B1F068421C0E
:10DCF000F26001557F1CF06AF168401AB169401A60
:10DD00003169401AF169401A7169401A316AA0EB11
:10DD1000010A96F83000400711D420208DF8400009
:10DD2000BAF1010F0BDBD346012310AA00A940462C
:10DD300000F02FFC002869D1BBF1010BF4D1F3688E
:10DD400011AA00A9404600F024FC00285ED1302032
:10DD50008DF84000D6F818B0BBF1010F0ADB0123A3
:10DD600010AA00A9404600F014FC00284ED1BBF1D7
:10DD7000010BF4D13369726800A9404600F009FC38
:10DD8000002843D130208DF84000D6F81CB0BBF1FC
:10DD9000010F09DB012310AA00A9404600F0F9FB9E
:10DDA000A0BBBBF1010BF5D17369306971684218F2
:10DDB00000A9404600F0EDFB40BB30208DF840004C
:10DDC000D6F820B0BBF1010F09DB012310AA00A98E
:10DDD000404600F0DEFBC8B9BBF1010BF5D196F867
:10DDE000300040077FF5ABAD20208DF84000BAF140
:10DDF000010FFFF6A4AD012310AA00A9404600F0D0
:10DE0000C8FB18B9BAF1010AF5D198E54FF0FF3017
:10DE100021B0BDE8F08F2DE9FA4782B0064635699A
:10DE20006F2908BF082705D041F02000782814BFCB
:10DE30000A2710273C24D6E90001804689469DF830
:10DE40000820642A18BF692A05D1002903DAD8F10D
:10DE5000000869EB4909B9F1000F08BFB8F1000FDC
:10DE60000CD1306B50B9082F3BD196F83800000721
:10DE700037D53B24302085F83B0032E0A4F1010A7D
:10DE80005446FB17404649463A46FCF7FFF8CDE9B1
:10DE90000089B846A8FB0023DDE90089A8EB02024F
:10DEA0003032D2B23A2A03D39DF80830513B9A1847
:10DEB0000AF8052080465FEA010908BFB8F1000FA3
:10DEC00003D0F06861198842D8D3082F09D196F899
:10DED0003800000705D5605D302802D0641E302070
:10DEE0006055C4F13C00B0616119F160316B88424A
:10DEF00007DA081A3062308F4FF6EF71084030872A
:10DF000010E000290ED596F8381001F01401102900
:10DF100008D1716B7269891A326A891A081A012844
:10DF2000A8BF306204B0BDE8F08700002DE9F24FD1
:10DF30008EB0044604AED4E90001CDE902019DF89B
:10DF4000380040F020008DF8000061280BD0206BD5
:10DF5000002848BF062005D404BF9DF800006728AC
:10DF600001D1012020636168C1F30A5040F2FF73C0
:10DF700098421ED1080304BF206800280AD103205C
:10DF8000A0619DF838006138C0B21A2838D30FF26A
:10DF9000446109E00320A0619DF838006138C0B2F7
:10DFA0001A282AD30FF224610322E068F5F7A8FDAE
:10DFB000B9E1012817DA204607F0B2FE012812DB8A
:10DFC000002700209DF80010612920D1E16830224F
:10DFD00001F8012B4A1CE2609DF83820612A0CBF31
:10DFE000782258220FE040F2FE31626861F31E523F
:10DFF0006260471A4FF0FF30E4E70FF2CC51D3E7ED
:10E000000FF2CC51D0E70A706169891C616110B9C7
:10E01000002500277EE19DF80000612840F09780F0
:10E02000206B00284CBF2125451C2DB26E1CD4E965
:10E030000089DDE902010022002307F093FE3ABFC8
:10E0400089F00040CDE90280CDE902893F1F8DF8BB
:10E0500010200DF11108012E35DBDDE9020100224F
:10E06000002307F097FE2ED21C2102A807F0AAFE7B
:10E07000DDE9020106F07CFE8146F61F012E09DB78
:10E08000FAF77AFE02460B46DDE9020107F024FFAB
:10E09000CDE9020108F20700072105E009F00F02AF
:10E0A00000F8012D4FEA2919B9F1010F01DB491ED2
:10E0B000F4D5491E5CBF002200F8012DF9D500F20D
:10E0C0000708012EC9DA0DF11100A8EB00010DF1CE
:10E0D0001106A942B8BF0D462DB2002D30D42846F6
:10E0E000884206DA04A941184978082928BF0F2177
:10E0F00000D2002104AA821800E06D1E401E12F812
:10E1000001398B42F9D00F2904D104A941184A786A
:10E11000521C4A70002802D504AE6D1C3F1D2DB262
:10E12000681E0DD481190A783032D2B23A2A03D34C
:10E130009DF838303A3B9A1801F80129401EF2D573
:10E14000206B002840F1E680681E2063E2E0DDE9F4
:10E1500002010022002307F005FE3CBF81F00041D0
:10E16000CDE902013FB247F297507843474990FB0F
:10E17000F1F73FB2C7F107069246DFF814B1012E5E
:10E1800019DBDDE90289F00707D552465B464046B8
:10E190004946FAF709FE80468946761050465946A8
:10E1A00052465B46FAF700FE82468B46002EEAD1C5
:10E1B000CDE9028921E076429046DFF8D89012E05E
:10E1C000F00707D552465B4640464946FAF7ECFD54
:10E1D0008046894676105046594652465B46FAF7C5
:10E1E000E3FD82468B46002EEAD1DDE9020142467C
:10E1F0004B4607F031FFCDE902019DF8000066288B
:10E200000CBF07F10A000620216B4518142DA8BF8A
:10E21000132530208DF810000DF11106DFF87890ED
:10E22000012D3BDBDDE9020106F0B8FD06F1080136
:10E2300004220A26B0FBF6F303EB830EA0EB4E009C
:10E24000303001F8010DB3FBF6F000EB8006A3EBD4
:10E250004603303301F8013D521EEAD101F10806B0
:10E26000083D012DDCDBDDE9020106F097FDFAF740
:10E270008DFD02460B46DDE9020107F02DFE00226E
:10E280004B46FAF791FDCDE90201CBE7A0860100EC
:10E29000000024400000F03F84D797410DF11100A9
:10E2A000301A0DF1110602E0401E7F1E761C3178F7
:10E2B0003029F9D09DF80010662902D13FB2791CAF
:10E2C00003E065290CBF01210021226B8D182DB2BE
:10E2D000A842B8BF05462DB2002D1BD42946814265
:10E2E00004DA885D352828BF392000D230208A1909
:10E2F000521E00E06D1E491E12F801398342F9D00A
:10E30000392802D1885D401C8855002902D5761E27
:10E310006D1C7F1C3FB200972BB232469DF838101F
:10E32000204600F003F80FB0BDE8F08F2DE9F04370
:10E3300085B00546894617461E46D5F83080012E21
:10E3400002DA01260FF2902749F02000BDF9304093
:10E35000662808BF641C18D0672840F082806FF0E0
:10E3600003008442C0F28380444580F28080641CB4
:10E3700095F83800000702D44645B8BFB04624B22D
:10E38000B8EB040848BF4FF00008E868A96924B258
:10E39000012C25DA4A1C30230B54B8F1010F03DAA3
:10E3A00095F83810090702D52E211154521CAA6184
:10E3B00018EB040FB8BFC8F1000424B261426962CF
:10E3C000A044B045B8BF464636B2EE613246394643
:10E3D000AB691818F5F794FBA8EB0600A862C1E03A
:10E3E0000818A64218DA32463946F5F789FBA969BA
:10E3F0007118A961A01B6862B8F1010F03DA95F8E2
:10E400003800000705D5E8682E220A54E869401C48
:10E41000E861C5F82880A5E022463946F5F770FB8B
:10E42000A8692018361BB8F1010F03DA95F83810E7
:10E43000090703D5E9682E224254401CA86136B270
:10E44000B045B8BF464636B23246E119EB68C0184F
:10E45000F5F756FBA8693018A861A8EB06006862BA
:10E4600080E0B9F1610F16D14FF0700918E0464510
:10E4700004DA95F83810090758BFB046B8F101081A
:10E4800048BF4FF00008B9F1670F14BF4FF04509BE
:10E490004FF0650904E0B9F1410F08BF4FF0500992
:10E4A000A9694A1CE86817F8013B0B54B8F1010F41
:10E4B00005DA95F83810090758BFAA6117D52E213B
:10E4C0001154531CAB61B8F1010F10DB761E36B24C
:10E4D000B045B8BF464636B2324639461818F5F749
:10E4E0000FFBA8693018A861A8EB06006862A8694C
:10E4F000E968471807F8019B002C03D42B2007F884
:10E50000010B03E02D2007F8010B644200260DF1FA
:10E51000080809E00A22214600A807F0C0FE019879
:10E5200008F8010B009C761C24B2012CF2DA022EB2
:10E5300006DA49F02000652804BF302007F8010BF7
:10E540004EB9302007F8010B07E0761E02A8305CB8
:10E55000303007F8010B012EF7DAA869E968401896
:10E56000381AE86195F8380000F0140010280DD131
:10E570006869A9690818696A0818E9690818A96A20
:10E580000818696B8842BCBF081A286205B0BDE84C
:10E59000F083F8B504460D4616461F46002077B1B5
:10E5A00016F8011BA868A047A86030B1E86A401CB3
:10E5B000E86200207F1EF3D1F2BD4FF0FF30F2BDC4
:10E5C000686A6C747A4C00006E616E004E414E00B9
:10E5D000696E6600494E4600300000000CB41CB560
:10E5E000044604A80190009401AB0A4600A907481C
:10E5F00078441830FFF78AF9009900220A70002841
:10E600005CBF0098001B16BC5DF80CFB7B74FFFF21
:10E6100001B58B0718D1121F21D351F8043BA3F188
:10E62000013C2CEA030C1CF0803C04BF40F8043B86
:10E63000F1E79CFA8CFCBCFA8CF1C1F118018B401B
:10E64000CB4040F8043B13E0042A09D311F8013B06
:10E65000521E00F8013B5BB18B07F7D1DBE7121DBF
:10E660005AB111F8013B521E00F8013B03B1F8D139
:10E6700011001CBF0022FAF7DDFC01BD002801D10A
:10E680000A48806890F84C10642901D0002000E00E
:10E69000806A7047002801D10448806890F84C10C7
:10E6A000642901D0002000E0406A7047F8990020FA
:10E6B0000248704702480149401A70470040002054
:10E6C000006000204C48C168002903D54B49016017
:10E6D0004B49016070474B48016841F000410160BF
:10E6E000704770B50446002600290BD0012902D1DD
:10E6F0004FF4807606E0022902D14FF4007601E063
:10E700004FF4407600F082F809281ED13D4D28686C
:10E7100020F440702860286830432860286820F082
:10E72000F8002860286844F002010843286028683F
:10E7300040F48030286000F069F8296821F0020177
:10E740002960296821F0F801296070BD70B5044680
:10E750000D4600F05BF8092813D12A4E306820F4EA
:10E7600040703060306840F400703060306840F0D5
:10E7700001003060256000F049F83168490849001F
:10E78000316070BD70B505460E4600F03FF80928AF
:10E7900011D11C4C206820F440702060206820605B
:10E7A000206840F0010020602E7000F02FF82168F2
:10E7B00049084900216070BD13490860704709206D
:10E7C00011490A68D20301D5012070470A68D206B0
:10E7D00001D5062070470A68D20501D5022070478E
:10E7E0000A6812F0EF0F01D0072070470968890707
:10E7F00000D5082070470000043C02402301674513
:10E80000AB89EFCD103C02400C3C024080B50920A2
:10E810008DF80000FFF7D3FF8DF8000003E0FFF74D
:10E82000CEFF8DF800009DF800000128F7D09DF87C
:10E83000000002BD0901002806D500F00F004C4A77
:10E84000801800F8041C70474A4A8154704710B57C
:10E85000B0F1807F01D3012010BD474C0002000AB7
:10E86000401E60600F214FF0FF30FFF7E3FF0020F4
:10E87000A06007202060002010BD38B53F4D2878EB
:10E88000401C28703E4C2078401C2070F7F7A7FFF2
:10E8900007F00CFD2878411E2970002802D198202D
:10E8A000F7F7F6F82078012804D16068002801D035
:10E8B000F7F751F92078401E207031BD10B5304C6B
:10E8C0006078F021084202D09920F7F7E1F8F7F7D5
:10E8D0004CF96078401C607007F042FD29480068E0
:10E8E0004FF47A71B0FBF1F0FFF7B1FF002800D0D0
:10E8F000FEE72548254901600E214FF0FF30FFF764
:10E9000099FF6078F021084202D09920F7F7C0F80B
:10E910006078401E6070C0B2002803D1BDE810408E
:10E92000F7F71DB910BD0000194C4FF400512046F7
:10E93000FAF758FD30BF4FF400512046FAF750FD6A
:10E94000F3E710B40E48006A0E4909684FF47A7272
:10E95000B1FBF2F10F4A1368CB1A0F4C2468640123
:10E9600002D512688B1A401C00FB013010BC7047A6
:10E9700018ED00E000E400E010E000E0B5660120E2
:10E98000F8990020AC9A002008ED00E00000000893
:10E990000010024018E000E004ED00E0EFF3058015
:10E9A000002847F03D85704780B5EFF3108072B6C0
:10E9B0000B49096851F47F01094A116080F31088FE
:10E9C0000848006810F4700F02D1A720F7F760F82C
:10E9D00005485FF00071016004480021016001BD3D
:10E9E00020ED00E088ED00E03CEF00E034EF00E0D7
:10E9F00080B5F3F729FFDFF828180860012002BD71
:10EA000010B5F6F76DFA0246C317DFF81848D4E9D7
:10EA10000001101A0021012905DB01DC002802D3C6
:10EA2000C4E90023084610BDF0B583B0044600A831
:10EA300000210A4606C0A069E16845182888ADF89B
:10EA40000000B5F9027000A84780B5F9046086801F
:10EA5000BDF80000B4F85810401A2880B4F85A00E5
:10EA6000381A6880B4F85C00301AA880BDF900003C
:10EA7000B5F90010C913B1EBE03F13D0B4F9581049
:10EA8000C913B1EBE03F0DD00FF2B470F3F799FB6F
:10EA9000B5F90000012802DBDFF88C0701E047F63A
:10EAA000FF702880B5F90210C913B1EBE73F13D00E
:10EAB000B4F95A10C913B1EBE73F0DD00FF28C70C7
:10EAC000F3F77FFBB5F90200012802DBDFF85807F6
:10EAD00001E047F6FF706880B5F90410C913B1EB87
:10EAE000E63F13D0B4F95C10C913B1EBE63F0DD08B
:10EAF0000FF26470F3F765FBB5F90400012802DB3F
:10EB0000DFF8240701E047F6FF70A88094F90800B9
:10EB1000002804D1002000E0401C0328FCDBF7BDE6
:10EB200000000000FEB5044600A800210A460B467E
:10EB30000EC0A069E1684518174694F90860052ED3
:10EB400080F09A80012E02D12046FFF76DFF3046FB
:10EB5000012802D9C01E40F08A80002E01D14FF654
:10EB6000FF77DFF8BC060068301890F88400401E7C
:10EB700006285ED8DFE800F004101D2936424F0059
:10EB8000B5F90200009000A8B5F90010791A4160AB
:10EB9000B5F90410816056E0B5F90000381A00900C
:10EBA00000A8B5F90210791A4160B5F90410816026
:10EBB00049E0B5F90200381A009000A8B5F9001034
:10EBC0004160B5F9041081603DE0B5F90000381AE4
:10EBD000009000A8B5F902104160B5F90410791A47
:10EBE000816030E0B5F90200009000A8B5F900108E
:10EBF0004160B5F90410791A816024E0B5F900008C
:10EC0000009000A8B5F90210791A4160B5F9041016
:10EC1000791A816017E0B5F90200381A009000A84F
:10EC2000B5F90010791A4160B5F90410791A8160BC
:10EC300009E0B5F90000009000A8B5F902104160A4
:10EC4000B5F904108160012E0AD1002106E050F8C8
:10EC5000212002F30F0240F82120491C0329F6DB92
:10EC60000098288000A8416869808068A880002EEC
:10EC700002D12046FFF7D8FE0120FEBD70B52DED74
:10EC8000028B84B000A9002213460CC18169C268BE
:10EC90008A1890F9081008460A2800F2A480DFE8D4
:10ECA00000F006317FA2A271A2A2A28C9A00108865
:10ECB000ADF80000B2F9024000A84480B2F9045057
:10ECC0008580DFF85C0500689FEDAF0ABDF9001094
:10ECD00000EE901AF8EEE00A60EE800AC0ED000A3D
:10ECE00000EE904AF8EEE00A60EE800AC0ED010AFC
:10ECF00000EE905AF8EEE00A20EE800A001D80ED4A
:10ED0000010A74E01088ADF80000B2F9024000A8D2
:10ED10004480B2F904508580DFF804050068061DC0
:10ED20009FEDC18BBDF9000000EE100AB8EEC00ADD
:10ED300010EE100AFAF70AF953EC182BFAF734F828
:10ED4000FAF72CF9B06000EE104AB8EEC00A10EEE7
:10ED5000100AFAF7FBF853EC182BFAF725F8FAF734
:10ED60001DF9F06000EE105AB8EEC00A10EE100A5D
:10ED7000FAF7ECF853EC182BFAF716F8FAF70EF945
:10ED8000306134E018460290106802909DED020A4E
:10ED9000BAEECA0ADFF88804006880ED0C0A26E0A3
:10EDA000DFF87C0400681188A0F85A1000F25A00BD
:10EDB000518841809188818019E0DFF864040068FF
:10EDC00000F25A001188C1805188018191884181E7
:10EDD000D18881810BE0DFF84804006892F90010C7
:10EDE00080F8681003E00FF27C40F3F7EAF90120A5
:10EDF00004B0BDEC028B70BD70B50D46DFF82C146D
:10EE000051F820400026207F002801D1304670BDF7
:10EE1000607A002803D0206E806880470646284626
:10EE2000216EC96988470546002E02D0206E4068D1
:10EE30008047284670BD01207047F0B4002A10D4E6
:10EE400000F11004A57C066992FBF1F76F43B7420D
:10EE500002DAA263E26304E096FBF5F25143A16398
:10EE6000E163002B03D4990701D510300374F0BC83
:10EE70007047002903D4002181644161816170479A
:10EE8000C0B2042817D101F10C008A7A012A09D0F6
:10EE9000072242750B228275DFF89423CA600B218A
:10EEA000416070471522427519228275DFF884236C
:10EEB000CA60192141607047F2B5044615461A46EA
:10EEC000E4B2162C47D264B2DFF8600350F8246035
:10EED0000227307F00283ED00846C82802D1B4203F
:10EEE000009003E0422801D13C2000909DF91830A9
:10EEF000002B06D4D80704D500993046FFF79BFFB6
:10EF0000F2BD00993046FFF798FFA4F10C00C0B2A3
:10EF1000062805D22146C9B200A8326E92699047F0
:10EF200031462046FFF7ACFF707A00281BD12946F6
:10EF300049B23046726E1268904700280DD0306E8C
:10EF400040688047002804D139464F1EC9B20029C5
:10EF5000F5D1002801D10020F2BD294649B2304642
:10EF6000726E52689047707A401C70720D2C08D0F7
:10EF70002A4652B200993046736E1B69984700F0DA
:10EF8000B7F80120F2BD000060F61C3A2DE9F0410F
:10EF900004460D4616461946E4B2162C08D264B251
:10EFA000A24850F824704FF00208387F002801D1A1
:10EFB000002036E0C82D01D1B42502E0422D00D159
:10EFC0003C253846FFF755FF787A012818D131469D
:10EFD00049B238467A6E9268904700280AD0386E57
:10EFE00080688047002805D14046A0F10108C0B2E2
:10EFF0000028F4D1314649B238467A6ED26890473B
:10F00000787A002801D0401E78720D2C08D0324644
:10F0100052B2294638467B6E5B69984700F068F823
:10F020000120BDE8F081000089AD84FA0A74313F07
:10F030002DE9F04104460D4616461A46E4B2162C58
:10F0400025D264B2794850F82470387F00281ED049
:10F05000C82D01D1B42502E0422D00D13C250D2C54
:10F0600001D1012042E09DF91830002B06D4D807C9
:10F0700004D529463846BDE8F041DCE606EB4600FB
:10F0800007EB8008D8F838008068002801D50020F8
:10F090002CE029463846FFF7D0FED8F838008068C3
:10F0A000854215D0012D13DB0FF2C410F3F789F858
:10F0B000324652B2D8F83800816838467B6E5B69B8
:10F0C0009847324652B2294638467B6E1B699847AC
:10F0D000A4F10C00C0B2062805D229462046FEF74E
:10F0E00025FB012002E000F003F80120BDE8F081DB
:10F0F00070B56FF0004634464F48016804E08A68F6
:10F10000A24200DA144609688142F8D14B4D2878B2
:10F11000401C28706878F021084202D09920F6F748
:10F12000B7FCF6F722FD6878401C6870B44200D145
:10F1300000243B4E3068C467D0F8802021468A42C4
:10F1400012D0002901D0002A0BD1C0F880100FF294
:10F150003010F3F736F83068D0F88000F3F70DF888
:10F1600002E0012007F082F96878F021084202D01D
:10F170009920F6F78DFC6878401E6870C0B20028B0
:10F1800001D1F6F7ECFCF7F746FB012070BD38B56E
:10F1900005462A4C2078401C20706078F0210842F7
:10F1A00002D09920F6F774FCF6F7DFFC6078401C7B
:10F1B000607029460FF2DC00F3F703F81848006886
:10F1C000C0F880501C48016805E08A68B2FBF5F27F
:10F1D0006A43CA6009688142F7D16078F021084229
:10F1E00002D09920F6F754FC6078401E6070C0B2DF
:10F1F000002801D1F6F7B3FCBDE83140F7F70BBBAF
:10F200000D490A6808E01369012B01DAD36813611C
:10F2100013691B1A136112688A42F4D17047000007
:10F2200018660120986501200080FFFF0060002023
:10F23000847000201062012070600020F899002086
:10F2400058206973206F7665720000005920697339
:10F25000206F7665720000005A206973206F766512
:10F260007200000055435354282564294E53000072
:10F270006368616E6765207261746532000000002A
:10F28000675F707453682D3E6354696D6572203DED
:10F29000202564006374696D6572203D202564003B
:10F2A00038B504000D0014480078401C124908705D
:10F2B00012480078002802D0A120F6F7E9FBF7F702
:10F2C00069FA607E662802D08220F6F7E1FBF6F745
:10F2D0004CFC05E03821200007F0CEF8F6F745FC9D
:10F2E000E06821698842F5D02900200007F0E6F89F
:10F2F000F7F791FA31BD00BFF8990020B6660120FA
:10F300004FF0FF31801E012814D9C01E042811D9E6
:10F31000801F05280ED908380CD0801E042809D972
:10F32000401F05D0401E102804D9113804D004E035
:10F33000072102E0012100E003210846704780B563
:10F3400001460020C91E1AD0C91E18D0C91E16D0E9
:10F35000C91E012913D90D39032910D9091F07D056
:10F36000491E0CD0C91F032909D9C91F07D002BDE6
:10F370001D210FF21000F2F724FF012002BD012031
:10F3800002BD000050443A204C4C5320256400003C
:10F3900038B504464FF0FF35F9F7B4FA2C2C36D8BF
:10F3A000DFE804F034353234343234343232353438
:10F3B0001932171734353532353434341934323480
:10F3C0003234341C1F23272B2E3232323232303269
:10F3D0003400B4251BE04FF47A7518E0D0F8DC5403
:10F3E00015E000F2DC40856A11E000F2DC40056DBA
:10F3F0000DE000F2DC40856F09E0D0F87C5506E0B6
:10F400000A2504E0052502E0142500E03C252846F5
:10F4100032BD38B5DFF8684AF3F716FAE06207F054
:10F42000B5F8F9F76FFA2063002512E0DFF8541AF7
:10F430000161DFF8541A4161DFF8502A8261DFF878
:10F44000502AC261DFF84C2A02624162406A80475A
:10F450006D1C2D2D80F21881216B05EB8500C000FD
:10F4600000224254401842704FF0FF3242600022A6
:10F470000272C2604272032D04D17431DFF8182A7F
:10F480008A62E3E7022D03D1DFF8102A4A67DDE73D
:10F49000002DCBD0042D04D17431DFF8042A0A6585
:10F4A000D4E7052D04D17431DFF8F8298A67CDE758
:10F4B000062D04D1DFF8F029C1F81421C6E7072D85
:10F4C00005D101F58A71DFF8E4298A62BEE7082DCB
:10F4D00005D101F58A71DFF8D8290A65B6E7092D4B
:10F4E00005D101F58A71DFF8CC298A67AEE70A2DCC
:10F4F0009CD00B2D9AD0012D98D00C2D04D1DFF883
:10F50000B829C1F80422A1E70D2D05D101F501713B
:10F51000DFF8A8298A6299E70E2D05D101F501715E
:10F52000DFF89C290A6591E70F2D05D101F50171DE
:10F53000DFF890298A6789E7102D04D1DFF8882940
:10F54000C1F8A42282E7122D3FF470AF142D3FF4CE
:10F550006DAF132D3FF46AAF162D3FF467AF2B2D1F
:10F560003FF464AF152D04D1DFF86029C1F86C2396
:10F570006CE7172D05D101F55B71DFF854290A6599
:10F5800064E7182D05D101F55B71DFF848298A671A
:10F590005CE71A2D05D101F20C41DFF83C298A62A3
:10F5A00054E71E2D05D101F2AC41DFF830298A6203
:10F5B0004CE7192D04D1DFF82829C1F80C2445E7C0
:10F5C0001F2D05D101F2AC41DFF818290A653DE78E
:10F5D000202D05D101F2AC41DFF80C298A6735E70F
:10F5E000212D04D1DFF80429C1F84C252EE7222D66
:10F5F00005D101F24C51DFF8F8288A6226E7232D65
:10F6000005D101F24C51DFF8EC280A651EE71B2DED
:10F6100005D101F20C41DFF8282A0A6516E71C2DF6
:10F6200005D101F20C41DFF81C2A8A670EE71D2D77
:10F6300004D1DFF8142AC1F8AC2407E7262D04D141
:10F64000DFF8082AC1F8142600E7272D05D101F2BA
:10F650001461DFF8FC298A62F8E6292D05D101F250
:10F660001461DFF8F0298A67F0E62A2D04D1DFF86B
:10F67000E829C1F8B426E9E62C2D7FF4D7AEDFF8EF
:10F68000DC29C1F80427E1E6012032BD0CB42DE9E4
:10F69000F04385B004460E4601251A2C46D02C2C8A
:10F6A00044D004EB8400C700DFF8D4870B2E20D1B0
:10F6B000D8F8300007EB000999F80100002818D0AD
:10F6C0002046FFF71DFE012813DB2046FFF718FE3A
:10F6D00099F8011081420CDB204600F0A9F905469B
:10F6E000D8F830003818002141700FF67C10F2F77E
:10F6F00068FDD8F83000395C00294ED139184A78B5
:10F70000002A4AD100223A54104648700CA983B00E
:10F7100068461822F4F704FA0EBC204600F07EF882
:10F72000022835D0032838D1032536E00B2E16D118
:10F73000FFF7E6FD012812DB2046FFF7E1FD04EBB1
:10F740008401DFF83C27126B02EBC101497881424A
:10F7500005DB0FF61C10F2F734FD022059E01A2CDD
:10F7600004D13046C0B202F0D3F805E02C2C03D10E
:10F770003046C0B207F030F80CA983B068461822B2
:10F78000F4F7CEF90EBC204600F048F8022801D16B
:10F7900002203EE0032800D103250A2E0AD1DFF81B
:10F7A000E086D8F8300004EB8401CF00395C491CB6
:10F7B000395416E00B2E14D1DFF8C486032C07D180
:10F7C000D8F8300090F87900002801D101F0F6FA5D
:10F7D00004EB8400C700D8F8300038184178491C81
:10F7E0004170DFF89C86D8F83000D8F82C1004EB74
:10F7F0008402D700D1E91C23CDE90223C96E009110
:10F8000039184B783A5C21460FF67000F2F7D9FCB4
:10F81000284605B0BDE8F0035DF80CFB0EB42DE9F9
:10F82000F04183B00546012405EB8500C600DFF8F2
:10F8300050761A2D0CD02C2D0AD02846C0B2FFF7D6
:10F84000A7FD396B7118486000200872C86011E08C
:10F85000386B315C00290DD130184078002809D16F
:10F860002846C0B2FFF794FD396B7118486000203C
:10F870000872C86009A984B068461822F4F750F9E4
:10F880000FBCD7F830C066443669B047022801D1B2
:10F89000022011E0032801D103240CE0D7F82C80CA
:10F8A000D8E91C67204600212A4600F035FC304389
:10F8B0003943C8E91C012046BDE8FE015DF810FB94
:10F8C0002DE9FF4704460D460126274607EB870032
:10F8D0004FEAC008DFF8A895D9F830001A2C58D0A4
:10F8E0002C2C56D008EB000A9AF80100022814D3F9
:10F8F0002046FFF705FD01280FDB2046FFF700FD3E
:10F900009AF80110814208DB2046FFF7F9FC8AF8DB
:10F9100001000FF27C70F2F754FCD9F8300018F8AF
:10F920000010002904D108EB00025278002A67D0A9
:10F930000A2D09D1002903D0491E08F8001017E04C
:10F94000002108F8001013E00B2D11D108EB000185
:10F950004A78002A02D0521E4A7001E000224A7002
:10F96000032C05D190F87900002801D101F035FA77
:10F97000D9F8300018F80010002941D140444078EF
:10F9800000283DD1204600F053F8032838D1032643
:10F9900036E018F80010002904D108EB0002527874
:10F9A000002A2DD00A2D09D1002903D0491E08F8BC
:10F9B000001012E0002108F800100EE00B2D0CD111
:10F9C00008EB000A9AF80100002803D0401E8AF8CC
:10F9D000010002E000208AF801001A2C04D1284618
:10F9E000C0B201F095FF05E02C2C03D12846C0B22F
:10F9F00006F0F2FE204600F01BF8032800D1032693
:10FA0000D9F83000D9F82C10D1E91C23CDE9022314
:10FA1000C96E009108EB00014B7818F800203946B8
:10FA20000FF27460F2F7CDFB304604B0BDE8F0870A
:10FA30002DE9F0410746012607EB8700C500DFF8F6
:10FA40004044206B281840698047032800D10326D2
:10FA50002C2F08D1206B90F8E01600290AD190F8DD
:10FA6000E106002806D1384640B200F080F90328AC
:10FA700000D10326206B295C002917D12818417872
:10FA8000002913D14FF0FF31416000210172C160A4
:10FA9000D4F82C80D8E91C4501203A4600F03CFB04
:10FAA00024EA000025EA0101C8E91C013046BDE84E
:10FAB000F08138B5044604EB8400C000DFF8C05381
:10FAC000296B002242544018114641702046FFF72E
:10FAD000AFFFE86AD0E91C2321460FF2D050F2F7BD
:10FAE00070FB012032BD2DE9F041B6B004460E4650
:10FAF000B6B201208DF86400DFF884531AA8E96AD1
:10FB00006C22F4F70DF817951AA984B068466C2298
:10FB1000F4F706F80FBC00F0EFF900270BE003281C
:10FB200003D1189703208DF86400286B404400210E
:10FB300001727F1C7FB22D2F2BDA012000213A4663
:10FB400000F0EAFAD5F82CC0DCE91C23104019407B
:10FB500001D10028EDD007EB87004FEAC008286BE1
:10FB6000404441680029E4D4027A521C0272D2B2A5
:10FB7000724389B28A42DCDB806980470228CED199
:10FB8000189702208DF86400DDE91801C4E900012E
:10FB900003E0DDE91801C4E9000136B0BDE8F081F9
:10FBA00000210A3842F20772904200D20121084631
:10FBB00070472DE9F04383B00446002001900422F1
:10FBC00004F1090101A8F3F7D6FF6168DFF8B0621C
:10FBD000376B282505FB01704068019A904204D1DB
:10FBE0000FF2D840F2F7EDFA6AE01046FFF7D8FFBF
:10FBF000002809D16168019B05FB017042680FF282
:10FC0000C840F2F7DEFA5BE0DFF854743868D0F8E9
:10FC1000008026E090F908906068316B05FB0010C9
:10FC2000C068012101FA09F1084217D04FF0FF30F6
:10FC300000900346012201994846FFF73DF940B282
:10FC400000280BD1616801980090306B05FB010022
:10FC500043684A460FF28440F2F7B3FA4046D0F8C0
:10FC60000080B842D6D13868D0F8008020E090F902
:10FC70000890C868012202FA09F2104215D04FF02C
:10FC8000FF33012249684846FFF780F940B2002857
:10FC90000BD1616801980090306B05FB010043684F
:10FCA0004A460FF25040F2F78CFA4046D0F80080F6
:10FCB0006168326B05FB0121B842D8D101984860D8
:10FCC000BDE8F7832DE9F84381464FF0000844462C
:10FCD0006B4E1FE004EB8400C500306B2F18002032
:10FCE000787201200021224600F016FAD6F82CC0C6
:10FCF000DCE91C231040194001D1002809D04846F6
:10FD0000F9698847002804D0306B28180121417216
:10FD10008846641C2D2CDDDB4046BDE8F283584844
:10FD2000C16AD1E91C23002B01D1002A0BD000218C
:10FD300007E001EB8102036B03EBC2020023537265
:10FD4000491C2D29F5DB704730B502460120002102
:10FD500000F0E2F94A4AD26AD2E91C452040294023
:10FD600001D1002801D0012030BD002030BD2DE997
:10FD7000F0478146012409EB8900C500404E306BF5
:10FD80002818C068002829D0DFF8D4723868D0F865
:10FD9000008003E003244046D0F80080B8421DD024
:10FDA00090F908A0306B2818C168012202FA0AF203
:10FDB000114021FA0AF149B20129ECD14FF0FF3389
:10FDC000012241685046FFF7E1F80028E2D0524690
:10FDD00049460FF23830F2F7F4F9DCE72046BDE887
:10FDE000F08710B58AB004460020ADF822000190DB
:10FDF0000A208DF8080000208DF809008DF80A000F
:10FE0000ADF82200600719D50520FFF79DFF0028F7
:10FE100007D004208DF800000520019000A8F8F715
:10FE20006DFE0220FFF790FF002807D004208DF818
:10FE300000000220019000A8F8F760FEE0060CD553
:10FE40000820FFF781FF002807D003208DF800006D
:10FE50000820019000A8F8F751FE0AB010BD024634
:10FE60000020092A00D0704780B5012902D107F08F
:10FE700069FE012002BD02492C22F3F751BE0000A9
:10FE80000C600120758C0008718C00087D8C0008C6
:10FE9000818C0008858C00089D070108393701080E
:10FEA0003D010108FD34010827300308ED41030836
:10FEB00035330108937A010853040108D52E03084D
:10FEC000D12303081D390308A33F03080543030892
:10FED00035450308F9370308A1240108172A030848
:10FEE000F53B0308CB9D0108D74003089336030870
:10FEF000A35B01084F9C01080FB41B980099016097
:10FF000001994160029981600399C160049901617E
:10FF100005994161BDF85A100183BDF85C10418319
:10FF2000BDF85E1081830C990162139941621499A6
:10FF3000816204B0704700004168122903D1C17A80
:10FF4000002000F0FCBF132903D1017B012000F049
:10FF5000F6BF142903D1417B022000F0F0BF152920
:10FF600002D1C07A00F0FCBF172961D1817A1B2928
:10FF700008D01C2932D01D2911D0262928D02C299F
:10FF80003CD07047C17B012903D1B0F80B0003F0CE
:10FF9000FFB802294CD1B0F80D0003F0F7B8017D8D
:10FFA000012903D1B0F80B0008F0BCB8022903D135
:10FFB000B0F80D0008F0AAB8042903D1B0F8170072
:10FFC00008F0B2B8032933D1B0F8150008F0B8B87A
:10FFD000C17B01292CD1807B08F0D5B9817B012917
:10FFE00002D1C07A08F0DBBB022902D1007B08F005
:10FFF000E0BB05291CD1407B08F0BBBB417D01293A
:020000021000EC
:1000000002D1C07B07F0F5B9022902D1C08A07F0FE
:10001000DCB9032902D1008B07F0E1B9042902D130
:10002000408B07F004BA052902D1808B07F0F1B9A3
:1000300070470C49086070470A4800687047000024
:1000400035310108ED850108AB800108CD8201083A
:10005000130D030829440308AD0E030807730108B4
:100060006C6900201C660120414C204558000000AE
:10007000414C2045582D415400000000414C25645E
:1000800020256420256420256420256C6C750000E3
:10009000524C204558000000524C25642025642015
:1000A000256420256420256C6C7500005445524D54
:1000B00020256420256C6C75000000004558204CFC
:1000C0004D435231202564004558204C4D43523257
:1000D0002025642025642025640000004558204C1C
:1000E0004D43523320256420256420256420256457
:1000F000000000004558204C4D4352342025642018
:10010000256420256420256400000000534D5241E1
:100110002025642025640000D2B2203A22BF00FAD4
:1001200002F1002070475242D041D2F120029140AA
:100130004140D040904041407047000038B5F8F74A
:10014000E1FB0446104DF2F77FFB286004F03CFE13
:1001500004F03FFE686004F077FF0C48C4F8B0007C
:1001600004F1B0000A4941600A4981600A49C1604E
:100170000A490161012032BD03494968896808477D
:100180000148406800680047B8650120758C000888
:10019000718C00087D8C0008818C0008858C00081B
:1001A0002DE9F04786B0044601A81421F5F722FC9A
:1001B000F1F785FF05464FF00208002601E0761CA6
:1001C00076B20A2E80F29E80022EF8D0032EF6D050
:1001D000062EF4D0524850F82670787A002806D1BE
:1001E00007F10C00406D406880470028E7D008F810
:1001F000046008F101084FFA88F8304609284FD802
:10020000DFE800F0050A4E4E10204E154E49C82179
:100210002846F2F741F943E04FF448712846F2F7D7
:100220003BF93DE032212846F2F736F938E0072065
:100230008DF80400FF208DF8050032212846F2F7E2
:100240002BF92DE03C212846F2F726F94FF0000A61
:1002500007F10C09BAF1030F22DA0020D9F8541083
:100260000969884714212846F2F716F90120D9F8C0
:1002700054100969884714212846F2F70DF9BAF19C
:10028000020F05DA062101A8D9F8542052699047D7
:100290000AF1010ADEE74FF416712846F2F7FCF87E
:1002A00007F10C0999F8151001A8D9F854205269E2
:1002B0009047002819D0D9F80C00F96800EB010A22
:1002C00099F8152001A95046F3F755FC3846FEF77A
:1002D00029FC99F81520514608EB0400F3F74BFC74
:1002E00099F9150080444FFA88F8787A00287FF44D
:1002F00066AFD9F854008068804700287FF45FAF6C
:10030000002009E0A8F10200ADF80000022200A9D7
:100310002046F3F730FC002006B0BDE8F08700006F
:100320000060002038B505000C0094F84C006428EB
:1003300002D08020F5F7ACFBF6F704FAF5F715FCD0
:10034000606928436061207C10F0F800082806D11D
:10035000A0696169084202D02000F6F798FA0748C0
:100360004078F021084202D09920F5F791FB03482C
:100370004078002801D1F5F7F2FB31BDF899002053
:100380000FB480B5BDF80B0065494880022802D340
:10039000801E088001E0002008800C229DF90A10D0
:1003A0000020F8F7B1FA032801D1022000E0012073
:1003B00002BC5DF814FB5A480121418000210180F4
:1003C00001207047574908707047000030B58DB064
:1003D00002A8F8F7FFFA524C2088401C2080618860
:1003E00080B2884232D300202080054628E0606831
:1003F000D0F8EC010121A940084220D0284606F09F
:1004000016F900281BD400EB80009FED440ADDEDB7
:100410000B0A60EE800AFDEEE00A10EE901A00AAC8
:100420008152DDED0C0A20EE800ABDEEC00A10EE0E
:10043000101A8218518000A94018012101716D1C09
:10044000172DD4DBDDE9000106F0FAF801200DB02C
:1004500030BD80B5F8F756FA314948603249C0F8E6
:10046000F01100F5F87031494160314981600FF2B7
:100470001101C1600FF225010161012002BD0000E0
:1004800010B50024274890F90000002804D106F098
:10049000F6F8002800D00124204610BDF8B5044627
:1004A0000D4640F24916287816FB004001210170E4
:1004B000287816FB00404170287816FB00400C217C
:1004C0008170287816FB0040164991F90010002928
:1004D00002D00221C17001E00121C170287816FB11
:1004E000004001210171287816FB0040C180287866
:1004F00016FB0047002006F064F83881287816FBC8
:100500000044002006F062F860812878401C2870C2
:100510000C20BDE8F24006F072B800000000C842AE
:100520001C9B00209866012081030108B703010885
:10053000CD0301080FB410B5032200210846F8F7D7
:10054000E3F9022801D102201CE00FF24000F1F78C
:1005500038FEDFF8304C00206073608220629DF826
:100560000C209DF80B109DF80A0008F0B3FE5822ED
:100570000021DFF8A40CF2F7CBFE00202074A0735A
:100580006063012010BC5DF814FB000050443A2069
:1005900053746172745065646F2D303632362D316C
:1005A0000000000080B5032200210120F8F7ACF91B
:1005B000032801D1032002BD012002BD30B58BB05C
:1005C00000A8F8F707FA05210320F8F781FA0028B8
:1005D00002D1DFF8480C0890DFF8A84BA069C56F7E
:1005E00008F00DFE207294F90800022806D13C2D77
:1005F00004D114210320F8F7EFF907E0012805D111
:10060000142D03D13C210320F8F7E6F9284680B2E7
:10061000DDED081A00A991EC030A08F0BDFCE069C1
:100620002818E06101200BB030BD10B5DFF8544B45
:1006300094F9000000283BD494F90A0094F90110C1
:10064000814229D1217B0818A07240B23D2801DBEC
:100650003C38A07294F90A100FF27000F1F7B1FD66
:100660000020E061DFF8B80B90F901004FF0FF3196
:10067000884201D1012010BD94F90110081AF8F741
:100680007BFB21F0004104F073FB40B2012801DB49
:10069000012010BD002010BDDFF8880B90F901206B
:1006A000914203D0D4E90023C0E90023002010BD0B
:1006B000E069DFF8781B884205DB0FF21C00F1F7D8
:1006C00080FD012010BD002010BD000050443A20E4
:1006D0004E5420256400000050443A204E6F546967
:1006E0006D6500002DE9F8430026DFF8984A07E021
:1006F0007A19A27252B231460FF26C00F1F761FD25
:1007000094F90A50002E21D46078461B76B294F9F1
:100710000C70002EECD53046F8F72EFB21F000418E
:1007200002460B46904699463846F8F725FB424666
:100730004B4605F017FBE3D2EA1BA272002652B229
:1007400031460FF23800F1F73CFDD9E73C2D02DBD2
:10075000A5F13C00A07294F90A100FF23400BDE834
:10076000F443F1F72EBD000050443A20636F6D70E2
:10077000312025642C2025640000000050443A20DC
:10078000636F6D70322025642C202564000000000A
:1007900050443A20435554202564000010B5DFF83A
:1007A000E4490020A07301202072002060724FF005
:1007B000FF3020700F20E07214202073002060733F
:1007C000608220626074E062206328220146DFF8C4
:1007D000600AF2F79DFDF8F795F8A061DFF8541A6A
:1007E000C0F888108830DFF8501A4160DFF84C1AE2
:1007F00081600FF28D21C1600FF64521016101205A
:1008000010BD10B582B04FF46163C1EB0114A400B8
:1008100013FB0043D3184FF47A746343DFF8104A94
:100820002360DFF860391B7C009313460A460146BB
:100830000FF20800F1F7C5FC13BD00005044204240
:1008400054202564202564202564202564000000B0
:100850002DE9F0412DED028BAAB0DFF8BC693146DD
:1008600084B068465822F3F75BF90FBC00F08CFCAB
:1008700010EE100AF8F76AFB41EC100B9FED7E8B2F
:10088000DFF8AC49656853EC102B51EC180BF8F706
:100890008BFA04F06DFA15FA80F060604FF6FF7580
:1008A000A84200D36560314684B068465822F3F709
:1008B00037F90FBC00F01EFC10EE100AF8F746FBEB
:1008C00041EC100BA76853EC102B51EC180BF8F708
:1008D0006BFA04F04DFA17FA80F0A060A84200D33A
:1008E000A5600020139002201290314684B0684623
:1008F0005822F3F715F90FBC00F090FAA1894018BF
:10090000A08180B2FF2801D3FF20A0810020139096
:1009100003201290314684B068465822F3F700F95C
:100920000FBC00F07BFA216940182061A84200D377
:1009300025610020139006201290314684B068464D
:100940005822F3F7EDF80FBC00F068FAA18A4018BE
:10095000A08280B2FF2801D3FF20A0820020139044
:1009600007201290314684B068465822F3F7D8F831
:100970000FBC00F053FAE18A4018E08280B2FF28F1
:1009800001D3FF20E082002013900820129031460E
:1009900084B068465822F3F7C3F80FBC00F03EFA63
:1009A000A1694018A061A84200D3A561002013905E
:1009B00009201290314684B068465822F3F7B0F807
:1009C0000FBC00F02BFAE1694018E061A84200D3A7
:1009D000E56114A808F017FCDFF8587DD7F82C80E3
:1009E0002398F8F7B3FA0022DFF82C3DF8F7DCF98A
:1009F00004F0BEF958FA80F0F862396B491C39638B
:100A0000B0FBF1F084F82000002013900120129038
:100A1000314684B068465822F3F782F80FBC00F0E4
:100A2000FDF9616A40186062A84200D36562F87BF4
:100A300000F0DFFA2AB0BDEC028BBDE8F081DFF8F0
:100A4000F0078189002914D10169002911D1818A17
:100A500000290ED1C18A00290BD18169002908D152
:100A6000C169002905D1406A401E8041C043C00FC2
:100A7000704701207047000000000000000059404E
:100A80002DE9F04FABB006460025DFF8A84CA07B5F
:100A9000314688420BD0012E40F09A80A06990F92F
:100AA000782090F979100FF6C440F1F78AFB14A86A
:100AB00008F0A9FBDFF860972846139001201290F8
:100AC000494684B068465822F3F72AF80FBC00F074
:100AD000A5F907469DED230AD9ED0F0A30EE600A0D
:100AE00010EE100AF8F732FA2A46DFF82C3CF8F735
:100AF0005BF904F03DF980461FFA88F8BDF89A00CA
:100B0000B9F84A10A0EB010A5FFA8AFAA06990F8D6
:100B1000D914002903D190F8D814002905D0A16A6E
:100B2000149A5118626B891AA16200F5AF61497875
:100B3000002903D190F87825002A05D0626A149B19
:100B40009A18636BD21A6262002E4ED1626A002A32
:100B500008D0002903D190F87805002802D00120A0
:100B600009F095F8A06A00280BD0A06990F8D91474
:100B7000002903D190F8D804002802D0012009F000
:100B800044F9002F02D15AEA080000D001250020C4
:100B9000E0614FF0FF302070DFF88826D4E90001D3
:100BA000C2E90001DFF8A42BC2E90001DFF87026DA
:100BB000C2E90001E07AA072A07B00284DD000209D
:100BC000A073207C002848D001206074054644E0D2
:100BD000002E04D10FF6A830F1F7F3FA67E70FF60D
:100BE000AC30F1F7EEFA2846E5E000F0A4F9002871
:100BF0001BD000A8F1F780FD204600A90522F2F7DE
:100C00007FFF28466072DFF81C26D4E90001C2E9A4
:100C1000000194F9023094F9012094F900100FF6C4
:100C20008830F1F7CEFAFFF75DFD00A8F1F764FD1B
:100C3000204600A90522F2F763FFFFF7F6FC002823
:100C40000BD0DFF8DC25D4E90001C2E90001207CEB
:100C5000002801D0012060740125012E06D1A07B5F
:100C6000012803D000F034FA0120A073012E58D1DE
:100C7000002F56D0DFF8D4BAE07B217C08430CD19A
:100C800001202074052221460BF10800F2F773FFC2
:100C9000A27861782078FFF7B4FD94F901009BF900
:100CA0000910401A411E222901D2012005E010F14D
:100CB000230F01DA012000E0002001282AD10020C2
:100CC000E0622063FFF7BBFE002823D0282200212A
:100CD000DFF85C05F2F71CFBE07B401CE073C0B260
:100CE000152809D10FF6D820F1F76BFA01206074AE
:100CF0000020E07301250DE0207C401C2074A278C8
:100D000061782078FFF77DFD052221460BF1080070
:100D1000F2F731FFFFF79CFD582214A94846F2F77D
:100D20002AFF607B012833D1608A002805D10FF6A5
:100D3000A020F1F746FA012523E0216A814218D26A
:100D4000002F02D15AEA080000D00125DFF8FCB9D3
:100D50009BF9020094F90220904212D0491C2162B2
:100D60000FF68020F1F72DFAD4E90001CBE900015C
:100D700007E000206073608220620FF67820F1F7B0
:100D800020FA012E04D1207C002801D001206074BB
:100D9000012D01D10020E061A06990F879000028C0
:100DA00006D10020E061012D01D100F091F900256C
:100DB0001498606328462BB0BDE8F08F10B5DFF8BB
:100DC00074090021C161032205210020F7F79CFD71
:100DD000044600F007F8204610BD0322052101203B
:100DE000F7F792BD00B597B000A808F00CFA5822AA
:100DF00000A9DFF84409F2F7BEFE012017B000BDDC
:100E0000DFF83009406A7047DFF8280900214162A5
:100E10007047DFF820090021816270470FB430B5B8
:100E200097B09DF9C0409DF9C400002501280BD161
:100E300008F0E1FA1A99884202D3451AEDB270E03F
:100E40008038451AEDB26CE000A808F0DCF9641EA9
:100E5000082C66D8DFE804F02905111D2936424E1A
:100E60005A0001981B99884201D3451A59E0DFF8CE
:100E7000E0281018401A451C53E002981C9988423B
:100E800001D3451A4DE0DFF8C8281018401A451C58
:100E900047E003981D99884201D3451A41E0DFF8E5
:100EA000B0281018401A451C3BE000981A99884257
:100EB00001D3451A35E0DFF8981808181A99401A36
:100EC000451C2EE004981E99884201D3451A28E05B
:100ED000DFF87C281018401A451C22E005981F995D
:100EE000884201D3451A1CE0DFF864281018401A24
:100EF000451C16E006982099884201D3451A10E057
:100F0000DFF84C281018401A451C0AE00798219970
:100F1000884201D3451A04E0DFF834281018401A3B
:100F2000451C284617B030BC5DF814FBDFF80408F8
:100F3000012141727047DFF8FC07407A704708F0E2
:100F400075B9DFF8F017792802D378224A8200E0D9
:100F5000488201224A7301460FF6AC00F1F731B91D
:100F600010B5040001D1012402E0072C00D30624AF
:100F700021460FF6A800F1F724F9641E052C2DD8A0
:100F8000DFE804F0030A11181F26DFF8A80737214D
:100F9000C1723C21017321E0DFF898071921C17269
:100FA0001E2101731AE0DFF88C070F21C172142192
:100FB000017313E0DFF87C070A21C1720F2101736E
:100FC0000CE0DFF870070721C1720C21017305E006
:100FD000DFF860070521C1720A210173DFF85407A9
:100FE000C17A8172BDE81040FFF77CBBDFF82C07A7
:100FF000704700EB80018800421CDFF820078C4915
:1010000092B20B681B0E1354521C92B20B681B0C4D
:101010001354521C92B20B681B0A1354521C92B206
:101020000B681354521C92B24B681B0A1354521C87
:1010300092B24B681354521C92B28B681B0A135421
:10104000521C92B28B681354521C92B28B89135467
:10105000521C92B20B691B0A1354521C92B20B69B8
:101060001354521C92B28B8A1354521C92B2CB8AE4
:101070001354521C92B28B691B0A1354521C92B225
:101080008B691354521C92B2CB691B0A1354521C25
:1010900092B2CB691354521C92B291F8203013547F
:1010A000521C92B24B6A1B0A1354521C92B2496AE8
:1010B0001154DFF88006511C8182704710B5DFF8AB
:1010C0007446A18A0FF26070F1F77BF8A08A10BD18
:1010D00080B5282200215648F2F71AF9DFF85406A5
:1010E0000021C1730121818200210174C162016369
:1010F00001BD00000FB400B597B000A808F083F858
:101100009DED090ADDED210AB4EE600AF1EE10FA58
:1011100002DB30EE600A05E09FED431A71EE600AD3
:1011200030EE800A10EE100AF7F710FFDFF8F02516
:10113000DFF8F03508F0AAFEF7F730FFF7F706FF03
:101140000022DFF8E435F7F72FFE03F011FE00EE82
:10115000100AB8EEC00A10EE100AF7F7F7FEDFF833
:10116000C025DFF8C835F7F71FFEDFF8C425DFF824
:10117000E43508F08BFEF7F711FF00EE100A17B008
:101180005DF814FB045F01200FB400B597B000A810
:1011900008F039F89DED0E0ADDED260AB4EE600A7E
:1011A000F1EE10FA02DB30EE600A05E09FED1E1A48
:1011B00071EE600A30EE800A10EE100AF7F7C6FEF4
:1011C000DFF85C25DFF85C3508F060FEF7F7E6FE37
:1011D000F7F7BCFE0022DFF85035F7F7E5FD03F026
:1011E000C7FD00EE100AB8EEC00A10EE100AF7F7BD
:1011F000ADFEDFF82C25DFF83435F7F7D5FDDFF845
:101200003025DFF8503508F041FEF7F7C7FE00EE55
:10121000100A17B05DF814FB205B012000007A442F
:10122000C8650120C06501200024744940771B0077
:10123000C460012035050108A5050108BD050108A8
:101240002DE9F0472DED068BAAB006460D4614A8F1
:1012500007F0D9FF40F24914287814FB00600121FF
:101260000170287814FB0060DFF8C874797B0129CD
:101270000CD103214170287814FB00600121C1705A
:10128000788A002804D10020787301E001214170A0
:10129000287814FB006003218170787C012820D11C
:1012A000387C00281DD0297814FB0161C0220A7106
:1012B000DFF868140870287814FB0068FFF7FEFE5A
:1012C000A8F83000287814FB0064FFF78FFEC4F8FC
:1012D00032002878401C2870FFF7FAFE002078744E
:1012E00015E20DF18C099FED868B9FED879BDFF852
:1012F00048740020139001201290394684B068464B
:101300005822F2F70DFC0FBCFFF788FD0A28287859
:1013100014FB006080F0FC8000210171287814FB30
:10132000006898F804A008461390022012903946ED
:1013300084B068465822F2F7F3FB0FBCFFF76EFD4E
:1013400040EA0A0088F80400287814FB00680020AE
:10135000139003201290394684B068465822F2F761
:10136000DFFB0FBCFFF75AFD88F80500287814FB57
:1013700000680020139004201290394684B068461B
:101380005822F2F7CDFB0FBCFFF748FD88F80600A6
:10139000287814FB0068002013900520129039462D
:1013A00084B068465822F2F7BBFB0FBCFFF736FD4E
:1013B00088F80700394684B068465822F2F7B0FB37
:1013C0000FBCFFF7E1FE10EE100AF7F7BFFD41EC8E
:1013D000100B287814FB006853EC102B51EC190B00
:1013E000F7F7E2FC03F0C4FCA8F80E00287814FB21
:1013F00000682398F7F7AAFD53EC182BF7F7D4FCF5
:1014000003F0B6FC88F81000287814FB0060B9F8E7
:101410000E104174394684B068465822F2F780FBBA
:101420000FBCFFF767FE10EE100AF7F78FFD41ECD7
:101430001A0B287814FB006853EC1A2B51EC190B8B
:10144000F7F7B2FC03F094FC88F81200287814FB3C
:101450000068D9F80800F7F779FD53EC182BF7F777
:10146000A3FC03F085FC88F81300287814FB0068BF
:101470000020139006201290394684B06846582206
:10148000F2F74EFB0FBCFFF7C9FC88F8080028787C
:1014900014FB00680020139007201290394684B096
:1014A00068465822F2F73CFB0FBCFFF7B7FC88F800
:1014B0000900287814FB006800201390082012907F
:1014C000394684B068465822F2F72AFB0FBCFFF772
:1014D000A5FC88F80A00287814FB0064002013900B
:1014E00009201290394684B068465822F2F718FB5A
:1014F0000FBCFFF793FCE0722878401C287004E1D1
:1015000000000000000024400000000000005940DE
:1015100080210171287814FB0068002013900220BC
:101520001290394684B068465822F2F7F9FA0FBC97
:10153000FFF774FCC8F80500287814FB0068002049
:10154000139003201290394684B068465822F2F76F
:10155000E7FA0FBCFFF762FCC8F80900287814FB13
:1015600000680020139004201290394684B0684629
:101570005822F2F7D5FA0FBCFFF750FCC8F80D005F
:10158000287814FB0068002013900520129039463B
:1015900084B068465822F2F7C3FA0FBCFFF73EFC4E
:1015A000C8F81100394684B068465822F2F7B8FAF4
:1015B0000FBCFFF7E9FD10EE100AF7F7C7FC41EC8E
:1015C000100B287814FB006853EC102B51EC190B0E
:1015D000F7F7EAFB03F0E2FBC8F82700287814FBD2
:1015E00000682398F7F7B2FC53EC182BF7F7DCFBF5
:1015F00003F0BEFB88F82B00287814FB0060B9F8D4
:101600000E1080F82C10394684B068465822F2F744
:1016100087FA0FBCFFF76EFD10EE100AF7F796FC85
:1016200041EC1A0B454A464B04F0B4FB06D8454A38
:10163000454B04F097FB01D29FED47AB287814FB94
:10164000006853EC1A2B51EC180BF7F7ADFB03F0C5
:101650008FFBA8F82D00287814FB0068D9F8080043
:10166000F7F774FC53EC182BF7F79EFB03F080FBA5
:1016700088F82F00287814FB0068002013900620BB
:101680001290394684B068465822F2F749FA0FBCE6
:10169000FFF7C4FBC8F81500287814FB0068002089
:1016A000139007201290394684B068465822F2F70A
:1016B00037FA0FBCFFF7B2FBC8F81900287814FB03
:1016C00000680020139008201290394684B06846C4
:1016D0005822F2F725FA0FBCFFF7A0FBC8F81D004F
:1016E000287814FB006400201390092012903946DA
:1016F00084B068465822F2F713FA0FBCFFF78EFB4E
:10170000C4F821002878401C2870FFF76BFB2AB032
:10171000BDEC068BBDE8F087000024407C39012039
:101720007B14AE47E17A743F00005940E17A843F70
:101730002D431CEB045F0120205B0120B81E85EBCC
:1017400051B89E3F9A9999999999B93F006401209F
:1017500080969800E2361A3F9A9999999999B93FDB
:1017600080B5C046C046012002BD00005044205252
:1017700065662045282564292C4928256429000010
:101780005044203A206C63646F6E00005044203A4D
:10179000206249734150536C656570696E672077AC
:1017A000726F6E672025640050443A54696D654E2F
:1017B0006F746920256420256420256400000000E2
:1017C00050442042542042462046554C4C000000D4
:1017D00050443A20526571205065646F496E666FBF
:1017E0003100000050443A207574696D65722025FF
:1017F0006400000050443A20526571205065646FC7
:10180000496E666F3200000050443A205374617292
:1018100074204461746120256400000050443A2023
:10182000555420256400000050443A204241544C55
:10183000454E4754482025640000000010B5DFF8ED
:101840009C4C4FF4287200212046F1F761FDFF20E7
:101850002070E07284F86202DFF8C00C0021417051
:1018600010BDF8B501240B2824D101290ED1DFF8D1
:101870006C3CD31893F954522E46DFF8A47CD75D04
:10188000BE4210DA6D1C83F8545230E002292ED18A
:10189000DFF8483CD31893F95452012D03DB6D1E39
:1018A00083F8545223E0DFF8343CD318002483F843
:1018B00054421CE00A281AD1012908D1DFF81C3C47
:1018C000D31803F515735D796D1C5D710FE0022966
:1018D0000DD1DFF8083CD31803F5157393F90550C3
:1018E000012D02DB6D1E5D7101E000245C71002C96
:1018F00005D1134602460FF20C00F0F762FC2046B9
:10190000F2BD000041542D25643A25642025640071
:10191000DFF8C81B81F85E0270470FB42DE9F04173
:1019200094B00124DFF8F45BE868DFF8B06B90F85E
:101930001014002957D190F81104002853D10FF248
:101940002C20F0F73EFCB4208DF8020046208DF8E4
:10195000030020468DF8040000208DF82C000320A1
:101960000C900DF1350000A91822F2F7C9F80A20F1
:101970008DF834000BA8F7F7C1F8002801D1022038
:10198000EEE000A8F0F7B8FE9DF80000B0779DF9F2
:101990000100F0779DF9021086F82010BDF90320B0
:1019A000A6F821209DF900304FF46167C0EB001CC0
:1019B0004FEA8C0017FB030040FA81F04FF47A7174
:1019C00001FB0020C6F80200C6F80D000020A86147
:1019D000E8702870A870687028712422014606F506
:1019E0002870F1F795FC9DF86A70A046012F1DD173
:1019F000DDF86B00202805D0D6F817100843C6F88C
:101A000017000BE0204607E0D6F8171008FA00F29E
:101A10001143C6F81710401C0528F5D3F07E9DF938
:101A20006F1008FA01F10843F0764EE0B81990F90A
:101A30005412002949D190F95902002845D1022FAA
:101A40002DD100A8F0F758FE9DF900004FF4616118
:101A50009DF90120C2EB02139A0011FB00209DF9B1
:101A6000021040FA81F04FF47A71BDF9032001FBB6
:101A70000020C6F89302C6F88F0206F12B0006F18B
:101A80001E010522F2F73CF84FF49660B083DFF8B0
:101A9000CC0CC6F8870200206861286115E0032F8E
:101AA00013D1DDF86B00C6F82300BDF870004FF4C9
:101AB0007A714843C6F827000020C6F89B0286F8D2
:101AC0006C0286F86D0286F89F0208FA07F0B17D75
:101AD0000143B175317800290FD0012F08D108FAE0
:101AE00001F1DDF86B20914202D1002186F86112EC
:101AF00096F86912084386F869023A46214696F834
:101B00005E02FFF7AEFE002800D10224E86896F9D5
:101B10005C120A9196F95B12099196F95A12089192
:101B200096F95912079196F95712069196F956129D
:101B3000059196F95512049196F95412039190F873
:101B40001114029190F810040190B08B0090F37E74
:101B5000D6F81720B17D0FF22400F0F732FB2046B3
:101B600014B0BDE8F0015DF814FB000041542D52A3
:101B700045563134313231320000000041542D419C
:101B80004C2025642025642025642025642C4154A4
:101B9000202564202564202564256425642564208F
:101BA000256425642564256400000000F0B595B027
:101BB000FEF742FA06460124002E00F08180DFF88D
:101BC0001C5905F51577B2780221B87AFFF749FE5E
:101BD000002800D10324B07801282AD1D6F80300C8
:101BE00005F21702202810D0D5F817108143C5F848
:101BF00017101079012396F90770BB4098431071B4
:101C00000FF25010F0F7DDFA03E00020C5F81700DE
